:020000040000FA
:100000000208AC021003FFFFFFFFFF02100BFFFF0F
:10001000FFFFFF021013FFFFFFFFFF02101BFFFF98
:10002000FFFFFF021023FFFFFFFFFF02102BFFFF68
:10003000FFFFFF021033FFFFFFFFFF02103BFFFF38
:10004000FFFFFF021043FFFFFFFFFF02104BFFFF08
:10005000FFFFFF021053FFFFFFFFFF02105BFFFFD8
:10006000FFFFFF021063FFFFFFFFFF02106BFFFFA8
:10007000FFFFFF021073FFFFFFFFFF02107BFFFF78
:10008000FFFFFF021083FFFFFFFFFF02108B8C00BA
:100090000000000000000400000001C00300010097
:1000A0000000880000008B00000078FFFFFF0010B8
:1000B000000074FC12081C53BEFBE59DA2E650FA3A
:1000C0000078F8790100E824FF18E934FFF9E849DD
:1000D00070F375C6807480659E70FA43BE049062AA
:1000E000707408F0D29043FE01D29143FE0253F5A2
:1000F000E6D2A043FF01C2A343FF0843F708C2A40E
:1001000043FF10794A1201B57401F5D575D4018009
:1001100035851882851983E0F8A3E0F97402120886
:10012000D4E8F0A3E9F07508017509007808120811
:100130006D74021208D4AC82AD837A227B0412065D
:100140002774021207E97508047509007808120877
:100150006D74021208D4AC82AD837A887B00790278
:100160001205B074021207E9851882E0F8A3E0F9DD
:1001700074021208D4E0687003A3E06970090210E9
:100180000074041207E922E849601D1202968A08E9
:100190008B09A808A909851882851983E06870036E
:1001A000A3E0697003020111798C1203A8E970962B
:1001B0001201CB8091781075B60FE5B4A2E750FA22
:1001C000E5BBC39940F118E870ED2274F11206A264
:1001D00074F012081C7E007F0479691201B575085D
:1001E0000C8E09780812086D74061208D4858208EE
:1001F000858309780812086D79019001091208C8F1
:100200001204C3EF1207E990010D780C12089D80CB
:100210006D750804750900780812086D74021208DB
:10022000D4858208858309780812086D7901120443
:10023000B51207E9EEF8EF5401F9E84970108E089D
:100240008F097409780812088EA90812068B7508A0
:1002500001750900780812086D74021208D4AC8286
:10026000AD83EEFAEFFB12062774021207E9EE24C3
:10027000010EEF3400FF900111780C12085A740639
:100280001208D4780C1207AF508774101207E98057
:10029000007F0802075074F11206A274F312081CC2
:1002A000750800750900750A0C750B00780A1208AC
:1002B0006D74031208D485820A85830B780A1208AC
:1002C0006D79009001091208C81204BD1207E97483
:1002D000031208D4C082C083900115780C12089DC7
:1002E000D083D082780C12087E40067A007B008092
:1002F0007690010D780C12089D803E750A01750BF1
:1003000000780A12086D74021208D485820A858367
:100310000B780A12086D79001204B51207E98518E6
:1003200082851983E0F9AA08AB0912036C8A088B4D
:1003300009900119780C12085A74031208D4780C29
:100340001207AF401490011D780C12083270AC9067
:100350000121780C12089D80D8E4F9AA08AB091293
:10036000036CE4F912036C740D02028CC008C0091E
:100370007C088A088B09740F780812088EEAC33348
:10038000FAEB33FBE9A2E7500474014AFAE508A24C
:10039000E0500874216AFA74106BFBE9C333F91C4E
:1003A000EC70CFD009D0082274ED1206A274F112BD
:1003B000081C890C7E007F0075080C8E09780812D5
:1003C000086D74051208D48582088583097808129F
:1003D000086D7901AA0CE4FBFCFD1204BD1207E9CB
:1003E00090010D781012089D806085100885110914
:1003F00085120A85130B900125780812085A90017E
:100400001178081207AF503A75080175090078088D
:1004100012086D74021208D4858208858309780851
:1004200012086D7901AA10AB11AC12AD131204BD04
:100430001207E9851882851983E0F9EEFAEFFB12BD
:1004400004A9900119781012085A74051208D4787A
:10045000101207AF50947900EEFAEFFB12036C799B
:10046000001204A9750802750900780812086D7455
:10047000031208D4858208858309780812086D79EB
:100480000190011D1208C81204BD1207E97401127F
:1004900008D4E06E7003A3E06F70047900800279E5
:1004A00001740F1207E902056512036C8A088B09B3
:1004B000AE08AF0922AA0CAB0DAC0EAD0F1204C3EF
:1004C00074042274ED1206A28A0C8B0D8C0E8D0F13
:1004D00074131208D4E0FCA3E0FD74151208D4E0F4
:1004E000F508A3E0F509E9603FAE08AF098C828DFD
:1004F00083120577C2A0790B12059C1208038510A0
:1005000008120559790012056A800953FFF712078E
:10051000A1E9F0A3EEF8EFF9E824FF1EE934FFFFAC
:10052000E84970E7D2A0802E900129780C12085A71
:10053000780812086D850C08850D09AA08E509548C
:1005400007FB740B780C120803850C08A908120528
:10055000B074021207E902056512058E850C08A920
:100560000812056A227F0C020750EEC0E043FF0824
:10057000120790D0E0FE22C2A0790512056A53FF4F
:10058000F71207A1E9A2E040F5D2A0000022A908D5
:1005900012056A850D09A90912056A2212056A85E4
:1005A0000C10850D11850E12850F13741078102212
:1005B00074F51206A28908740B1208D4E0FEA3E0B9
:1005C000FF740F5508F50A750B00740B780A1208B2
:1005D00047EA2400F8EB3480F9E82400E9350BF908
:1005E000E5C7F509E508C4540FFAE5C754F84AF51C
:1005F000C7801C88828983E08C828D83F088828901
:1006000083A3A882A9838C828D83A3AC82AD83EE61
:10061000FAEFFBEA24FF1EEB34FFFFEA4B70D485B0
:1006200009C77F0402075074F71206A27409120862
:10063000D4E0F508A3E0F509ED900101F0ECA3F09A
:10064000A37462F0A37473F0A3E0541FF0E50833C1
:100650003354FCA3F07406780812088EE508900164
:1006600005F09001077412F0A37442F075D1FE7585
:10067000D601EA906271F0EBA3F0906270E0D2E1F3
:10068000F0E0A2E740FB7F02020750C082C083E98E
:10069000C333906272F0906270E0D2E0F0D083D009
:1006A00082222518C582C0E0E51934FFC583C0E069
:1006B000E518C3958224F910AF088583198582183F
:1006C0008008858319858218D2AFCEF0A3E520F08B
:1006D000A37808E608F0A3DEFAEFF0A3E58124FB97
:1006E000F8E608F0A3E608F0A30808E608F0A3E699
:1006F00008F0A315811581D0E0FED0E0F815811532
:1007000081E8C0E0EEC0E0221208E3B9000302076E
:100710004AE4900101780979018002F0A3D8FCD95C
:10072000FA900109AA82AB8390008E782579018026
:1007300015E493A3AC82AD838A828B83F0A3AA8253
:10074000AB838C828D83D8E9D9E71200B21208DE20
:10075000851983851882E0A3FEE0A3F5207808E0E0
:10076000A3F608DFFAE0A3FFE0A3C0E0E0A3C0E047
:10077000E0A3C0E0E0A3C0E010AF08858218858345
:10078000198008858218858319D2AFD083D0822240
:10079000E97A0833C2A492A300D2A4DAF600C2A474
:1007A000227A08A2A3D2A43300C2A4DAF6F922C0A6
:1007B00008C3E096F50808A3E096420808A3E0966F
:1007C000420808A3E09645087001D3D008222518F6
:1007D000F58210AF08F518400215198008F5184089
:1007E000021519D2AF85198322C0D0251810AF0881
:1007F000F518500205198008F51850020519D2AFF6
:10080000D0D0226016080808C6C313C618C613C67F
:1008100018C613C618C613C6D5E0EA22251810AFAD
:1008200008F518400215198008F51840021519D26C
:10083000AF22E066701008A3E066700A08A3E066C5
:10084000700408A3E06622700422600D18C6C3334A
:10085000C608C633C6D5E0F41822E026F608A3E0A1
:1008600036F608A3E036F608A3E036F622740280D6
:1008700000C0E0F4041207CED0E01208BB22C3E0AF
:100880009608A3E09608A3E09608A3E09622600CE1
:1008900008C6C313C618C613C6D5E0F422E0F6088E
:1008A000A3E0F608A3E0F608A3E0F62275D00075F1
:1008B0008140751801751901020708CAC0E0E6F009
:1008C000A308DAFAD0E0FA22E0FAA3E0FBA3E0FC06
:1008D000A3E0FD222518F582E43519F583220000F6
:1008E0000080FB790122FFFFFFFFFFFFFFFFFFFFFB
:1008F000FFFFFFFFFFFFFFFFFFFFFFFFFFFFFFFF08
:10090000FFFFFFFFFFFFFFFFFFFFFFFFFFFFFFFFF7
:10091000FFFFFFFFFFFFFFFFFFFFFFFFFFFFFFFFE7
:10092000FFFFFFFFFFFFFFFFFFFFFFFFFFFFFFFFD7
:10100000021BA50211E1FFFFFFFFFFFFFFFFFFFF34
:10101000FFFFFF021478FFFFFFFFFF0214B9FFFF7D
:10102000FFFFFFFFFFFFFFFFFFFFFF021A1BFFFF96
:10103000FFFFFFFFFFFFFFFFFFFFFF02145FFFFF48
:10104000FFFFFFFFFFFFFFFFFFFFFF022FE0FFFF9C
:10105000FFFFFF021112FFFFFFFFFF022FE1FFFF63
:10106000FFFFFF022FE2FFFFFFFFFFFFFFFFFFFF7A
:10107000FFFFFF02148FFFFFFFFFFFFFFFFFFFFFD8
:10108000FFFFFF021176FFFF99E0FFFFA55ADDB3D6
:1010900001000010F8F8AD0001FF0FF320F320F37A
:1010A00020F320AF1FA91FF320D33100000000352B
:1010B00032000000000C0000000C0001FFFF0101E5
:1010C00001004F0500000001CA05E8036400640048
:1010D000B80102050000000205020701051E020515
:1010E0001E020A0A03B80B02803E010201252502F6
:1010F0000A1401E002020612727373693A2020207A
:1011000020202064426D20206C71693A20307820C4
:101110002000C0E074F21215ACA2AFE433FED2AFEF
:10112000E5A7FFE5A1F5085F541060061228D37506
:10113000A1EFE5085F540860081228D975A1F7806F
:101140002BEFA2E0C0D0E508A2E092F0121AC91578
:101150008182F05017906198E0F8900B31E0C398CD
:10116000A2D265D0335002E8F075A1FEEEA2E09263
:10117000AF7F0102160BC0E074F21215ACA2AFE40F
:1011800033FED2AF9061A4E0F8759B00E59158540E
:101190000860087591F712291B802AE591585410B0
:1011A00060087591EF122921801BE8A2E0C0D0E50C
:1011B00091A2E092F0121AC9158182F05007E0C2A4
:1011C000E0F0122A6B9061A3E0F8E5E9585404605E
:1011D0000E122A4175E9FB906193E0A2E640F2808D
:1011E0008BC0E074F21215ACA2AFE433FED2AF9024
:1011F00061A5E0F8E5BF585404600675BFFB122AEC
:101200008302116C000000000000000000000000DC
:101210000000000000000000000022121204121260
:1012200004121204121204121204121204121204F2
:1012300012120412120412120412120412120412D4
:1012400012041212041212041212041212041212C4
:1012500004121204121204121204121204121204C2
:10126000000000000000000000000000000000007E
:101270000000000000002212121B12121B121204A6
:10128000121204121204000000000000000000000E
:101290000000000000000000000000002212121BED
:1012A00012121B12121B12121B121204121204121F
:1012B0001204000000000000000000000000000018
:1012C000000000000000000022C3E498F8E499F94F
:1012D00012130A8026C3E49AFAE49BFBE920E7E9AB
:1012E00012130AE498F8E499F922C3E498F8E4990F
:1012F000F912130AE498F8E499F9C3E49AFAE49B22
:10130000FB22EB20E7CFE920E7E0B90010BB0008A3
:10131000E88AF084F8AAF022E4FBC8FA22EB7022F3
:101320007B10C833C8C933C9335007C39AC3DBF233
:1013300080069A50012ADBEAC833F4C8C933F4C9DD
:10134000FA2275F008E4C833C8C933C933C99AC949
:101350009B5004C92AC93BD5F0ECFBC833F4C8E460
:10136000C9FA22080808EAC0E0EBC0E086F0E7A46A
:10137000FA180986F0E7A42AFA180986F0E7A42AE1
:10138000FA180986F0E7A42AFA1986F0E7A4FBE523
:10139000F02AFA190886F0E7A42BFBE5F03AFA19CF
:1013A0000886F0E7A42BFBE5F03AFA18180986F056
:1013B000E7A4C5F02BFBE43AFA1908E7C5F0C6A488
:1013C00026F6E5F03BFBE43AFA1886F0E7A4F6E5EA
:1013D000F00826F6E43B08F6E43A08F6D0E0FBD045
:1013E000E0FA22D083D082ECC0E0EDC0E0EEC0E0B5
:1013F000EFC0E0E493A3FCE493A3FDE493A3FEE435
:1014000093A3FFEF4E4D4C6015121824EC24FFFC03
:10141000ED34FFFDEE34FFFEEF34FFFF80E5E49393
:10142000A3FCE493A3FDE493A3FEE493A3FFEF4E98
:101430004D4C60151218BDEC24FFFCED34FFFDEEA1
:1014400034FFFEEF34FFFF80E5D0E0FFD0E0FED0B8
:10145000E0FDD0E0FCE493A3C0E0E493C0E022C050
:10146000E074F21215AC900B1D1214B16006121448
:10147000AB122FE3C2E9802EC0E074F21215AC90DB
:101480000B1F1214B160061214AB122FE38017C0A9
:10149000E074F21215AC900B211214B16006121414
:1014A000AB122FE3C2EA7F0102160BE0F5838882BC
:1014B00022E0F8A3E0F9E84922C0E074F21215AC8A
:1014C000900B231214B160061214AB122FE380D6D6
:1014D000E4CFC0E0E4CEC0E0E4CDC0E0E4CCC0E0C6
:1014E00075F020C3E633F608E633F608E633F6086F
:1014F000E633F6181818EC33FCED33FDEE33FEEF4F
:1015000033FFC3EC9709ED9709EE9709EF97191987
:1015100019400FFFEC97FC09ED97FD09EE97FE19B6
:101520001906D5F0BEECF709EDF709EEF709EFF76C
:10153000191919D0E0FCD0E0FDD0E0FED0E0FF2288
:101540002518C582C0E0E51934FFC583C0E0E51861
:10155000C3958224F810AF08858319858218800806
:10156000858319858218D2AFCEF0A3E520F0A37849
:1015700008E608F0A3DEFAEFF0A3E58124FAF8E626
:1015800008F0A3E608F0A3E608F0A30808E608F0D0
:10159000A3E608F0A315811581D0E0FED0E0F81590
:1015A0008115811581E8C0E0EEC0E022C0D0251889
:1015B000C582C0E0E51934FFC583C0E0E518C395D6
:1015C0008224F310AF0885831985821880088583EB
:1015D00019858218D2AFC8F0A3E9F0A3EAF0A3EB13
:1015E000F0A37908E709F0A3D8FAECF0A3EDF0A393
:1015F000EEF0A3EFF0A3D0E0F0A3D0E0F0A3D0E0B2
:10160000F0A3E520F0A3E5F0F0A322851983851867
:1016100082E0C0E0A3E0F9A3E0FAA3E0FBA378082E
:10162000E0F608A3DFFAE0FCA3E0FDA3E0FEA3E000
:10163000FFA3E0C0E0A3E0C0E0A3E0F5D0A3E0F5A5
:1016400020A3E0A3F5F010AF0885831985821880E8
:1016500008858319858218D2AFD082D083D0E0F874
:10166000D0E032121C07B900030216A5E490030172
:10167000781C79108002F0A3D8FCD9FA90121CAA29
:1016800082AB83901098787B79018015E493A3ACAA
:1016900082AD838A828B83F0A3AA82AB838C828DF6
:1016A00083D8E9D9E77582A77583A37403121961FA
:1016B0007582DB75832F74001219610575F0108E29
:1016C0001A8F1B85821F85831E851882851983E0EA
:1016D000CEA3E0CF851F82851E83EBC9EAC8EDCB80
:1016E000ECCAC3E833C8E933C9EA33CAEB33CBC326
:1016F000EA9EF51DEB9FF51CB35004AB1CAA1DEC34
:1017000033CCED33CDD5F0DAAE1AAF1B22D083D077
:1017100082ECC0E0EDC0E0E493A3FCE493A3FDED14
:101720004C600D1217E5EC24FFFCED34FFFD80EF5B
:10173000E493A3FCE493A3FDED4C600D121892EC2E
:1017400024FFFCED34FFFD80EFD0E0FDD0E0FCE4B1
:1017500093A3C0E0E493C0E022851983851882E05A
:10176000A3FEE0A3F5207808E0A3F608DFFAE0A3E3
:10177000FFE0A3C0E0E0A3C0E0E0A3C0E0E0A3C0BE
:10178000E0E0A3C0E010AF088582188583198008C7
:10179000858218858319D2AFD083D082021967D091
:1017A00083D082E9C0E0E493A3C386F0C5F095F04E
:1017B000F908E493A386F0C5F095F0700BE493A3C9
:1017C000C3994005E9048002A3E475F002A42582D0
:1017D000F582E5F03583F583D0E0F9E493A3C0E02A
:1017E000E493C0E022C0E0C3E493960874019396AA
:1017F00018400FE49366700808740193661870002F
:101800007019A3A3C3E49396087401939618A3A335
:10181000400DD0E0D0E0D0E0021749A3A3A3A3A3DA
:10182000A3D0E022C0E0C0F088F0121AB5A8F040C2
:1018300007121A02A8F0701AA3A3A3A3121AB5A83C
:10184000F0A3A3A3A34013D0F0D0E0D0E0D0E002F7
:101850001449A3A3A3A3A3A3A3A3A3A3D0F0D0E05D
:10186000227404800474028000CCC0E0EDC0E0E586
:1018700018C39CCCAD1950011D10AF068C188D19E2
:1018800080068C188D19D2AF121902D0E0FDD0E07D
:10189000FC22C0E0C0F088F0E49366700808740190
:1018A0009366187000A8F0A3A3700BD0F0D0E0D01E
:1018B000E0D0E0021749A3A3D0F0D0E022C0E0C0FE
:1018C000F088F0121A02A8F0A3A3A3A3700BD0F023
:1018D000D0E0D0E0D0E0021449A3A3D0F0D0E022C1
:1018E000CAC0E0E493A3C582CCC582C583CDC583BD
:1018F000F0A3C582CCC582C583CDC583DAE5D0E02F
:10190000CA22CAC0E0E0A3C582CCC582C583CDC5CA
:1019100083F0A3C582CCC582C583CDC583DAE6D06A
:10192000E0CA22C008C3E096F50808A3E096420882
:1019300008A3E096420808A3E09645087001D3D0BA
:1019400008227009080808226016181818C6C33340
:10195000C608C633C608C633C608C633C6D5E0EACD
:1019600022C09FF59FE473D09F22D083D082C09F76
:10197000E493C0E0740193C0E0740293F59F2225C4
:1019800018F58210AF08F518400215198008F518EF
:1019900040021519D2AF851983227404800A74039A
:1019A0008006740280027401C0E0F40412197FD032
:1019B000E0121BE222BB0102E722C082C0838982BF
:1019C0008A83BB0003E08002E493D083D08222C0EC
:1019D000D0251810AF08F518500205198008F51821
:1019E00050020519D2AFD0D0226016080808C6C32D
:1019F00013C618C613C618C613C618C613C6D5E034
:101A0000EA22E4936670130874019366700C0874FC
:101A10000293667005087403936622C0E0C0D0E8A4
:101A2000C0E0E5A8D2AFC2C7A2E792AFD0E0F8D03D
:101A3000D0D0E032C3E0C696F608A3E0C696F6081A
:101A4000A3E0C696F608A3E0C696F622251810AFC6
:101A500008F518400215198008F51840021519D22A
:101A6000AF22E066701008A3E066700A08A3E06683
:101A7000700408A3E06622C3E09608A3E09608A3DA
:101A8000E09608A3E096A2D265D03322E7667010F4
:101A90000809E766700A0809E76670040809E7663E
:101AA00022C3E096F008A3E096F008A3E096F008C1
:101AB000A3E096F022C3E493960874019396087409
:101AC000029396087403939622C0E0E8C0E0E58193
:101AD00024FCF8E6A2E7D0E0F8D0E022700422600F
:101AE0000D18C6C333C608C633C6D5E0F41822E0C5
:101AF00026F008A3E036F008A3E036F008A3E036AD
:101B0000F022E657F60809E657F60809E657F60800
:101B100009E657F622E056F608A3E056F608A3E0D9
:101B200056F608A3E056F622E026F608A3E036F6BD
:101B300008A3E036F608A3E036F622E056F008A344
:101B4000E056F008A3E056F008A3E056F022E6477E
:101B5000F60809E647F60809E647F60809E647F6F3
:101B600022E627F60809E637F60809E637F60809F7
:101B7000E637F622E4C396F608E496F608E496F60D
:101B800008E496F622C6F4C608C6F4C608C6F4C62B
:101B900008C6F4C622C3E09608A3E09608A3E09620
:101BA00008A3E0962275D00075814075180175195B
:101BB0000300021663E0F608A3E0F608A3E0F608C7
:101BC000A3E0F622600C08C6C313C618C613C6D518
:101BD000E0F422E6F008A3E6F008A3E6F008A3E6A6
:101BE000F022CAC0E0E6F0A308DAFAD0E0FA22E078
:101BF000FAA3E0FBA3E0FCA3E0FD22EAF0A3EBF0F4
:101C0000A3ECF0A3EDF022E5C754F84401F5C77941
:101C100001222518F582E43519F58322C2AF75D665
:101C20009F0200002212196A87D40112196AADD4EA
:101C30000112196AE8D40112196A31D50112196A20
:101C400082D50112196A32D60112196AEAD6011236
:101C5000196AB2D70112196A8FD80112196A15D9F7
:101C60000112196A24D90112196A2FD90112196AAD
:101C700040DA0112196A51DA0112196AD6DA011230
:101C8000196A65DB0112196ABDDB0112196A87DC6A
:101C90000112196AB8DC0112196AF5DC0112196A1D
:101CA00002DD0112196A91DE0112196AF4DF0112D4
:101CB000196A30E00112196A43E10112196A8AE3D4
:101CC0000112196A95E30112196A9FE30112196A58
:101CD000AAE30112196AB4E30112196ABEE3011200
:101CE000196AC9E30112196AD4E30112196A23E4DB
:101CF0000112196A05E60112196A8BE60112196AC6
:101D000066E70112196A5FEA0112196AB4EA011260
:101D1000196ADCEA0112196A14EC0112196A5CEC06
:101D20000112196AB1EC0112196AB2ED0112196AB5
:101D30004AEE0112196ACCEE0112196A6CEF011217
:101D4000196A3B340012196A74340012196A4E364B
:101D50000012196A8D360012196AD7360012196AF4
:101D60007C370012196ADB370012196A0F3800122B
:101D7000196A7C380012196A99390012196AA13A55
:101D80000012196A5C3B0012196A9E3E0012196A21
:101D9000473F0012196A3B400012196A9C4000122A
:101DA000196AB9410012196AC6430012196A7D44C2
:101DB0000012196A87440012196AB5440012196AA0
:101DC0008C450012196A53460012196AEE46001239
:101DD000196A53470012196A7C470012196A9E4714
:101DE0000012196ACD490012196AA44A0012196A30
:101DF000E84A0012196A554B0012196A104C001279
:101E0000196A424C0012196A864C0012196ABC4CBD
:101E10000012196A114D0012196A664D0012196AF2
:101E2000FA4D0012196A5C4E0012196AC44E001273
:101E3000196A6D500012196A55510012196A9752A9
:101E40000012196AC5540012196A85550012196AE0
:101E5000BA570012196A5D580012196A9B5800128D
:101E6000196A475A0012196A5B5A0012196A655AB0
:101E70000012196A8F5A0012196A9B5A0012196AC5
:101E8000BA5A0012196A715B0012196AB05B00122B
:101E9000196ABA5B0012196A135C0012196AC35CF2
:101EA0000012196AC25D0012196ABB5E0012196A3B
:101EB000585F0012196AFA5F0012196A1160001265
:101EC000196A48600012196A66600012196AAA60ED
:101ED0000012196ACF600012196AB5610012196AFE
:101EE00021620012196A9B620012196AAA63001229
:101EF000196AE9640012196AC7650012196A29662D
:101F00000012196AE3660012196A06670012196A5C
:101F1000DA670012196A25680012196A67680012E8
:101F2000196ADF680012196A0D690012196A466998
:101F30000012196A6B690012196AF3690012196AB2
:101F4000166C0012196A756C0012196A096D00127C
:101F5000196A756D0012196AC06D0012196AED6D6B
:101F60000012196A36C20312196A75C20312196A7D
:101F70005B840112196AB5840112196A1185011274
:101F8000196A5D850112196A78850112196AA98595
:101F90000112196AC6850112196AD2850112196ADD
:101FA00046870112196A5F870112196AC6870112F2
:101FB000196AD9870112196AE7870112196A9B8881
:101FC0000112196A7F890112196A858A0112196A38
:101FD0000B8B0112196A158B0112196A828B01127F
:101FE000196A998B0112196ACB8B0112196A048C38
:101FF0000112196A2E8C0112196A8F8C0112196A4A
:10200000AF8C0112196ACD8C0112196A138D01125D
:10201000196A398E0112196A868E0112196AB58EF3
:102020000112196A2B8F0112196A538F0112196A52
:102030008C8F0112196A9A8F0112196AF28F01129C
:10204000196A41900112196A80900112196AB090C0
:102050000112196ADC900112196AE7900112196ADB
:1020600005910112196AC7910112196AD1910112E1
:10207000196A0C920112196A22920112196A2B92A2
:102080000112196A80920112196A94920112196A56
:1020900091930112196AA4930112196AB99301125A
:1020A000196A5B940112196ADE940112196A9C95EF
:1020B0000112196AA7950112196ACD960112196ABF
:1020C000E9960112196A3B970112196A7A9701126F
:1020D000196A8F970112196AD1970112196A1E9A0B
:1020E0000112196A9C9A0112196A0F9B0112196A4E
:1020F000319D0112196A499D0112196A4C9D011204
:10210000196A589D0112196A6C9D0112196A749D11
:102110000112196AA79D0112196A579E0112196AC4
:10212000CD9E0112196A409F0112196AF49F011293
:10213000196AA9A00112196AC8A00112196A68A136
:102140000112196A74A10112196A9FA10112196A78
:10215000A2A10112196A0CA20112196A34A3011278
:10216000196A0CA40112196A97A40112196AB0A580
:102170000112196A6DA60112196AA6A60112196A3E
:10218000D7A60112196A77A70112196AA7A7011227
:10219000196A82A80112196A1BA90112196AA6A953
:1021A0000112196A57AA0112196AD9AA0112196AE9
:1021B0000BAB0112196A4CAB0112196A91B10212F0
:1021C000196AF6B10212196A2EB20212196A7DB2A8
:1021D0000212196A9FB40212196A82B60212196AAF
:1021E000EFB90212196A24BA0212196A46BA021227
:1021F000196AABBA0212196AE1BA0212196A04BB6F
:102200000212196A31BB0212196A8DBB0212196AD5
:10221000E28D0312196AE58D0312196A878E031283
:10222000196AD68E0312196AF78E0312196A7F8F04
:102230000312196AAA900312196ADA900312196A32
:1022400085DA0212196ACFDA0212196A4FDB02121A
:10225000196A5BDB0212196A73DB0212196AC9DBA5
:102260000212196ADADB0212196AF1DB0212196A28
:1022700078DC0212196AC3DC0212196A1BDD021231
:10228000196A71DD0212196AE4DD0212196A2FDE81
:102290000212196AA9DE0212196AFADE0212196A1A
:1022A00055DF0212196AC6DF0212196A49E00212EA
:1022B000196AE3D30212196A2FD40212196A9DD443
:1022C0000212196ABED40212196A6ED50212196A74
:1022D00077D50212196ACAD50212196AF3D5021209
:1022E000196A5AD60212196AEBD60212196A2DD748
:1022F0000212196A77D70212196AD6D70212196A1E
:1023000067D80212196AA6D80212196AE5D8021211
:10231000196A1AD90212196A2CD90212196A3ED9FD
:102320000212196A5DD90212196A66D90212196A73
:102330001CDA0212196A5CDA0212196ACABC0312A8
:10234000196AD0AD0312196A06AE0312196A3AAEC1
:102350000312196A8AAF0312196A00800212196AFD
:102360003F810212196A7B810212196A3A830212B2
:10237000196A63830212196AF6850212196A3A868B
:102380000212196AC3870212196A5B880212196A5B
:10239000C3880212196A64890212196AA689021294
:1023A000196AE6890212196A718B0212196AE18CA4
:1023B0000212196A068F0212196A348F0212196A00
:1023C0005B8F0212196A648F0212196ABF8F0212A0
:1023D000196A52900212196A70930212196AA1C303
:1023E0000312196A00800312196A33800312196AF2
:1023F000D0800312196A0C810312196A2381031217
:10240000196A48810312196A8D810312196ABE8103
:102410000312196AF6810312196A70830312196A8A
:102420008A830312196AB5FF0112196A63BE031287
:10243000196AABBE0312196AEABE0312196AFDBE1D
:102440000312196A07BF0312196A14BF0312196A2B
:1024500086F60212196A49F70212196A5CF702122B
:10246000196A35F80212196A93F90212196A2D874E
:102470000312196A85870312196A93870312196A6E
:10248000A1870312196AD2870312196AF28703120D
:10249000196A16890312196ADE890312196AC4AF10
:1024A0000312196ADAAF0312196A74B00312196AB7
:1024B000276E0012196A766E0012196A206F0012D8
:1024C000196AC86F0012196A25700012196AD6714C
:1024D0000012196A32730012196A4D730012196AD8
:1024E0009C730012196AB2730012196ABF7300124A
:1024F000196AEF730012196A35740012196A8F7421
:102500000012196ADD740012196ADF750012196A67
:102510005D780012196AFB780012196A4679001278
:10252000196A9F790012196AA2790012196AC17991
:102530000012196A1D7A0012196A207A0012196AAB
:10254000237A0012196A977A0012196AB27A001275
:10255000196AC57A0012196AB4D00112196A2C7B63
:102560000012196AE8BF0312196AF4BF0312196A4C
:1025700030C00312196A9FCC0212196AEECC021203
:10258000196A90CE0212196A4CD00212196A94D0BC
:102590000212196A7CD10212196AADD20212196AAA
:1025A000CFD20212196A2BD30212196AAFD30212C8
:1025B000196A6ED40112196A34F00112196A84F191
:1025C0000112196A09F20112196A72F20112196AEA
:1025D000B5F20112196A3CF30112196AD0F3011223
:1025E000196A5FF40112196AA1F40112196A79F9E2
:1025F0000112196AA5FB0112196A39FC0112196A44
:10260000BBFC0112196A8DA60212196A7CA702127C
:10261000196AECA70212196A20A90212196AFCA908
:102620000212196A6DAA0212196AEAAB0212196A39
:10263000ACAC0212196AD6AD0212196AE0AE0212EF
:10264000196A7FAF0212196A3CB00212196AC5C337
:102650000312196AC7C30312196AF1930212196AA5
:1026600001940212196A18940212196A75940212DE
:10267000196AFD940212196A2B960212196A93962E
:102680000212196A51970212196A93970212196A73
:10269000DB970212196AF8970212196A319802122E
:1026A000196A84980212196AB6980212196A359941
:1026B0000212196A58990212196AB1990212196A1A
:1026C000E6990212196A729A0212196AEC9A0212B7
:1026D000196A6B9B0212196A959B0212196AB19BC7
:1026E0000212196AD09B0212196ADF9B0212196A40
:1026F000149C0212196A9B9C0212196A729E0212A1
:10270000196AC79E0212196AE39E0212196A1C9F77
:102710000212196A6B9F0212196A8E9F0212196ABD
:10272000D89F0212196A00A00212196A43A002126D
:10273000196A15A10212196A63A40212196A3FA547
:102740000212196A54A50212196A03A60212196A22
:10275000A7B10312196AD8B10312196A92B203120F
:10276000196AF8B20312196A38A40312196A4AC323
:102770000312196A5DC30312196ADCA70312196AEE
:1027800007A80312196A2DA80312196A41A8031297
:10279000196A6DA80312196ACFA80312196A67A9EA
:1027A0000312196AD7AB0312196A4DAC0312196AE6
:1027B00084AC0312196A0EAD0312196A61AD0312DB
:1027C000196A8EAD0312196A87C30312196A9DBD77
:1027D0000312196AABBD0312196ACCC30312196A3A
:1027E00069C10312196A79C10312196A88C10312F7
:1027F000196AD0C10312196AD6BB0312196A4DBCFB
:102800000312196AB1BC0312196AF47F0012196A23
:10281000928A0312196AA08A0312196A1A8B031288
:10282000196AF28B0312196A7D8D0312196A72A15B
:102830000312196ABAA10312196AC7A10312196A0D
:1028400057A20312196A67A20312196A88A2031217
:10285000196A95A20312196AD0A20312196AE4A296
:102860000312196AD3C10312196A0DC20312196A3D
:102870007FC20312196ACBF10212196A20F2021206
:10288000196A1CF40212196A4EF40212196A70F4E1
:102890000212196A89F40212196AA2F40212196A60
:1028A000ACF50212196A47F60212196ADAFE021230
:1028B000196AFFFE0212196A0FFF0212196A2EFF2F
:1028C0000212196A66FF0212196A9BFF0212196A44
:1028D000DDFF0212196AECFF0212196AF6FF0212FA
:1028E000196A5DFD0112196A83FD0112196AB5FDAD
:1028F0000112196AC4FD0112196AE3FD0112196A75
:1029000043FE0112196A4CFE0112196AABFE011254
:10291000196ACFFE0112196A71FF0112196A7EFF4E
:102920000112196A8FFF0112196AB5C20312196ADE
:10293000D2C20312196A97830312196AF18403122F
:10294000196AFE840312196A11850312196A308507
:102950000312196A46850312196A5A850312196A05
:10296000BD850312196A00860312196AB086031224
:10297000196A0E870312196A1E870312196AECC0BE
:102980000312196A10C10312196A3DC10312196AB0
:1029900053C10312196A909A0312196AB79A031263
:1029A000196AD89A0312196A3D9B0312196AEF9C9F
:1029B0000312196A089D0312196A1F9D0312196AEE
:1029C000289D0312196A469D0312196A509D03122D
:1029D000196A5A9D0312196A6D9D0312196ACF9DD7
:1029E0000312196A089E0312196A2B9E0312196AB0
:1029F000709E0312196A979E0312196AB29E0312FF
:102A0000196ABC9E0312196AE39E0312196A299F70
:102A10000312196A6DC00312196A89C00312196A78
:102A20006DC30312196AD9BB0212196A05BC0212DE
:102A3000196A21BC0212196A34BC0212196A4ABC12
:102A40000212196AB5BC0212196AEFBC0212196AA5
:102A500002C10212196A1FC20212196A53C202127B
:102A6000196A98C20212196AEBC30212196A13C4D6
:102A70000212196A28C40212196A38C40212196AA9
:102A80006BC40212196AC0C40212196AD0C40212BD
:102A9000196A8EB70312196A9DB70312196AC1B772
:102AA0000312196AE1B70312196A01B80312196A0D
:102AB0001FB80312196A37B80312196A65B80312EE
:102AC000196A7FB80312196AEAC20312196A3191AE
:102AD0000312196A38910312196A22920312196AB1
:102AE00052920312196A78920312196A9B92031286
:102AF000196ABD920312196AE8920312196A419386
:102B00000312196A7A930312196AC6930312196A97
:102B1000F3930312196A13940312196AD3BA0312B6
:102B2000196AE5BA0312196AD0BB0312196AD3BB3A
:102B30000312196AB0B80312196A22B90312196A8A
:102B400060B90312196AA1B90312196AFFB403121A
:102B5000196A20B50312196A48B50312196AB3B588
:102B60000312196A0DB60312196A80E00212196A7B
:102B700093E00212196AA9E00212196AE9E002124E
:102B8000196A01E10212196A86E20212196A9FE2C9
:102B90000212196AAEE20212196ACBE20212196A33
:102BA00081E30212196A77E40212196AEEE5021251
:102BB000196A26E60212196A5EE60212196AF0E63E
:102BC0000212196A13E70212196A65E70212196AFA
:102BD0009FE70212196AFBE70212196A78E80212EB
:102BE000196AB3E80212196A71E90212196A0BEA4A
:102BF0000212196A18EA0212196AC3B90312196A91
:102C000034BA0312196A51BA0312196AB9BA031213
:102C1000196ABAFA0212196AF2FA0212196AFDFA6C
:102C20000212196A37FB0212196A54FB0212196A5E
:102C3000D7FB0212196A04FC0212196A07FC02127D
:102C4000196A09FC0212196A0CFC0212196A88FC42
:102C50000212196A77FD0212196AEDFD0212196A51
:102C600026BF0312196A82BF0312196A81B30312C5
:102C7000196A2AB40312196A4FB40312196A83B489
:102C80000312196AB1B40312196AC8B40312196A9B
:102C9000EBC40212196A1EC50212196A68C5021233
:102CA000196A85C50212196AA1C50212196ACDC531
:102CB0000212196A11C60212196A3BC60212196A77
:102CC00063C60212196AB5C60212196AF2C6021266
:102CD000196A1BC70212196A56C70212196A94C7E9
:102CE0000212196AC3C70212196AF4C70212196ADA
:102CF00041C80212196ABBC80212196A2EC902120F
:102D0000196A81C90212196A2ECA0212196AAACA5C
:102D10000212196AC1CA0212196AEDCA0212196AAC
:102D20004CCB0212196A1FEC0212196A31EC021222
:102D3000196A63EC0212196ACEEC0212196A15EDD7
:102D40000212196A4AED0212196A83ED0212196A17
:102D500005EE0212196AADEE0212196ACDEE0212E8
:102D6000196AFCEE0212196A27EF0212196A5FEF64
:102D70000212196A17F00212196A54F00212196A43
:102D8000E3F00212196A69B60312196AC4B6031293
:102D9000196AD9B60312196ADBA90312196A00AAC3
:102DA0000312196A24AA0312196A95AA0312196A4E
:102DB000B4AA0312196AA9AB0312196A6494031224
:102DC000196AD5940312196AE0940312196AF994E6
:102DD0000312196A29950312196A57950312196A81
:102DE00067950312196A60960312196A9696031280
:102DF000196A6C970312196A349F0312196AA59F06
:102E00000312196A5AA00312196A90A00312196AD0
:102E100061A10312196AC4A50312196A35A6031227
:102E2000196A6BA60312196AA2A70312196A7D9781
:102E30000312196A99970312196AE8970312196A1B
:102E400004980312196A35980312196A45980312F7
:102E5000196A31990312196A3B990312196A489940
:102E60000312196A589A0312196A6C9A0312196AA2
:102E7000759A0312196A657B0012196A857F001220
:102E8000196A8A7F0012196A1DC30312196A11D0C8
:102E90000112196ABECE0112196A6FCC0112196AA9
:102EA0000ACC0112196AC2CB0112196A35CB011280
:102EB000196A28CB0112196A26C80112196A78C545
:102EC0000112196A4CC40112196AA0C30112196ACD
:102ED000F1C10112196AACBF0112196A23BF0112B4
:102EE000196ACABE0112196A5EBE0112196A35BE9C
:102EF0000112196A39BC0112196AF7BB0112196A69
:102F0000DBBB0112196A36BB0112196AEEBA011253
:102F1000196A23B90112196A1AD40112196A76D3EF
:102F20000112196AECD20112196A8BD20112196AC4
:102F300039D20112196AA3B80112196AA0B8011294
:102F4000196ADBB70112196A27D20112196AA9B7E7
:102F50000112196AE6B60112196A11B50112196A4D
:102F6000CAB40112196AF6D10112196A1FF00112CE
:102F7000196A9CB40112196A99B40112196A86B4CB
:102F80000112196A34B40112196A23B40112196AC0
:102F900021B30112196AB7B20112196A7EB2011285
:102FA000196A39AF0112196A2AAE0112196AB9AD4C
:102FB0000112196A7EAD0112196A49AD0112196A2E
:102FC00054AC0112196A81AB0112196AABAB011240
:102FD000196AD8D10112196AF17A0000000080FB49
:102FE000323232E4738F000100C60A870001007399
:102FF00012240002004E1225000200501226000288
:103000000052122700020054122800010056122913
:103010000001005712840004005812860001005C71
:10302000122A0001005D122B0001005E122C00012B
:103030000061122D000800B20A2E00010062122F5A
:1030400000010063123000010064123100010065CC
:103050001232000100BA0A33000100BB0A34000139
:1030600000661236000100BC0A3800010067123900
:10307000000100601283000200711263000100C5AC
:103080000A64000100AF0A650001005F126D0001D3
:103090000070126E000200B00A4300010068124482
:1030A0000002006912450001006B12460002006C2C
:1030B0001247000800BD0A480001006E124B0001D3
:1030C000006F12040001007412A100010077123792
:1030D0000001007612880001007512000000000057
:1030E0000000013636010100010201000103010068
:1030F0000104010606050200000701003408010072
:103100000F090401010D0100FF0E08000017020065
:1031100000190100FF1A0100011B0100FE1C010043
:10312000081D0200001F0100012001000121020012
:10313000002301000F2402000026010001270100E6
:1031400008280200FF2A0100072B0102402C010081
:10315000002D0100012E0100012F0100FF30010BA5
:103160001C310800003A0100083B01000F2F01004C
:1031700000030271023001600211027002010202BA
:103180000202028002100261023A004100630273EF
:1031900002720262024302000213023800000200BF
:1031A00002040212020002000200020002040204F1
:1031B00002370037003C02440200023900000200DE
:1031C00002650200023502810200020502820283CA
:1031D0000200020300710030016000110070003134
:1031E00002200350048000100061000000140063FE
:1031F000007300720062004300000013000600002C
:1032000000000004001200000000000000000004A4
:10321000000400370037003C0244000000000000BA
:10322000000000650000003500810000000500007E
:103230000083000000010371030103010301030186
:103240000301032203020301031003000300030030
:1032500003000300030003000342030003240306EA
:1032600003000300030403120325032303250323A0
:1032700003040304030003000300034403000300EA
:1032800003230300036503210035038103000305C5
:103290000300030003000301017101010101011199
:1032A0000101013101010101018001100161013BB6
:1032B00000140063017301720162014301000113F4
:1032C0000106013D01350004011201000100010069
:1032D00001000104010401330133013C01440132C6
:1032E0000136000001000165010001350081010087
:1032F0000105018201830100013600010006000082
:10330000000F0000000000000000000000000003AB
:10331000FFFF00000403FFFF0000FFFF0FF40100A8
:1033200005C4040320000100130B0000000000008E
:10333000000003010F00000F261300EB2501000F12
:10334000260200C7250300CD250400D3250500D99A
:10335000250600E525FFFF0000092039200F201574
:10336000203320272021203F2045204B2057201BA1
:10337000200320FD1F0AC91D028D1D059F1D0793F7
:103380001D0C6F1D0D811DFF000000160F00000BAE
:10339000150B020002220F32000006F32005210B5C
:1033A00021D31F1121CD1FD91F140AE5D5C5B5A5FD
:1033B000A595858575655321712177215921652151
:1033C0005F2100034948424D18172505020C0E02E3
:1033D0000B040B0A0708000F000119161816161522
:1033E00023030000383C3E363B3B352B432C30302A
:1033F00017181921301B1D1F3030301618192023C3
:103400001A1C1E302D2051206B215D206320472186
:1034100017211D2129212321020402010101010993
:103420000200BE040A0100FA06A9332800E80308D6
:1034300008040C0A03090CFF1E1E0074F712154045
:10344000E99003A9F090035EE4F0122B199003BDFC
:10345000E4F0A3F09003AAF0A3F0121F0D122B1FAB
:10346000900330E4F0A3F090343A93FA7902122EEC
:103470006102621C74F2121540EAFEEBFF54806098
:10348000699003A9E0F91222DF8A088B09EA45094D
:10349000604F7C0080010CEC75F003A4F8A9F07477
:1034A0007528F582743339F583E493F4602CE49342
:1034B000F88508828B83E06870DCAA08EC75F0035D
:1034C000A4F8747628F582743339F583E493C0E068
:1034D000740193F583D082122FE3AA08AB0912225C
:1034E000D3EEFAEF6480FB023641EF5420601D12E8
:1034F0001E238A088B09EA4509600A121D81AA0861
:10350000AB091222D3EEFAEF642080DAEEA2E0508B
:103510001A900363E0640F700B7900121D4BE96091
:1035200003123644EE6401FAEF80BB5420700302AC
:10353000360F750C00124C038B09EA450970107C9C
:10354000027D007A207B009003A9E0F91223FF7C22
:103550000079047A007B00121DFF8A088B0980180D
:10356000850882850983A3A3A3A3A3A3A3A3A3740C
:1035700001F0850A08850B09E5084509606D7C00A6
:103580007904AA08AB09121DFF8A0A8B0B750C017E
:10359000E5082404F8E5091249A724FFF0A3E03464
:1035A000FF126DE470CC850882850983A3A3A3A3D1
:1035B000A3A3A3A3A3A3E0640170A5850882850942
:1035C00083A3A3A3A3A3A3E05404709485088285D6
:1035D0000983A3A3A3A3A3A3A3A3A37406F07AB709
:1035E0008508828509831237708087121DCF7C0081
:1035F00079017A007B00121DFF8B09EA45097009E9
:10360000E50C70057A20125B66EE6420023527EF28
:103610005402600B121F07EEFAEF64020234E6EF69
:1036200054046019125D52125C72790190035C12AD
:103630005FD6121CC7EEFAEF64040234E67A007B10
:103640000002387790124E123F2E121D6322C08264
:10365000C08374EA121A4C851882851983AA82AB3A
:1036600083794B122E377408121C127402F07409FD
:10367000121C12AA82AB837950122E377413121CBB
:1036800012E41261A5122E55741602512474F71219
:10369000154074E1121A4CEAFEEBFFEE4F603385E1
:1036A0001882851983AC82AD83121E477406121CE2
:1036B00012E0601E7417121C12E0FD7401121C123D
:1036C000E0FCEEFAEFFB7900122FCFE9600479A459
:1036D0008002790002621774F6121540EAFEEBFFD1
:1036E0008E828F83A3A3A3A3A3A3E05440601B12E5
:1036F000677212383E60067AFF7BFF801A8E828FD7
:1037000083124DB0FAA3E0FB8003121E6B74FE6AB5
:10371000700374FF6B6041126772125BAA121EC5C0
:10372000E98E828F836006123769E480051237695B
:103730007401F07C517D1D8E828F83125FD6122E14
:103740005BE9F5087015EE4F60097901EEFAEFFBC1
:10375000121DDBA908025BDB7508CDAA088E828FDB
:1037600083123770E960DF80EAE0240D12527F2275
:10377000E0240C12527FE0F9121D5D2274F612153E
:1037800040E9FEEAFF7A0F7B001222CDEA4B601976
:103790008A828B83740CF0EEA3A3F0EF8A828B8372
:1037A000A3F0125C5B7900802FEEF9121E058A08E7
:1037B0008B09A808A909E849601C88828983A3A30A
:1037C000A3A3A3A3A3A3A374061269E7E0F9121DA0
:1037D00015EEF9121DE17910025BDBC082C0839007
:1037E0000363E0640F7014EA4B601090035EE064C2
:1037F000086005E0640470031237FE02514EEAFCD3
:10380000EBFD7A017B009003A9E0F91223F922C0B5
:1038100082C0837900EA241DF582EB124DAD24FDB0
:10382000600B14600824FD600424FD70010902513E
:103830004E8E828F83A3A3A3A3A3A3A3A3A3123813
:103840004222124DF5FB121EC5E9228E828F83A300
:10385000A3A3A3A3A3A3A3A31238426402228E822C
:103860008F83A3A3A3A3A3A3A3A3A3125145900350
:103870004FE068221219CF7F0602175974F412150F
:103880004074FD121A4C8A088B098A828B83A3A389
:10389000E0F9121E058A0A8B0BAE0AAF0BEE4F70D1
:1038A00003023983850882850983A3E064F16030CF
:1038B000850882850983A3E064CD6024850882851C
:1038C0000983A3E0641A6018850882850983A3E050
:1038D00064E9600C850882850983A3E064E17008CF
:1038E0007900121DDBE9706C850882850983A3E0ED
:1038F000C0E07402121C12D0E0125129EEF0A3EFC6
:1039000012439C851882851983AA82AB83700512A5
:103910001CAF8003121EAD7402121C12E064E97029
:10392000338E828F8312398F750A01780A1219A695
:10393000750AE9780A1219A6E508240CF582E5094A
:10394000123E7E124379FCA3E0FD8A828B831243F0
:10395000931219CF8E828F83A3A3A3A3A3A3A3A3A0
:10396000A3E0640270108E828F83A3A3A3A3A3A3FA
:10397000A3A3A37406F0850882850983A3A3E0F9B5
:10398000121DE1121DCF901252123647023F33E052
:10399000F8A3E0F9E8FAE9FB2274F4121540EAFE14
:1039A000EBFF7508008E828F83A3A3A3A3A3E0601F
:1039B000427508088E828F83A3A3A3A3A3A3A3A306
:1039C0001250588B0BEA450B601075082C8E828FB5
:1039D00083A3A3A3A3A3E0D2E0F08E828F83A3A34B
:1039E000A3A3A3E0540364016003023A82430811D5
:1039F000023A82EE2418123F406033EE241A123F3E
:103A000040700F12385E7003A3E06970757508226C
:103A10008070EE241BF582EF123A87241AF582EFAC
:103A20001243A4EE24191267A6121D038054123803
:103A30004B700375080112385E7003A3E0697006CD
:103A4000E508D2E1F508E50860158E828F83A3A30F
:103A5000E07006E508D2E58004E508D2E6F5081234
:103A6000383164017006E508D2E0F5088E828F8354
:103A7000A3A3E0600D123A9564016006E508C2E078
:103A8000F508A908023F38124D9B123A8E22E0FC3D
:103A9000A3E0FDEE22124D95124DCDF9121EB3E9B1
:103AA00022C082C08379018A828B83A3A3E0C3945E
:103AB000024001198A828B83A3A3A3A3E0C39402CB
:103AC000400279008A828B83A3A3A3A3A3A3A3A309
:103AD000A3E064F87003A3E0F460458A828B83A3BB
:103AE000A3A3A3A3A3A3A3A3E064F97003A3E0F497
:103AF000602E8A828B83A3A3A3A3A3A3A3A3A3E083
:103B000064FA7003A3E0F460178A828B83A3A3A3F3
:103B1000A3A3A3A3A3A3E064FB7003A3E0F4700238
:103B200079008A828B83A3A3A3E0F890034CE0681A
:103B300060027900903439E493C394805013EA24EE
:103B400011123B54903439E493C333C39850027933
:103B50000002514EF582EB125C8BF82274F01215C4
:103B60004074DE121A4CEAFEEBFF8E828F83A3A311
:103B7000A3A3E0600E901250125BD2600690125028
:103B80001236477403121C12AC82AD838E828F836F
:103B9000A3A3A3125CA91264E2E9600F7403121CD0
:103BA00012AA82AB83121D7BE970087901122B2BBC
:103BB000023E73EE241B124DA07410121C12125CF4
:103BC000727409121C12E06021741A121C12E0FDBA
:103BD0007404121C12E0FC8E828F83125FD4790170
:103BE000122FCFE96004790280C37403121C12AA59
:103BF00082AB83121D75E9F50A7409121C12E0707C
:103C00002A900346E060247422550A6422601C74E2
:103C100042550A644270CF7420121C12123E896011
:103C20000A7420121C12123E8270BBE9A2E65041B7
:103C30007403121C12AA82AB83121D69E97003027D
:103C40003BAB7420121C12124DB06403700F742031
:103C5000121C12A3125BC4A3E0640D60147403125F
:103C60001C12AA82AB83121ED7E964017003023EC4
:103C700073EE242C123E7B1241AF7003A3E06970F7
:103C80001C75080078081219A678081219A6EE24E7
:103C90002E1267A6123E8F1243931219CF74091287
:103CA0001C12E07003023D50123E8F125FD6121FAD
:103CB0002B8A088B09EA45097003023DED74041252
:103CC0001C12E0F88E828F83A3A3E028F8A3E034CF
:103CD00000F9E8240DF582E9123B578A828B83A311
:103CE000A3A3E068601CE88A828B83A3A3A3F0905F
:103CF000830D121BEF850882850983A3A3A3A3125A
:103D00001BFB7904E9121C121264BF2AF8A3E034E9
:103D1000008882F583A3AA82AB831222C18A0C8B0E
:103D20000D8C0E8D0F850882850983A3A3A3A3782C
:103D30000C1219234003023E73908309780C121B66
:103D400028850882850983A3A3A3A3780C121BD31B
:103D500090035EE064046008E064096003023E735F
:103D6000E50AA2E54003023E2BEE242E123F4085D9
:103D70001882851983F0EE242F123F40C0E07401B1
:103D8000121C12D0E0F0EE2430123F40C0E074026A
:103D9000121C12D0E0F07414121C12E0640170279F
:103DA000740E121C12124DA6EE2412123F406870BF
:103DB00003A3E0697011740C121C121238587007BA
:103DC0007414121C12E4F0EE2424123E7B121861CB
:103DD0007404121C12AC82AD837407121C12AA82E6
:103DE000AB83121CB574041219CF023E739003A367
:103DF000E064016003023D507420121C12123E89DF
:103E00007009E50AA2E65003023D507410121C121C
:103E1000E0F47003A3E0F4605AEEFCEFFD740312CB
:103E20001C12AA82AB83121D878048A2E6504474FC
:103E300020121C12125FE5701A741A121C12E06430
:103E40000270307403121C12AA82AB837900121E16
:103E5000A180207420121C12123E827016741A1255
:103E60001C12E06404700C7403121C12AA82AB834F
:103E7000121E9B7422026391EE240BF582EF124D09
:103E80009B22126784E0640722124DCD640622EE65
:103E9000242A124D98123A8E2412124D982274F44C
:103EA000121540EAFEEBFF8C088D09900ABAE0601B
:103EB0000F12385E7003A3E0697005121CF1804F89
:103EC0007900125FC9121D218A828B83E5824583A6
:103ED0006035A3A3A3A3A3A3E05418602AE5082494
:103EE0001BF582E509123E7E121865124641123E0C
:103EF0007E121865EE24181267A6123F11121D33A8
:103F000074041219CF80087900123F11121CF78037
:103F1000278E828F83A3A3A3A3A3A3A3A3A3123A51
:103F20008E240BF582EF123F2A223400F583124DC6
:103F3000F5FB2274031219CF7F04021759EE2417E0
:103F4000F582EF125C8B2274F712154074F7121A87
:103F50004CEAFEEBFF90035EE06403600DE0640159
:103F60006008E0640960030240298E828F83A3E029
:103F700060030240087C007D007A027B00122B2542
:103F8000EE2402FAEF1249AE124DA690034F125CD6
:103F9000727953122E3D790012402EE064096009B7
:103FA00090035C125FD6121F2585188285198374D1
:103FB00001125BF390035E7404F07401121C12AAE8
:103FC00082AB83794A122E377401121C12AC82AD77
:103FD000837A547B03122B4390034F1264D87A03E5
:103FE0007B00122B259003521264D87A047B0012B6
:103FF0002B25900349E0A2E35004D2F08002C2F0E6
:10400000125BE0123644801E8E828F83A3AE82AF95
:1040100083FC7D007A037B10122B258E828F83E038
:10402000F912402EE4F0121DB174090262199003D6
:104030005C123F2E121CC790035E22C082C0839088
:104040000330125BD2701F90035EE014600924FC01
:10405000600A14600C800F90033880329003348023
:104060002D9003368028E84960089003311243738D
:10407000700C8A828B83A3E0F9121CBB801B900317
:10408000311246DD7005121EFB800E9003DA125BC2
:10409000D26006125BC4122FE302514E74F4121563
:1040A0004074FB121A4C8A088B097A0F7B0012228B
:1040B000CD8A0A8B0BAE0AAF0BEE4F70030241A301
:1040C0008E828F831261A37950122E3785088285E4
:1040D0000983A3E0600302418B90035CE0F470036A
:1040E000A3E0F4603490035CE064FE7003A3E0F4AA
:1040F00060278518828519831241AF7003A3E06998
:104100006017850882850983A374EA1243A97A5C43
:104110007B037950122E3D80728518828519831297
:104120006765125C727A4F7B037953122E379003C6
:104130004F125CA3125C727A527B03794B122E37BA
:104140007A517B0379E1122E37900363E0C3940F19
:104150005021900351E0C0E07402121C12D0E0F034
:104160007404121C127401F004121C12AA82AB8394
:10417000122E4F750A00780A1219A6780A1219A68B
:1041800090127AE0F912438A1219CF8508828509C4
:10419000831241A8A3F090035E7403F0EEFAEFFBE4
:1041A000125C5B7405023F35A3E08E828F8322127E
:1041B0006769E068221252862274F512154074D89D
:1041C000121A4C8A088B098A828B83A3A3A3124DEF
:1041D000D27415121C12AC82AD838A828B83A3A386
:1041E000A3A3A3A3A3A3124379FAA3E0FB121DBDCB
:1041F0007415121C12E0706B850882850983A3A3D5
:10420000A3A3A3A3A3A3E0C3940B40578E828F83E1
:10421000A3A3A3A3A3A3A3A3E064027046EE240B6D
:10422000123F40F4703D90035EE06402603AE06447
:10423000066035900330125BD26005124373604F05
:1042400090035EE064086005E06404701674171261
:104250001C12E0F9741C121C12AC82AD83125FC9EF
:10426000121DC37428026C6D900330125BD2701F54
:1042700075080078081219A678081219A6EE2410FD
:10428000123E7B1267BE124A961243931219CF8ECA
:10429000828F83125F451249C0124DA67402121C10
:1042A00012125C72EE240D123F40C0E07404121C26
:1042B00012D0E012439CF508A3E0F509740F7808CA
:1042C000121BC47405121C12E508F07419121C129A
:1042D000E0C0E07406121C12D0E0F0741B121C1235
:1042E000E0C0E07407121C12D0E0F07416121C1229
:1042F000E0C0E07409121C12D0E0F07417121C1216
:10430000E0C0E07408121C12D0E0F0EE2410123F5E
:1043100040C0E0740A121C12D0E0F0741A121C1291
:10432000E0C0E0740B121C12D0E0F07427121C12D3
:10433000E0C0E0740C121C12D0E0F0741C121C12CD
:10434000A982AA8389088A09750A00780812199E29
:104350007C087D007410121C12AA82AB8312578154
:104360001219CF851882851983AA82AB83121CC1CA
:104370000242631246E3640122E0F98A828B83A33E
:10438000A3A3A3A3A3A3A3A3E02290035C1264DCD2
:10439000900352123F2E121E7D740222F0EE240B67
:1043A000125C8822125C8BFA22F07A4F7B037953DD
:1043B0001243B422122E3D7A527B03794B122E3DCA
:1043C00022F01267C92274F212154074F8121A4CC6
:1043D000EAFEEBFF8C0A8D0B890C85188285198308
:1043E000AC82AD837583827582CA7408121902F596
:1043F0000DEEFCEFFD851882851983AA82AB83122E
:104400005EA67003750D019003AA803BEEFCEFFDE4
:10441000E508240BFAE5093400125EA5601E850844
:1044200082850983A3A3E0650C7011850882850944
:1044300083E0650A7004A3E0650B6038E508241486
:10444000F582E509123E7E1249B8E5084509602467
:10445000E50DA2E040B6850882850983E0650A7013
:1044600004A3E0650B70D5850882850983A3A3E0CA
:10447000650C70C8AA08AB097408023874C082C001
:10448000839003AA02514B74F71215409003AA12AD
:104490004DF58012EA2414F582EB123E7E124DD2C5
:1044A000122351EEFAEFFBEA4B70E99003AAE4F015
:1044B000A3F002621C74F11215408A088B09ECFE0D
:1044C000EDFF890A8A828B831263858A828B83122D
:1044D00041A81245738A828B83A3A3E0C454F0FAE7
:1044E00088828983E04A1245831241A812457DE003
:1044F000333354FCF88E828F83E04812457DA3E06D
:1045000033333354F8F88E828F83E0481245738535
:1045100008828B83A3A3A3A3A3A3E0A2E0E43313A5
:1045200013FA88828983E04AF0E5082407F50CEB4A
:1045300012578712199E7C0812577B1219CF1264EA
:10454000B6E508240FF50CE5093400F50D780C12DA
:10455000199E7C0312577B1219CFE50AC3940F40B2
:104560000D124641123E7E1241A9A3A3A3F07F077C
:10457000021759F0EEF8EFF9A30EAF83221245832C
:10458000A3A322F08508828B83A3A32274F11215C2
:1045900040EAFEEBFF890A8C088D098E828F83E04A
:1045A0008C828D83125062AE82AF83E0125841122A
:1045B00057B2C412584112464AE054038C828D838C
:1045C0001257B0A2E2E4338C828D831257AF1313DB
:1045D00013541F1258411257AEA2E7E4338C828D58
:1045E00083A3A3A3A312464A8E0C8F0D750E0078E9
:1045F0000C12199E7C087D00E508240712644B12FA
:1046000019CF1264B68E0C8F0D780C12199E7C0394
:104610007D00E508240F12644B1219CFE50AC394FC
:104620000F40148E828F83A3A3A3E0C0E012464103
:10463000123E7ED0E080061246411269DBF0024550
:104640006EE5082412F582E50922A3A31250660E36
:10465000AF832274F412154074F9121A4CEAFEEB7F
:10466000FF8908900330125BD2600E1246DD70099C
:10467000EEFAEFFB121EF5805F90035CE06E7003B4
:10468000A3E06F70537401650860097A707B0312B0
:104690005EA670447A007B02124C078B0BEA450B36
:1046A000703690035F121BEF851882851983121BE9
:1046B000FB900365E0C0E07404121C12D0E0F074BB
:1046C00005121C127401F07406121C121261A3125E
:1046D0001C85E9609B121C8B7407023F351246E370
:1046E000640222126785A3A3A3A3A3A3E02274F507
:1046F0001215408A088B098A828B83A3AE82AF830E
:10470000E0F9121CDF8E828F83E064EB600C850879
:1047100082850983A3E064E17009850882850983A5
:10472000A3E4F0123644750A01780A1219A6850826
:1047300082850983A3E0F50878081219A67900128A
:10474000438A1219CF121DCF026C70EAF0A3EBF06E
:1047500002514E74F61215409003BCE0701B7C00B1
:1047600079017A007B00121DFFEA4B600C8A828B74
:1047700083125BD26003121D57025BDBC082C083D1
:10478000124BEF401079FF121DF9E9F8903436E42E
:1047900093C398500479018002790002514E74F05D
:1047A0001215408A088B09890B750C008A828B834D
:1047B000A3A3A3A3A3A3A3A3E0F9121E058A0E8BB0
:1047C0000FAE0EAF0F750A01EE4F600302487C85F5
:1047D0000882850983A3A3A3A3A3A31264D8850891
:1047E00082850983A3A3A3A3A3A3A312557B125F6E
:1047F000D6121DED8A0C8B0DAE0CAF0DEE4F700373
:1048000002499F8E828F83A3A3A3A3E4F0A3F0E5C4
:1048100008240B1249ABE0C0E0123E78D0E0F01261
:104820001ECBEE240CF582EF125BA6E508240EF5F4
:1048300082E509124DA3EE240EF582EF125C6F752E
:104840000C01EE2406F8EF1249A7547FF0A3E054C0
:10485000FC12681BE05404600302490290125612D5
:10486000556C74077808121ADC8E828F83A3A3A379
:10487000A3A3A3E04508F0A3E04509F08E828F834F
:10488000A3A3A3A31249B674077808121BC4E508B2
:104890005407F508E50B607A8E828F83A3A3A3A348
:1048A000A3A3A3A3A374021257B3240D12527BE057
:1048B000A2E2500B90034A125CA3A3A3125C72E520
:1048C000087003024974EE2406F8EF3400F9E8FAA0
:1048D000E9FB8A828B83E0547FFCA3E054FCFDE576
:1048E0000824FFF508E434FFF50974077808121A64
:1048F000DCEC4508F8ED4509F98A828B83125C727D
:1049000080728E828F83A3A3A3A3A3A3E04480021B
:10491000487BE5087005750A0080598E828F83A355
:10492000A3A3A3A3A3E0542060121222C7EA547FDA
:10493000245F8E828F83A3A3A3A380238E828F8381
:10494000A3A3A3A3A3A3E05410600A1222C7EA54AE
:104950000F240A80DD8E828F83A3A3A3A37401F0AA
:10496000A3E41249C07404124BFE8B09EA45097096
:1049700003125B99E50CA2E050288E828F83A3A3DB
:10498000A3A3126209F9EEFAEFFB121DF3E960121C
:10499000125BC86003124D8BEEFAEFFB12235175C8
:1049A0000A00A90A026394125D6622FAE50934003E
:1049B000FB8A828B8322A3A3E0F508A3E0F50922FA
:1049C0001249C422126467A3A3A3A3A32274F412FE
:1049D000154074F7121A4C7E00121E05EA4B700344
:1049E000024A8F8A828B83A3A3A3A3A3A3A3A3A317
:1049F000E064066003024A8F8A828B83A3A3A3A389
:104A0000A3A3A3E0FF8A828B8312528EE0C0E074DE
:104A100008121C12D0E0124DC6125EAC125C72126B
:104A20001E17EF540860668518828519831264D8B2
:104A30007A007B00121DE78B0BEA450B704F900349
:104A40005C124EB6122E677C007D007A007B0080DF
:104A5000288E828F83124DB0F47003A3E0F4602D92
:104A600090035C124A96125FD6122879E9641A60A4
:104A70001C7C007D00EEFAEFFB121DE78A0A8B0B0F
:104A8000AE0AAF0BEE4F70C97900122E6D7E01EEAB
:104A9000F97409023F35124A9A22E0FCA3E0FD8E28
:104AA000828F8322C082C083EA4B70059003BD8051
:104AB000068A828B83A3A3124CB660258A828B83DD
:104AC000A3A3A3A3A3A3A3E0540860E5EC4D601542
:104AD0008A828B83124DB06C7003A3E06D70D2801C
:104AE000047A007B0002514E74F2121540EAFEEB8C
:104AF000FF890A8C088D097A107B0012234BEA4B40
:104B0000603F8A828B83A3A3A3A3A3A3A3A3A3E44D
:104B1000124DB4A3E50A12678BA3124B4B8A828B0A
:104B200083A3A3A3A3E4F0A3124DC0A3F012661FB6
:104B3000EA240CF582EB125052124B44A3A3F0A3CB
:104B4000F0023877A3F08A828B8322A3A3E508F0D2
:104B5000A3E509F02274F4121540EAFEEBFF890880
:104B60008C0A8D0BEE4F6055740165087014790145
:104B7000121DF9E9F890342FE493C398500F79117E
:104B8000806A74046508702F124BEF40F18E828F9B
:104B900083A3A3A3A3A3A3A3A3A3E508125062A383
:104BA000126CFA8E828F83A3A3E4F0A3F09003BD6E
:104BB000125BD26021800D7402650860D079C180DB
:104BC0002BE0F8A3125C9CA3A3124CB688828983C5
:104BD000A3A370ED80039003BDEEF0A3EF124BFE94
:104BE0008B0BEA450B7003125B997900023F387911
:104BF00004121DF9E9F89016BBE493C39822F01251
:104C00004C03227A207B009003A9E0F912240B22A6
:104C1000C082C083E9F879009003BD801D8A828B31
:104C200083A3A3A3A3A3A3A3A3A3E068600574FF26
:104C3000687001098A828B83A3A3124CB670DE02CE
:104C4000514E74F7121540EA4B70059003BD800673
:104C50008A828B83A3A3124CB660248A828B83A39F
:104C6000A3A3A3A3A3A3A3A3E06970E4EC60148AA5
:104C7000828B83E0240D1264C9A2E240D380047ABF
:104C8000007B0002621CC082C0839003BD80068A44
:104C9000828B83A3A3124CB660128A828B83A3A358
:104CA000A3A3A3A3A3A3E06970E580047A007B001B
:104CB00002514E3BF583123F2EEA4B2274F212153D
:104CC000408A0A8B0B8C0C8D0D750800750900EA63
:104CD000450B602E9003BD80068E828F83A3A312A6
:104CE0004D09601EAC0CAD0DEEFAEFFB850A828516
:104CF0000B83122FE3E9640170DFEEF8EFF9880807
:104D00008909AA08AB09023877E0FEA3E0FFEE4F5D
:104D10002274F71215409003BD124DA67C007D0051
:104D2000800DE8FCE9FD88828983A3A3124DA6E8E3
:104D3000496030EA687002EB6970E79003BD125F6A
:104D4000D6E86A7002E96B88828983A3A37008128F
:104D50004DA69003BD8009124DA68C828D83A3A31E
:104D6000125C7202621C74F7121540EAFEEBFFEE51
:104D70004F6015121E11124DD8125BC86003124D00
:104D80008BEEFAEFFB12235102621CEE240C124D43
:104D900098124DED22EE241DF582EF3400F58322AA
:104DA000F582EF124D9B12514522F582EF124D9B79
:104DB000124DCD22124DB822126793A3A3A3A322B2
:104DC000124DB8A3A322124B45124DCD2212677E7D
:104DD000E022E0FEA3E0FF228E828F83E0241C12FB
:104DE000527F124DED8E828F83124DED22124DF5C2
:104DF000FB12235122E0FAA3E022C082C083EAFC26
:104E0000EBFDEC4D700479058044EC24FBF582ED5C
:104E100034FF125BD07007124E51E0F4600512228D
:104E2000D380E39003A9E0C0E0124E51D0E0F090AF
:104E30003433E493F97ABF7B031222FDE9640170F5
:104E40000B7A007B20125B9D79008002790402516D
:104E50004EEC24FFF582ED34FFF5832274F4121535
:104E600040A2AFE433F508C2AF9003BF124D096012
:104E700038EE24FBF582EF34FF125BD07A007B2002
:104E80009003A96005125BA08005E0F9122309E4F4
:104E9000F50AF50B780A1219A2EEFCEFFD7ABF7B3A
:104EA000031222F774021219CFE508A2E092AFEEC6
:104EB000FAEFFB023F381264DC851882851983AA59
:104EC00082AB832274F212154074FC121A4CEAFE73
:104ED000EBFF750AFE750BFF121DD5E96005791110
:104EE000025047EE2415123F40603790126FE0C425
:104EF0003354E0F8E0333354FC48C0E0EE2415129C
:104F00003E7BD0E01250621250588B09EA4509608E
:104F100011750AFFEE240F123F404404125C80D248
:104F2000E0F08E828F8312383C6006EE241212501D
:104F30004FEE2413123F407010903439E493C0E0D8
:104F4000EE2413123E7BD0E0F08E828F83E0A2E746
:104F500050045403801CEE2414123F40701590033B
:104F60003BE0C0E0EE2414123E7BD0E0F090033B27
:104F7000E004F0EE2411123F4064017016900AAF75
:104F8000E0600D900346E0700A8E828F83E070032C
:104F900012504C8E828F83E064017013EE240B124A
:104FA0004DAA64027009EE240F123F404440F08580
:104FB0001882851983AC82AD83EEFAEFFB121E3B9B
:104FC0008A088B0974FE650A700374FFF470098EF9
:104FD000828F83A3A3126457EA450960668E828F8D
:104FE00083E0C0E07401121C12D0E0F07402121CC5
:104FF000121266237401121C1285820C85830D78AF
:105000000C1219A2EE240F123E7B121865EE240E2C
:10501000123F40F50C780C1219A690034F12186538
:105020007407121C12E0F9AC0AAD0B121E3574079E
:105030001219CFE9FE74106E700BAA08AB09122387
:105040005180027E10EEF97404023874EE2411F5DA
:1050500082EF124D9BE4F022A3123F2E79FF122E15
:10506000A32212506622F08E828F83A322C082C0B8
:105070008374DE121A4C8A828B83A3A3A3A3124DDE
:10508000A6740E121C12E8F0A3E912513C740C1223
:105090001C12125135240DF582EB123F43C0E0740F
:1050A0001A121C12D0E0F01263A4EB124DA374206C
:1050B000121C121251352415F582EB123F43C0E049
:1050C0007408121C12D0E0F0EA241CF582EB124D99
:1050D000A37412121C121251352411F582EB123FE7
:1050E00043C0E07409121C12D0E012512974FFF081
:1050F0007401121C1274FFF07402121C1274FFF07F
:1051000090830D1218617404121C12AC82AD83746A
:1051100007121C12AA82AB83121CB574041219CF99
:10512000790074221219CF802512512D22F0851892
:105130008285198322E8F0A3E9F0EA22124B45A305
:1051400012514422A3E0F8A3E0F922125FD6D083E3
:10515000D08202196774EC12154074EE121A4C8A50
:10516000128B13ECFEEDFF89097426121C121264D7
:10517000577428121C12E0F5107429121C121252D6
:1051800070742B121C12E0F50EA3E0F50F750810D9
:105190007A1E7B0012234B7402121C12125BAA743B
:1051A00002121C12125BD2700302526985188285AA
:1051B0001983AA82AB837950125A85125FD6740282
:1051C000121C1212528EA3125BAA7410121C12121D
:1051D0006CFC7402121C12E0240B12527B7402F05D
:1051E000121C1212528E7402F0121C1212677612E6
:1051F00066237402121C12125FEBE509F0740212AE
:105200001C12E0240C12527BE510F07402121C12E6
:10521000125278E512F0A3E513F07408121C12E59F
:105220000CF0A3E50DF0740A121C12E510F0850EC7
:1052300082850F83C082C083740D121C12AC82ADB4
:1052400083D083D0827403121902F97402121C12E3
:10525000AA82AB83121DDBE964017005750800802A
:10526000087402121C12124D91A908741202646E85
:10527000E0F50CA3E0F50D22E0241C12527F22F889
:10528000A3E0125286223400F98882898322125FB9
:10529000DEA3A3A3A3A32274EE121540EAFEEBFF44
:1052A0008C088D098E828F83A37408125CBBE0602A
:1052B000088E828F83A37410F0123F3D60098E82A6
:1052C0008F83A3E02408F0EE2415123F4060088E7F
:1052D000828F83A3E004F08E828F83A3A3A3A3A372
:1052E000A3E060198E828F83A3A3A3A3A3A3A3E04B
:1052F000C3332402F88E828F83A3E028F0EE2411BA
:10530000123F406005750B0E8003750B008E828F77
:1053100083A3C082C083EE240D123F40D083D0828D
:10532000F8E028250B8C828D83F0EE2411123F408B
:10533000600512579128F0850882850983E0C3949F
:10534000754009750800750900025479E0FA7B0080
:105350001266D17003025479EEFAEFFB121E41EA95
:10536000850882850983125BABEE2402F8EF1241B7
:10537000B51255731254B5F0EE24040808EF12412B
:10538000B51259BBA31254B5A3A3F0EE24131254C3
:105390009BF0EE241412549BA3F0750A08EE241619
:1053A000123F406010EE24181264D5E5082408125C
:1053B00067B4750A10123F3D6016EE241A1264D5C8
:1053C000850A0CE508250C1267B47408250AF50A4D
:1053D0008E828F83A3A3A3A3A3A3E06059EE240727
:1053E000F510EF3400F511851082F583E0C0E0126E
:1053F0005482123E7ED0E01254A5E0C0E0125482E6
:10540000123E7ED0E01254A5A312548E12199E852E
:105410001082851183E0C333FCE433FD850A0CE57B
:1054200008250C12644B1219CF851082851183E078
:10543000C333250AF50AEE2415123F40600BC0E085
:10544000125482123E7ED0E0F0123E7812548E1238
:10545000199EEE240D123F40FC7D00850B0A8E82C2
:105460008F83A3E0F8E50828F8E5093400F9E8257A
:105470000AFAE912644E1219CFAA08AB097F0A0290
:105480001759850A0CE508250CF582E50922E0F597
:105490000CA3E0F50D750E00780C22124D981254F5
:1054A000BFA3A3A322F0050A8E828F83A3A3A3A385
:1054B000A3A3A3A322A3A312681FA31254BF221263
:1054C00059BFA3A32274F61215408A828B83E0FC95
:1054D00090034C12556C74027808121ADCEC4508E3
:1054E000FCAD09EA241212556674067808121ADC1B
:1054F000EC4508FCED4509FDEA2415F582EB123F69
:10550000436004780180027800E4C8F9ED49FDEABF
:105510002411F582EB123F43F508880974097808D5
:10552000121ADCED4509FDEA2416125566740B7853
:1055300008121ADCED4509FDEA2417125566740CB1
:105540007808121ADCED4509FD8A828B83A3A3A398
:10555000A3A3A312556C740A7808121ADCECFAEDB6
:105560004509FB025BDBF582EB124D9BE0F508750C
:10557000090022E085088285098322A3E0F98508D5
:10558000828509832274EE1215408A0A8B0BECFE89
:10559000EDFF750F01E9C3940850057900025778B3
:1055A0008E828F83E9F01259E4E96003750F0012CF
:1055B00059C88E828F83125A12EE1263A5EF125AC7
:1055C00007C0E0EE2411123E7BD0E01259FFC0E08C
:1055D000EE2412123E7BD0E0125062740812645F17
:1055E000A3A3A3E060151259B0EE2413F582EF12C5
:1055F0005C6F8E828F83A3E02408F08E828F83A35A
:10560000A3A3A3A3A3A3A3E060218E828F83A3857A
:1056100082088583091259F3EE2415F582EF125C96
:105620006F850882850983E02408F08E828F83A32A
:10563000A3A3A3A3E0601A8E828F83A3858208852B
:1056400083091259D78E828F83A3A3A3A3A31257D2
:10565000A3EE241912504FEE241B12504FA3125CDC
:10566000B3E0700302570CEE2419F8EF3400F98E02
:10567000828F83A3858208858309E0FAE50A2AF5EB
:1056800082E50B123F43888289831257A3FAE50A09
:105690002AF582E50B123F43C0E0EE241A123E7B4E
:1056A000D0E01257A388828983E06059F8903432A1
:1056B000E493C398500575110C8008EE2419123F2D
:1056C00040F5118E828F83A3E0F8E50A28F50CE5FA
:1056D0000B12578712199EE511C333FCE433FD7A90
:1056E0001C7B0D1257811219CFEE241B123E7B74C6
:1056F0001CF0A3740DF0E511C333F8850882850909
:1057000083E0288006EE24181269D8F08E828F83F9
:10571000A3E0F88E828F83E0C398500302559BA3C9
:10572000E0FA8A08E50A2508F8E50B3400F9EE24CA
:105730001DF582EF125D7B1257B3C39AC0E0EE24D1
:1057400017123E7BD0E0125C78602BEE2417F8EF46
:105750003400F9880889098882F583E024F2125D13
:105760005C240EFAA3E03400FB88828983125BAAD2
:10577000125791C398F0A90F02547D7D00EEFAEF05
:10578000FB1222AF7403223400F50D750E00780C65
:1057900022900347E0F9122F63E9F8850882850912
:1057A00083E022F0850882850983E004F022A3A328
:1057B000A3A3A3F08E828F83E02274F41215408A93
:1057C000088B09EA125848F0EA1313543F12584163
:1057D000A3A3A3F0EAC41313125848A3A3F0EB1237
:1057E000583A1258527409780A121BC412583812C7
:1057F0005851740A780A121BC4E50A5401C0E0EC3F
:105800002418F582ED123E7ED0E0125857740B78C2
:105810000A121BC4125838A3125851740C780A1279
:105820001BC4125838A3A3A3A3A3A3A3A3F0740D6E
:105830007808121BC4023A82E50A54018C828D83D7
:1058400022540F8C828D832254038C828D83A3A3D8
:1058500022A3A3A3A3A3A3F08A0A8B0B22C082C016
:105860008379008A828B83A3A3A3A3A3A3E09003DD
:1058700046600FE070228A828B83A3A3E07019092F
:105880008016E060138A828B83125FCD90034FE015
:105890006A7003A3E06B70E702514E74F01215407A
:1058A0008A0A8B0B890C8C088D091259E41259C88D
:1058B000850882850983125A12E5081263A5E50955
:1058C000125A07C0E0E5082411F582E509123E7E70
:1058D000D0E01259FFC0E0124641123E7ED0E012E5
:1058E0005D837408125D9C60111259B0E5082413A1
:1058F000125D77125D83E02408F0850882850983B4
:10590000A3A3A3A3A3A3A3A3E0601785088285098B
:1059100083A31259EFE5082415125D771257B324BB
:1059200008F0850882850983A3A3A3A3A3E06019D7
:10593000850882850983A3AE82AF831259D7850873
:10594000828509831257AE04F0AA08AB09121E53D0
:10595000E9F50D7056850882850983A3A3A3A3A347
:10596000A31259BB7014E0FA8A0EE50A250EF8E579
:105970000B125C64E50CC39A80211259EFE8240EE7
:10598000F8E9125C64900347E0F9122F638E828F6E
:1059900083E0F8E50CC39824F2C399C0E0E508243D
:1059A00017F582E509123E7ED0E0F0A90D0263945E
:1059B000E50A2408F8E50B3400F9221259BF22E069
:1059C000850882850983A322850A82850B83A3A388
:1059D000125A28E0F9EA22E0F8E50A28F582E50BF8
:1059E000125C8B228A828B83126399121E4D22AE27
:1059F00082AF83E0F8E50A28F8E50B3400F92212BB
:105A00005A3BA3A3A3E022124D9BE8125A34A3A34E
:105A1000E022A3A3A3A3A3A3A3A3A3125A34125ABD
:105A200028A3A3E0F9EAF822E0FA850A82850B832D
:105A3000A3A3A322F0A3E9125A3B22F0850A828590
:105A40000B83A3A3A3A322C082C0837ACD7B037957
:105A5000E2122E377ACD7B0302514EC082C0839072
:105A6000034F02514BC082C08374FE121A4C85183A
:105A700082851983AA82AB83794B125A85125FD62D
:105A80007402025124122E3785188285198322C090
:105A900082C083794A122E3702514E74F612154095
:105AA0009003D5E0FE04F0EEF9121E058B09EA45DD
:105AB0000970EDEE60EAF9025BDB74F0121540EA62
:105AC000FEEBFF8C088D09890A7410121C12E0F598
:105AD0000B7411121C12E0F50C121F2BEA4B701301
:105AE000E50C7042A90AAC08AD09EEFAEFFB121FF3
:105AF00043806EE50A6021EA2402F582EB123F43FF
:105B0000850A082508F8E4340013E813F070098AC0
:105B1000828B83A3A37401F0E50C6045E50B70064E
:105B20008A828B83E4F07401650C7035E50B900379
:105B3000DC7004E4F0802AE004F0901257E0F89062
:105B400003DCE0C398401AE4F0900352E06E700367
:105B5000A3E06F700CEEFAEFFB7901121CD9125B17
:105B6000640263947A017B009003A9E0F912240592
:105B700022C082C08374016A7001EB70077A01123F
:105B80005B9B801290124E125BAAEA4B60051237A3
:105B9000FE8003125B6402514E7A207B009003A9C1
:105BA000E0F9122303223400F583EAF0A3EBF0229C
:105BB000C082C08390125002474BC082C0839012B3
:105BC0005202474B12678522EE240CF582EF340017
:105BD000F583125145E849221219CF7F0202175965
:105BE000A2F0E433851882851983125BFC79521286
:105BF0002E3D22125BFC7942122E3D22F0AA82AB8E
:105C00008322AA82AB83121DB77AAC7B037945123B
:105C10002E3D2274F712154074ED121A4CE9FE90D5
:105C200003A8125FF2125C3F7412121C12EE125C97
:105C30004C851882851983125C02741302621990D4
:105C4000121EE0F97AAC7B03121DBD22F090121EE9
:105C5000E0F97CAC7D0322AA08AB099003A9E0F926
:105C60001222D9223400F9E508241DF582E5091233
:105C70004D9BE8F0A3E9F022126463A3A3E022A302
:105C8000F0EE2415125C8822F582EF3400F583E0F3
:105C900022125C95223400F583E0F8A3E0F98882B3
:105CA000898322E0F8125CA922A3E0F98E828F8317
:105CB000A3A322F0EE2418124D9822F0EE2416121F
:105CC0004D982274F4121540EAFEEBFF7A007B0433
:105CD000125B68125D52125C7290035E7409F012DE
:105CE0001E5F8A088B09AC08AD09EE2413123E7BB7
:105CF000125FD6125EA6640170487A0F125D45608D
:105D0000418A828B837402125D5CFAA3E0FB8A8273
:105D10008B83A3E0FC8A828B83A3A3E0FBEC850842
:105D200082850983A3A3125BAB88828983125FDA21
:105D3000125573125C7FFAA3E0FB794A122E3D12D2
:105D40005C57023F387B001222CD8A088B09EA4556
:105D5000092290033212514590125222F0EE241D76
:105D6000F8EF125D6622125286E022125D6F223435
:105D700000F5837401F022F582E509124D9BE8F0ED
:105D8000A3E922125D8722125D8B22F085088285AD
:105D90000983A322125D8BA3A3A3A322125D94A364
:105DA000A3E0221261AD121EB922EE2417F582EF94
:105DB000125D6F121E5FEE241A124D98EAF0A3EBEB
:105DC000F02274F412154074F3121A4C8908EAFE9A
:105DD000EBFF7C0D7D007900851882851983AA82EE
:105DE000AB831222BBEE241D123E7B126776A3E02A
:105DF000F8741F58600A7901122B2B7900025E9DFE
:105E0000E8A2E55008740C121C127401F0E8A2E735
:105E10005008740B121C127401F0E8A2E6740A50C8
:105E200008121C127401F08008121C12E064017048
:105E300005EE24138003EE24151264D57402121C9F
:105E400012AA82AB83122B43123E78125EAB125C15
:105E500072740A121C12E064017033123831703B04
:105E6000121E6B8A0A8B0BA80AA90BEE240B123F99
:105E700040687003A3E0697022121E5FEAFCEBFD2C
:105E80007402121C12AA82AB83125EA6600D8518E2
:105E900082851983AA82AB83121CD3A908740D02D0
:105EA0003F35EEFAEFFB122B3DE922E0125EB02205
:105EB000F8A3E0F98518828519832274F61215403B
:105EC00074F3121A4C8A088B09ECFEEDFF7C0D7DF1
:105ED000007900851882851983AA82AB831269052F
:105EE000A3A3A3A3A3A3A3A3A3125F45125F4EF88A
:105EF000A2E55008740B121C127401F0E8A2E750DE
:105F000008740A121C127401F0E8A2E6EE50042490
:105F100013800224151264D57402121C12125F370A
:105F2000A3A3E0C0E0740C121C12D0E01261A51211
:105F30001CCD740D025BD8AA82AB83122B4385085B
:105F40008285098322E0125EB0E8F0A3E922F01214
:105F50004D9512677AA3E02274F712154074E1128E
:105F60001A4CEAFEEBFF8E828F83125FDAA3A3A3A3
:105F7000E0A2E050518E828F831239918A828B8306
:105F8000A3A3A3A3A3A3E054FE125FF28A828B8390
:105F9000125FEBE0F98A828B83E0241CFAA3E01203
:105FA00049AE125FD6121E59E9701B741D121C12E5
:105FB000125FE57011851882851983AC82AD83EE7E
:105FC000FAEFFB121EA70262178E828F83A3A3A390
:105FD000A3A3A3A3A3A3123F2E22125FDE22126764
:105FE0007EA3A3A322124DCD640422E0241B1252EF
:105FF0007F2212512DAC82AD8322E9F8790074041E
:1060000068600A740A6860057403687001090219FF
:106010006774F61215408A828B837420F0A3A374F0
:1060200001F0121C798A088B09AE08AF09EE4F60A7
:10603000108E828F837401F090039CE07003125DD8
:10604000AAEEFAEFFB025BDBC082C0839003C1744F
:1060500001F0E9A2E350037403F0E9A2E15004E087
:10606000D2E2F002514E74F612154079007C008A9B
:10607000088B09780812179FF8FF079960976097B7
:1060800060976097609060946099608D600C800963
:106090007C0480050C80F67C089003C1E05C600302
:1060A000098003EC600109025BDB74F61215408A7B
:1060B000828B83E07012A3125BD2600C8A828B8386
:1060C000125FD5122F8D80047A007B00025BDB7497
:1060D000F512154074F3121A4C8A088B09ECFEED88
:1060E000FF750A12EA45097005790002619E900366
:1060F0004FE065087004A3E065097014121E5FEAA2
:10610000FCEBFD125EA27005750A018003750A00A2
:10611000851882851983E4F004121C12E508F0A3A7
:10612000E5091261A5121C3DE960277403121C12D7
:10613000AA82AB83121C25E964017016750A0174EA
:1061400003121C12AC82AD83125EA26021750A009C
:10615000801C7412650A701690039BE06402700E36
:10616000EEFCEFFDAA08AB09121C55E970DFEEFC4E
:10617000EFFDAA08AB09121F31E9F8740A6870052F
:10618000750A01801774A0687012EEFCEFFDAA0872
:10619000AB09121F3DAA08AB09121F4FA90A740DC3
:1061A000026C6D74021261A9221261AD2212512D8E
:1061B000AA82AB832274F7121540EAFEEBFF8E82AF
:1061C0008F83A3A3A3A3A3A3A3A3E06015EE241529
:1061D000123E7B123F1E121ED1E964017004790148
:1061E00080258E828F83A3A3A3A3A3A3A3E060151E
:1061F000EE2413123E7B126209FAA3E0FB121ED1B9
:10620000E9640160D979008013124A9AA3A3A3A379
:10621000A3A3A3A3A3E022741F1219CF7F01021727
:106220005974F012154074FD121A4C8A088B09EC4F
:10623000FEEDFF890B7413121C12E0F50C750A01B8
:106240007401121C1274041267AE6048E50C601DE4
:10625000EA2417F582EB1269DB12679C8A828B8332
:10626000E0D2E7F0EA2414F582EB1250521263A454
:10627000EB125C917403126CFEEE88828983A3A3F7
:10628000F0EF88828983A3A3124B44124B4B121C5C
:1062900073E9F50AA90A740302639174EC121540BC
:1062A00074F5121A4C8A0A8B0B890C8C0E8D0F74A4
:1062B0001F121C12E0F50D7420121C12E0F510A341
:1062C000E0F5117E01EE121C12740AF0E97007E588
:1062D0000DC333240AF012647670030263781264EB
:1062E0008B7409F0A3E50CC43354E0450D12649D92
:1062F000E50C702D7C008023ECC333F8E433F9E522
:106300001028F8E51139F98882898312638588821B
:1063100089831241A8F0A30EAF830CECC3950D4006
:10632000D7E5082417F582E509125D6B121E5FE5BB
:1063300008241AF582E509125BA67403121C12AC3C
:1063400082AD83AA0AAB0B121C2BE96019E5082465
:1063500016F582E50912637F121C12A882A983E553
:10636000082418125C6B850882850983126CFAAACE
:1063700008AB09121C73E9FEEEF9740B02646E128D
:106380005D6F740322E08E828F83F0A3AE82AF83B1
:10639000221219CF7F08021759124DF5F9EA24008D
:1063A000E439FB22EA240BF5822274EE1215408AAE
:1063B0000C8B0D890E8C088D097412121C12E0F5DD
:1063C0000F7413121C12126457900586125BD26070
:1063D00077E50FC333F8E433F9E8240EFAE9340023
:1063E000FB1222CD8A108B11AE10AF11EE4F605808
:1063F0008E828F8374D4F0A3A3E50CF0A3E50D1275
:10640000645FE50EF0AC08AD09EE2405FAEF126703
:10641000B7EE240D123E7BE50FF0850A08850B09C7
:10642000750A00780812199EE50FC333FCE433FDAA
:10643000EE240EFAEF12644E1219CFEEFAEFFB9033
:106440000586126776122FE302547DFAE5093400BF
:10645000FB1222AF740322E0F50AA3E0F50B22122F
:1064600064632212646722125066A3A3A322121946
:10647000CF7F0C021759851882851983AA82AB83B6
:10648000121EB98A088B09EA450922EA240BF58213
:10649000EB125C8BFEA3E0FF8E828F8322F0A3AE13
:1064A00082AF83AC0EAD0FEEFAEFFB1264AF221297
:1064B0002B431264B622EE2408FEEF3400FF22E0E4
:1064C000FA8E828F83A3A3E022FEA3E03400FF8E26
:1064D000828F83E022124D981264DC22E0FCA3E05C
:1064E000FD22123F2E121E472274F7121540E9FEBC
:1064F0007C007D0078007900800D1265A7E02CFCFF
:10650000A3E03DFD126B9D126C06502CE8FAE9FBEE
:10651000EA75F012A4FAAFF075F012EBA42F126B2B
:10652000A6F460E01265AE124CB360D8EE60CB12F8
:1065300065A7E4F0A3F080CC78007900800D1265A7
:1065400087E02CFCA3E03DFD126B9D126BF95030EF
:10655000E8FAE9FBEA75F017A4FAAFF075F017EB6B
:10656000A42F126BD57003A3E0F460DC12658E12C9
:106570004CB360D4EE60C7126587E4F0A3F080C826
:10658000ECFAEDFB02621C12658E3BF58322E8FA01
:10659000E9FBEA75F017A4FA75F017EBA42FFB746A
:1065A000BD2AF582740B221265AE3BF58322E8FA10
:1065B000E9FBEA75F012A4FA75F012EBA42FFB7454
:1065C000A62AF582740B2274F6121540EAFEEBFF40
:1065D0009003C2801388828983E06E7003A3E06F0A
:1065E000603A88828983A3A3125BD270E87A047B25
:1065F0000012234B8A088B09A808A909E849601CE6
:10660000888289831266239003C2125FD6888289AA
:1066100083A3A3125BAA9003C2125C72025BDB8AA3
:10662000828B83EEF0A3EFF02274F41215407E000B
:106630009003C280070E88828983A3A3125BD27065
:10664000F4EEC333FAE433FB1266D1607E7F009030
:1066500003C28024888289831264D8EFC333FAE4AA
:1066600033FBE5082AF582E5093BF583ECF0A3ED61
:10667000F00F88828983A3A3125BD270D79003A402
:1066800012386B7003A3E069780870191219A2EE32
:10669000F50A780A1219A67C707D0379009003A48C
:1066A0001266DC801A1219A2EEF50A780A1219A6EF
:1066B0007C707D0379009003A4125FD6121EE374F0
:1066C000031219CFAA08AB09122351121C8B023FE7
:1066D0003812234B8A088B09EA450922123F2E12F1
:1066E0001EE922C082C08380128A828B83A3A312F8
:1066F0004DA69003C2125C721223519003C2124C39
:10670000B670E602514E74F612154090035C124DBD
:10671000D29003D6126765125C727AD67B037950E9
:10672000122E3D9003D6123A8AFAEFFB121F4990BF
:1067300003D6124DD2900588125BD260257A067B73
:10674000001222CDEA4B601A8A828B8374D5F0A3A3
:10675000A3E412678B0412679C9005881267761277
:106760002FE3025BDB12676922E0F8A3E0F99003F4
:106770005C228E828F8312677A2212677E22E0F873
:1067800012678422A3E0F58388822212678F221287
:10679000679322F08A828B83A3A3A32212678FA31D
:1067A000EEF0A3EFF022F582EF125C8BF922125D7E
:1067B000A3EA4B22FAE5093400FB122B4322125CB8
:1067C000AAA3A3A3A3A3A3A322903434E4932401F4
:1067D000F8E43400F97A027B002274F71215407E47
:1067E000008004126DB10E1268D540F77E00EE12E3
:1067F000680674FEF0A30412681BE4F00EEEC39466
:106800000340EB02621C75F003A4F8A9F074C428DD
:10681000F8740339F988828983A32212681F22F051
:10682000888289832274F71215407F0080010F90BF
:106830003431E493F8EFC3985026EF1269C16A70BF
:1068400003A3E06B70E8126D5E6C7003A3E06D60F3
:106850000A74FF6C700374FF6D70D31268BE8004FD
:106860007A007B0002621C74F61215407CFF7DFFEB
:106870007AFE7BFF121F13EA4B70407508008036CA
:10688000E50875F017A4F8A9F074B728F582740B21
:106890001269D3600C74B628F582740B1269D37038
:1068A0001374A828FE740B39FF8E828F831269E05F
:1068B000EEFAEFFB050812693B40C5025BDB74A8EA
:1068C00028FA740B39FB22EE75F017A4F8A9F01220
:1068D00069CC64FE22903431E493F8EEC3982274BC
:1068E000F7121540EAFEEBFFEE4F60101268FF74DE
:1068F000FEF0A304126D0414F0A304F002621C7CE9
:10690000177D0079001222BB8E828F832274F712CA
:106910001540EAFEEBFF7508008018E50875F017D2
:10692000A4F8A9F0126D697003A3E06F6003126D03
:10693000B9050812693B40E302621C903431E493CC
:10694000F8E508C3982274F6121540121F138A083E
:106950008B09A808A909E849600AE8240DFAE93476
:1069600000FB80047A007B00025BDB74F4121540AC
:106970008A0A8B0BECFEEDFF750800750900802E6E
:10698000E50975F017A4F8A9F0126DA4601EE509D9
:106990001269C1650A7004A3E0650B700375080AEB
:1069A000EEFCEFFD126C6060034308A00509903413
:1069B00031E493F8E509C3985004E50860C2023A4F
:1069C0008275F017A4F8A9F01269CC2274A828F5F2
:1069D00082740B39F583E022F582EF124D9BE4229D
:1069E000123F2E121D392212681FA3A3A3A3A3A333
:1069F000A3A32274F21215408A088B09ECFEEDFF66
:106A0000740E121C12126457750C007C007D0180FC
:106A1000101222C7E50CF5F0EA84ACF0750C007D8D
:106A200000780079008003126B9D126BF94003021D
:106A30006ABFE8FAE9FBEA75F017A4FA85F00D756C
:106A4000F017EBA4250D126BD57003A3E0F460D70B
:106A5000126BB365087004A3E0650960CA126BB3DA
:106A60006E7003A3E06F60BF126BB3650A7004A37E
:106A7000E0650B60B2E8FAE9FBEA75F017A4FA7575
:106A8000F017EBA4250DFB74B62AF582740B126B7C
:106A900094509474016D050C608DE50CC39C408787
:106AA000E875F017A4F8AAF075F017E9A42AF974AC
:106AB000A828F582740B39F583125FD6026B9178A2
:106AC0000079008003126B9D126C064003026B7804
:106AD000E8FAE9FBEA75F012A4FA85F00D126BE50D
:106AE00064FE7003A3E0F460DC126BDB65087004E5
:106AF000A3E0650960CF126BDB6E7003A3E06F60EB
:106B0000C4126BDB650A7004A3E0650B60B7E8FA9A
:106B1000E9FBEA75F012A4FA75F012EBA4250DFB5F
:106B2000749F2AF582740B126B945099E8FAE9FB72
:106B3000EA75F012A4FA75F012EBA4250D126BA6FB
:106B400064016081E064027003026AC574016D052E
:106B50000C7003026AC5E50CC39C5003026AC5E8C9
:106B600075F012A4F8AAF075F012E9A42AF9749647
:106B700028F582740B026AB6E50C6011EC700E7495
:106B800001650C6003026A117C01026A1C7AFE7BBB
:106B9000FF0238773BF583E014C3940622E8240112
:106BA00008E93400F922FB749A2AF582740B3BF54C
:106BB00083E022E8FAE9FBEA75F017A4FA75F0170A
:106BC000EBA4250D126BC822FB74A82AF582740B66
:106BD0003BF583E022126BC864FE22E8FAE9FBEA87
:106BE00075F012A4FA75F012EBA4250DFB74962A29
:106BF000F582740B3BF583E022903431E493FAC3C1
:106C0000E89AE9940022903425E493FA740193FB06
:106C1000C3E89AE99B2274F51215408A088B09ECA7
:106C2000FEEDFF750A008002050A903431E493F806
:106C3000E50AC3985028EEFCEFFDE50A75F017A4AD
:106C4000F8A9F0126C6060E0E50A75F017A4F8A9E5
:106C5000F074A828F582740B39F583124B4D80101F
:106C600074AA28FA740B39FB122B3DE9221219CFB2
:106C70007F0302175974F01215408A088B098C0A99
:106C80008D0B890C121F198A0E8B0FAE0EAF0FEEF3
:106C90004F60551268FFE508F0A3E509126D041274
:106CA0006CFCE50C600AEE240F123E7BE50C8006BE
:106CB000EE240F126CF4F09003D8125BD2601A909D
:106CC00003A3E064017008EE240E1269D88010EE70
:106CD000240E123E7B74078006EE240E126CF41212
:106CE00043C1121302126CEB026394EE240D124D99
:106CF00098E8F022124D98740122A3A3E50AF0A3AC
:106D0000E50BF0221249C4A32274F51215408A083B
:106D10008B09ECFEEDFF750A00800F126D697003A0
:106D2000A3E06F6003126DB9050A903431E493F863
:106D3000E50AC3985025E50A75F017A4F8A9F012E2
:106D40006D5E65087004A3E0650970CF74B228F524
:106D500082740B39F58312662380CD026C7074B295
:106D600028F582740B1269D32274B228F582740B51
:106D70001269D36E2274F7121540EAFEEBFF750814
:106D8000008019E5081269C16E7003A3E06F700AF4
:106D9000126DA47005E508126DB2050812693B403A
:106DA000E202621C74AA28FA740B39FB121C25E952
:106DB00022EE75F017A4F8A9F01268BE121F1F2268
:106DC00074F71215407E0080131268C77003A3E0A9
:106DD000F46008126DA47003126DB10E1268D540F4
:106DE000E802621C12681F125145E84922C082C0A5
:106DF0008374F8121A4C851882851983AC82AD838E
:106E00007583827582DA74081219028518828519D1
:106E100083AC82AD83125EA66401700479008002A7
:106E20007901740802512474F7121540E990054F56
:106E3000F09005397402F090053174FEF0A304F06F
:106E4000121E5F122F697A457B121221BF901244E5
:106E5000E060097A007B001224B980147AFF7BFF7E
:106E60001224B97CF47D017B327A0079081228194A
:106E700012255B02740074F6121540EAFEEBFF5413
:106E8000807032EEA2E050469012447401127017E6
:106E90007C0F7B0F900552E0FA900554E05407F9FF
:106EA0001225B5EE6401FAEFFB80721224C5AA0820
:106EB000AB091222D390054FE0F91222DF8A088B2A
:106EC00009A909EA4970E4EEFAEF648080DA541007
:106ED0006023901244E0F91225BB900ABAE06401E5
:106EE000700E7C647D007A007B089003A9127347C2
:106EF000EE641080B1EE54086006EE6408FA801D5E
:106F0000EF54026005EF6402809EEE5404600A7A3A
:106F10000279FF12275F121C1C7A007B000274307A
:106F200074F612154074FE121A4C127B3F901244F4
:106F3000E070057900122753122561900556E09004
:106F40000349F01224BF1222C7851882851983EAEB
:106F5000547FF8E028F8A3E03400F9E82464FEE95F
:106F60003400FF790112264B851882851983E0F4DD
:106F70007003A3E0F460359012447401F01224D73A
:106F8000851882851983AC82AD837A447B121224E2
:106F9000E9901244E0700E7A0279FF12275F126FB7
:106FA000BB79028011EEFAEFFB122543900556E003
:106FB000F9121EBF7901740202742D7A107B0090C1
:106FC000054FE0F912230322C082C083901273E0C0
:106FD000700E9005527402F0900554E054F8802E23
:106FE0006401700A900554E054F84401800DE06497
:106FF000027009900554E054F84402F07A037B03D0
:10700000121F5BE99005527003E480027403F002E2
:1070100079BA9012447406F07A107B0090054FE024
:10702000F91223032274F612154074FF121A4C8AC7
:10703000828B83E01460191470030271741470035E
:1070400002718624E960030271B01226450271B014
:10705000901244E0640260030271B0901273E06425
:10706000016008E0640260030271B01225018A0821
:107070008B09A808A909E8FEE9FFE8497003027135
:107080006A901242E0C39403500302716A90055261
:10709000E070599012447403127835E0F912254FCC
:1070A0008E828F83A3A3A3A3A3A3A3A3A3A3E0F58B
:1070B0000878081219A68E828F83A3A3A3A3A3A383
:1070C000A3121865900556E0F50878081219A68EE7
:1070D000828F83A3A3E0F98E828F83E0FCA3E0126A
:1070E00071B5121CA374041219CF806B6403706D08
:1070F0009012447404F090034FE064FE7003A3E028
:10710000F470121222C790034F127B457A4F7B0313
:107110007953122E3D90035CE064FE7003A3E0F40B
:1071200070141271BF90035CE8F0A3E9F07A5C7B05
:10713000037950122E3D8518828519837401F0AAB7
:1071400082AB837952122E3D8E828F83A3A3E0F906
:107150007A3B7B05121C97E9600312732390055656
:10716000E0A2E3504B12730D8046901243E0604062
:107170007A968037901273E064016005E0640270D3
:107180002F1224CB802A901273E064016005E06422
:1071900002701D900553E4F090055204F090053AFA
:1071A0001271C990125C7402F07A007B00122543C0
:1071B000740102742DFDEE240BFAEF3400FB228ED5
:1071C000828F83E0F8A3E0F922F07C707D037A3BA4
:1071D0007B05122B432274F612154074FE121A4CD2
:1071E000901244E064036015E0640A60030272993F
:1071F000900554E054076401600302729E900550AC
:10720000E07017126FBB901244E064037003122FFA
:10721000D59012447406F002730A900552E064019E
:10722000702E900553E004F0C39403402390035C58
:10723000E0F47003A3E0F4600D90035CE064FE7082
:1072400003A3E0F47006900552E48003127A11F073
:10725000121E658A088B0974FE6508700474FF6548
:1072600009700D90034FE064FE7003A3E0F4601B0F
:1072700085188285198374FEF0A304F090034F14DF
:10728000F0A3041278DB7953122E3D1279FB901291
:10729000427401F01273238071E06404705E900503
:1072A00050E07013127012900556E0A2E3500312E2
:1072B000730D122FD58053900552E0640170389001
:1072C0000553E004F0C39404502590035CE0F4708F
:1072D00003A3E0F4600D90035CE064FE7003A3E0A0
:1072E000F47007900552E4F0800D127A1180F89046
:1072F000030BE0640160EC1279FB809890039BE043
:1073000064027006122FD5126FBB026FB67A007B33
:1073100000121E837A007B00121E897A007B001205
:107320001E8F221222C7EA547F2464FA7B001225A2
:107330004322C082C083EAFCEBFD7A04127342024E
:1073400079BA7B0090054FE0F91223F92274F61206
:107350001540900551E4F07508517509057808123B
:1073600019A27C017D007A857B001223C37402126E
:1073700019CFE9701C78081219A275080175090067
:1073800078081219A27C007D007A85127394121974
:10739000CF0274307B001223D574042274F61215C8
:1073A00040E9FE9005517401F06E70037403F00221
:1073B000740A74F6121540900551E4F002740AC084
:1073C00082C0838C828D83E4F0A3F0900551E0A20B
:1073D000E05019A2E1500C8C828D837488F0A37464
:1073E0001380058A828B83E4F01224E30279BA7455
:1073F000F71215401224DD7A887B131224D1800005
:107400007F010217597F0602175975085175090542
:1074100078081219A275080175090078081219A2D6
:107420007C007D007A857B001223CF74041219CF73
:107430007F0202175974F0121540890B8A0C8B0DCC
:107440008C088D098B0EAA0E7B001222CD8A0E8B22
:107450000FAE0EAF0FEE4F6031E50D601DE5084534
:10746000096017750A00780812199E850D08AC0886
:107470007D001222AF74031219CF8E828F83E50C28
:10748000F0EEFAEFFBA90B1222D97F08021759C0C0
:1074900082C08374FD121A4CE9851882851983F025
:1074A0009005471278D36015851882851983AA82C2
:1074B000AB83900548127940122FE38016740212B4
:1074C0001C12E4F004121C12AC82AD837B027A0120
:1074D0001278CA790074031219CF0279BA74F212C1
:1074E0001540750800121DAB8A0A8B0BAE0AAF0B54
:1074F000800505081278E7EE4F70F7750B007509E7
:1075000000121DAB8A0C8B0DAE0CAF0D750A0080FE
:1075100023E0640270128E828F83A3A3A3A3A3A38C
:10752000E064017003750B01E50960030275D8057D
:107530000A1278E7E50AC395085077901271E0F4D3
:107540007003A3E0F4600F1271BF901271E06870D5
:1075500003A3E06970D9EE240BFCEF3400FD7A3B05
:107560007B05122B438E828F83A3A3A3A3E060BF6E
:107570008E828F83A3A3A3A3A3E0F890034CE068BB
:1075800070AD8E828F83A3A3A3A3A3A3E0F8901270
:107590005DE0686043E0640160030275118E828FD4
:1075A00083A3A3A3A3A3A3E064026003027528023C
:1075B0007525E50B600C0509E509C394025003022B
:1075C0007501E508650A7010E50860069005C77446
:1075D00001F07A007B008004EEFAEFFB0274057480
:1075E000F21215408A088B099005491278D3600978
:1075F000127940122FE30278029003AA1278ED90DC
:1076000003AAE0F50AA3E0F50B802D1271BF8A8270
:107610008B83A3A3E0687003A3E06970148E828F4C
:1076200083A3A3E0F88A828B83A3A3A3A3E068606B
:107630005F8E0A8F0B1278E7EE4F70CF7A167B00C1
:1076400012234B8A0C8B0DAE0CAF0DEE4F70030264
:1076500078027C167D0079001222BB8E828F83A374
:10766000A3A3A3A3A3A374FEF0A304127835A3A33A
:10767000A3A3F09003AA1278D370059003AA800BFD
:10768000E50A2414F582E50B1278F6EEF0A3EFF08C
:10769000850882850983A3A3A3A3A3A3A3A3A312FD
:1076A000780EA3A3A3F0E5082408F8E5093400F94F
:1076B0008882898312780E127825A3A3E08E828FA8
:1076C00083127825E0FAA3E0FB8E828F83127B453C
:1076D000E508240CF582E509127A92C0E0EE241345
:1076E0001278F3D0E0F088828983E064016011E5CC
:1076F00008240DFCE50934001271B5122B43800CEF
:107700007C087D0079FF1271B61222BB8508828544
:107710000983A3A3A3A3A3A3A3A3A3A3E0F8901205
:107720007AE0C3984003027802850882850983A322
:10773000A3A3A3A3E06401600990053AE0700302EB
:107740007802790090039BE0640270308E828F8310
:10775000A3A3A3A3A3A3A3A3A3E0C398500D12784C
:1077600005127A92C39414402D802C8E828F83A3AD
:10777000A3A3A3A3A3A3A3A3E068701B8E828F83FC
:10778000A3A3A3A3A3A3A3A3A3A3E0F81278051222
:107790007A92C398500109850882850983A3A3A31F
:1077A000A3A3A3A3E06042E9A2E05032850882854A
:1077B00009831271C38E828F83A3A3A3A3A3A3A360
:1077C000E8F0A3E9127841A3A3A312781BF0127882
:1077D000051278F612781BA3127841E0600B8E82B6
:1077E0008F83A3A3A3A37401F0850882850983A3D3
:1077F000A3A3A3A3A3E0600A8E828F83A3A3A37491
:1078000001F0027405E508240BF582E509221278DF
:107810001222E08E828F83A3A3A322127812A3A345
:10782000A3A3A3A322A3A312782B22F08508828509
:107830000983A3A322F08E828F83A3A3A3A3A3A370
:107840002212782BA3A3A3A3A3227A0179041228DE
:10785000137A007908122813901244E02274F71268
:10786000154074FB121A4CE9FE900550F0700A1294
:10787000784A70087403F08003127A0290054B1264
:1078800078D36033EE851882851983F090034F1208
:1078900071C37401121C12E8F0A3E9F090035212B4
:1078A00071C37403121C12E8F0A3E91278DB90058F
:1078B0004B12793D122FE37C007D007B027A02128D
:1078C00078CA74051219CF02740090054FE0F912BE
:1078D00024F522E0F8A3E0F9E84922F08518828532
:1078E0001983AA82AB8322EE24141278F3E0FEA35C
:1078F000E0FF22F582EF3400F5832274F612154082
:10790000EAFEEBFF121E5FEAFCEBFDEE2402FAEF4B
:107910003400FB122B3DE96401701F90054D127875
:10792000D36011EEFAEFFB127940122FE38B09EAD4
:1079300045097006EE240B127996027430E0F8A324
:10794000E0F58388822274F6121540EAFEEBFF8E82
:10795000828F83A3A3A3A3A3A3A3A3A3A3E06401F0
:107960007008EE240C1279968029121E6B8A088BFF
:1079700009A808A9098E828F83E0687003A3E069D3
:107980007011127A8C640160D9900554E054076438
:107990000260CF0274301278F3E0F91224EF220271
:1079A0001967C082C083121F0D90124B7401F07CC6
:1079B000007D007B027A031278CAD083D08202193C
:1079C0006774F612154090035CE0F47003A3E0F4D2
:1079D000600D90035CE064FE7003A3E0F470069019
:1079E0000552E48003127A11F01279FB127A0290A8
:1079F000124B7401F0127323027430121F0D121C0B
:107A00008B227A0079041228137A0479041228133D
:107A1000229005527403F090053A7401220219670E
:107A200002196774F6121540EAFEEBFFEE240C1201
:107A300078F3A3E054807051127A8C704CEE240CD1
:107A4000127A8F64137002A3E0603EEE240C127A67
:107A50008FF508A3E04480F50978081219A2E4F52F
:107A600008F50978081219A2EE240E127A8FFD7C0F
:107A700084EE24020A0AEF3400FBEE240F127A8F00
:107A8000F912262D74041219CF027430EE240BF56E
:107A900082EF1278F6E022C082C083EA4B600BEAE4
:107AA000FCEBFD7A0112734280057A01126FBD0270
:107AB00079BAC082C0837A007B0290054FE0F91248
:107AC000240B0279BA74F7121540E9FE900556E0CE
:107AD000A2E1501A90125DE06E6013900554E054DC
:107AE000F84402F0900556740CF0F9121EBF0274AF
:107AF0000074F61215407A007B00122FB7121E5F39
:107B00008A088B09AE08121E6575080078081219DC
:107B1000A6900556E0F9EEFCAD0912260974011293
:107B200019CF7A007B00122FB7027430C082C08355
:107B30007A00127B4B0AEAC3940640F60279BA85B2
:107B40001882851983EAF0A3EBF022EA127B54E451
:107B5000F0A3F022C333F8E433F9744328F58274B8
:107B60000539F5832274EE12154074FC121A4C8507
:107B70001882851983EAF0A3EBF0127F43E0F50A3F
:107B8000F508127F56F87402121C12E8F0A3E4F014
:107B90007402121C12E07003027ECC740D650A7030
:107BA00048AA82AB83795312299F7402121C12E0F7
:107BB00064FE7003A3E0F460157402121C12E0F47A
:107BC0007003A3E0F46007127F3CA3E0700D8518FA
:107BD00082851983AA82AB83027EC98518828519A2
:107BE00083E0FEA3E0FF027DCF7405650A70148573
:107BF0001882851983E0F8127F652421F8E43400A7
:107C0000F9802A7407650A7030127F31700F740290
:107C1000121C12E0241BF0A3E03400801B851882A4
:107C2000851983127F6575F021A4F8A9F0740212FA
:107C30001C12E028F0A3E039F07402121C12127F2B
:107C4000288A088B09AE08AF09EE4F7041740C65A5
:107C50000A6003027ECCA2AFE433F508C2AF127F04
:107C6000181220BD7402121C12127F288A0C8B0D70
:107C7000AE0CAF0DEE4F7009E508A2E092AF027EA8
:107C8000CCE508A2E092AF127F3CE4F0A3F08518A7
:107C900082851983E0F508A3E085080CF50D750EC3
:107CA00000780C12199E850A08127F56FC7D00EEA2
:107CB000FAEF127EEC1219CF7405650A7073127E0A
:107CC000E1EE2403F510EF3400F511851082127FE8
:107CD0000C12199E7C217D00AA08AB09127EED12C0
:107CE00019CF851082851183E508F0A3E509F0120C
:107CF0007ED6850882127F0C12199E8E828F83A3F6
:107D0000A3A3A3A3A3A3A3E0FC7D008510828511F8
:107D100083E02421FAA3E03400127EEC1219CF850F
:107D20001082851183E02421F8A3E0127EFD027DFC
:107D3000CF7407650A6003027DCF901217E0F8A3A5
:107D4000E0F9E8497003027DCF901217E0F510A327
:107D5000E0F511901217E4F0A3F08E828F83A3A3B5
:107D6000E07027127ED6EE240BF8EF127EFD851010
:107D70000C85110D780C12199E7C1B7D00850882E4
:107D8000850983E0FAA3E0FB8038127EE18E828FC2
:107D900083A3A3A3A3A3A3A3A3A3E508F0A3E50937
:107DA000F0880C890D780C12199E8E828F83A3A304
:107DB000A3A3A3A3A3A3E075F021A4FCADF0AA089C
:107DC000AB09127EED1219CFAA10AB1112235190FC
:107DD000121AE0F8A3E0F9E8496010EEFAEFFB129E
:107DE0007F50122FE3E96003027EC0740D650A60C4
:107DF00003027E8C127F31F8A3E0F988828983A385
:107E0000E054E0FA88828983E05403C3940240037B
:107E1000027BCE127F7EE01313543F540FF8900381
:107E20004CE0686003027BCEEA6003027BCE8518DB
:107E300082851983E0241A127F7264026003027B38
:107E4000CEEE2412F8EF3400F9E8241CFAE93400ED
:107E5000FBE8241DF582E9127EF3851882851983DB
:107E6000E0241B127F72F47003A3E0F47046127FCB
:107E70007EA3A3A3A3A3A3E0C394024037EEFAEF2B
:107E8000FB121E1DE96003027BCE8040740C650A64
:107E900070228E828F83A3A3A3E0240E127F72A28E
:107EA000E05011EE240CFAEF3400FBEE240DF582C5
:107EB000EF127EF3EEFAEFFB9003A9E0F91222D95C
:107EC000740C650A7006127F181220BD7404121912
:107ED000CF7F0A021759EE2409F508EF3400F5099F
:107EE00022EE240BF508EF3400F50922FB1222AF35
:107EF0007403223400F583E0F9122E7F223400F956
:107F0000850882850983E8F0A3E9F022F583E0F58E
:107F10000CA3E0F50D780C22851882851983E024E6
:107F200003FAA3E03400FB22E0FAA3E0FB1222CD27
:107F300022127F3522127F47A3A3E022127F43A3A0
:107F4000A3A322127F4722851882851983E0F8A314
:107F5000E0F583888222748A2508F5827433340020
:107F6000F583E49322127F4FA3A3A3A3A3A3A3A308
:107F7000E022F8A3E03400F988828983E022127FAE
:107F800035127F4E22790002196774F6121540E906
:107F9000FEEAFCEBFD901219E060548C828D83E0C8
:107FA000F87900EEC3943250047E328008EEC39418
:107FB0006F40027E6E901219E0640170228E08E517
:107FC0000824CEF508E434FFF509E88508F0A4C8D4
:107FD000AAF08509F0A42AF97A3C7B0012130AC39F
:107FE000E99401400474FF8001E88C828D83F07F66
:107FF00002021759021967FFFFFFFFFFFFFFFFFF94
:108000002020202020202020202020202020202070
:10801000202020D3FEFD2020D9DA20202020D9DA0C
:10802000202122232425262728292A2B2C2D2E2FD8
:10803000303132333435363738393A3B3C3D3E3FC8
:10804000404142434445464748494A4B4C4D4E4FB8
:10805000505152535455565758595A5B5C5D5E5FA8
:10806000606162636465666768696A6B6C6D6E6F98
:10807000707172737475767778797A202020E92090
:1080800041A042A1E045A3A4A5A64BA74D484FA8F7
:10809000504354A9AA58E1ABACE2ADAEC4AFB0B105
:1080A00061B2B3B4E365B6B7B8B9BABBBCBD6FBE15
:1080B00020202020202020202020202020202020C0
:1080C00020202020202020202020202020202020B0
:1080D0002020202020202020202020FF20202020C1
:1080E0007063BF79E478E5C0C1E6C2C3C4C5C6C742
:1080F000A2B50001020320202020202020202020E3
:10810000420030004D6F64656C3A204570736F6EAD
:1081100020544D2D5438783B204D6F64653A2045EE
:1081200053432F504F533B20426175647261746515
:108130003A2039363030206270733B000000000076
:108140003C833F833C833C833C833C833C833C8334
:108150003C833C833C833C833C833C833C833C8327
:108160003C833C833C833C833C833C833C833C8317
:108170003C833C833C833C833C833C833C833C8307
:1081800046572076657273696F6E3A202020202052
:108190005A474B47616D6520332E312E302E3231D8
:1081A000000E11101C10110E0000000E111C110EFB
:1081B000000A000E0404040E00000A000C04040E61
:1081C0000091ABA8E8AAAEAC20A1EBE1E2E0EBA9FC
:1081D00020AFE0AEA2AEA420AAA0E0E2AEA92100AA
:1081E0004E6F20636F6E6E656374696F6E20202022
:1081F0007769746820686F73742E2E2E004445567C
:1082000049434520545950453A20202020005365C9
:108210007276696365206D6F6465204F4646004D38
:1082200041433A2020202020202020202020200010
:1082300050414E2049443A20202020202020202058
:10824000004348414E4E454C3A202020202020201B
:1082500020005A474B20414444524553533A202072
:108260002020000305070A0F14191E28323C4B6416
:1082700096C8FAB120451DE927C92FA92EB3247944
:1082800025892453657276696365206D6F64652066
:108290004F4E0015000000010003000000007300B5
:1082A000000077506C6561736520776169742E2ECC
:1082B0002E0001040F0100000142830142831004DB
:1082C00001100402100403100404FFFFFFFFFFFF6E
:1082D000FFFFFFFFFFFFFFFFFFFF000000000000A8
:1082E000000082003A003B00030603000000580033
:1082F00000640000000000FFFF001000000001000B
:108300000000000C0000F8FF070100000000000062
:108310000000000100000002000000030000000453
:1083200000E803000000080000030519FA3000000F
:108330000000000004100401001D560100000003AD
:10834000398301001B40081296AFF9EA22E0F508D4
:10835000E4F509F50AF50B2274091219CF7F04021E
:108360001759EE2412FAEF3400FB1220CFE92279DC
:10837000051220DB740422E024F5C3941222122893
:10838000BB8A0C8B0D8C0E8D0F221221B3900B60CB
:10839000129E4B7A147B0022FB1283A3E8F0A3E920
:1083A000F0EE221283AB8A828B83228A828B83E057
:1083B00024FFF8A3E034FFF922EE240E12A0A174EA
:1083C00001221284031219CF7F080217591283FD6C
:1083D000A2E52212A0A4E4F0227F05021759E508C5
:1083E0001299EAE5091283FD227ADD7B031222F756
:1083F0007402221283F722EE2410F582EF3400F586
:1084000083E0221221A7740422F582EF1283FDF883
:1084100022EE240DF582EF1283FD640122E0FEA31B
:10842000E0FFEE4F22F582EF1283FD22FAEF3400D7
:10843000FB79E11229A522F0EEFAEFFB22EE240EE1
:10844000F582EF12A0A422F0A3F0028B92F582EB4A
:108450001283FDFA221219CF028FEDC082C08374FD
:10846000FE121A4C80077ADD7B031284999003DD9B
:1084700012945570F19003DF12945560097ADF7BF6
:108480000312849980EF9003DDE4F0A3F09003E3FE
:10849000F0A3F0A3F0740280161222F185188285F1
:1084A0001983EAF0A3EB12A6441220BD2274111224
:1084B00019CF028B9274F6121540E9FF8F0874E30E
:1084C0001295747433129579FE8E08FA7B0012228D
:1084D000CDEA4B6017EA2508F8EB3400F98A828B65
:1084E00083129F34A3A3A3A3E4F080227A027B002B
:1084F0001222CDEA4B60138F0874EE129574743318
:1085000012887CF0A3741A1288917A007B00029F73
:10851000EFE9FDEAFC74062DFAECA2E0501EEA75C4
:10852000F00A84A8F0E86014740A2AC398FAE8C331
:1085300094054004740A2AFA740B2AFAEDC39413C2
:108540004004781480027806E82A2409F8E434000C
:10855000F97A0A7B00121302E8F9021967C082C097
:108560008390040DE05402600A122E79E9600479C8
:108570000180027900028B92C082C08390040DE0DA
:10858000540260149003E3E0700A129452600912DE
:10859000859D5004790180027900028B929003E658
:1085A000E02410128A6CA2E722C082C0839082EA83
:1085B000E0F89003E5E0C39850051222CD80047ADC
:1085C000007B00028B92C082C0831220BD79000222
:1085D0008B92C082C08374FE121A4C851882851952
:1085E00083128738600D14606524FE700302867262
:1085F0000286FC900B40E0640F6018122093E97033
:10860000128518828519831296AA901223128AF372
:10861000122FE3900B68E0C0E08518828519831261
:108620009195D0E012871EF812870C741412871EE1
:10863000FCA3E0FD7ADF7B031222EBE5A8F8C2AFD2
:108640009003E512872F7920122081028495122051
:108650008DE98518828519836011128AF3740D12D1
:10866000871EFAA3E0FB122E7380E0128AF37415C2
:1086700080BB128A7270030286FC8518828519837A
:10868000129FC5C0E0128711D0E012871E2402F8A5
:108690001289632401FAA3E03400FB8882898312E3
:1086A000873814C394095020128A72FA851882857B
:1086B0001983A312A86BA3A3A3E0F8741728F5826B
:1086C00074341295796A600F128711E06408702C77
:1086D000128A7264087025851882851983E0F81261
:1086E0008A781412873C240AC0E085188285198391
:1086F00012870CD0E012873C0402862D85188285F3
:108700001983AA82AB831220BD02864BA3128AFE74
:108710002285188285198312A878A3A3A322128721
:10872000222212A734E022E5A8F8C2AF9003E4E0C9
:1087300004F0E8A2E792AF22EAF0A3EB128722F856
:10874000128A7DA3E022C082C0839003E812945570
:10875000600812870D122FE380027900028B927459
:10876000F7121540EAFEEBFFEE240D1283BCF0EE8B
:10877000242F128425C0E012843DD0E0F0EE243096
:10878000128425C0E0EE2412128440D0E0129CFB3B
:10879000C0E0EE2413128440D0E0F0EE242B1284CB
:1087A00040121865EE2422FCEF3400FDEE242D1259
:1087B0008425F9129AF21219CFE97007EEFAEFFB4D
:1087C000121FC7028FEDC082C083122093E960049C
:1087D000792080027901028B92C082C083EA1299CB
:1087E000E1E0D2E0028449C082C0831299DA1284A7
:1087F000177011128886400C8A828B83A3E0F912CD
:1088000020878069128870128428A2E650128A821A
:108810008B83A3E0F9901225128AF3122FE3804D87
:108820001299DA128417700D12888650088A828B8A
:1088300083743080358A828B83A3E0641B8A828BA9
:1088400083700474228023A3E0700F1299DA1284DB
:108850000C74F928F5827433800D1299DA12840CA5
:1088600074EE28F582743312887C128891028B9200
:10887000EA128877EB22EE240FF5822212A0A4E4FC
:10888000938A828B8322EA128877EB1283FDA2E31C
:1088900022F0900408E0F91222D92274F712154050
:1088A000E9FE129452602EEE702E9003E612A09212
:1088B000E4F09003E61296AA121FB59003E6E024B6
:1088C0000E1285A3500312A1579003E6E4F0A3F023
:1088D0007910122081028FED741B6E70101289675F
:1088E000640570C69003E612A092EE80C474E96E2F
:1088F00070509003E6E02411F812896360E690035B
:10890000E6E0240E181818128963A2E29003E6E04C
:10891000400C241112896014F0122AE980B7240F48
:10892000128962C2E7F01289676403700C9003E653
:10893000E02410128960D2E2F0128971122FE30252
:1089400088BB741C6E709D9003E61296AA90122B41
:10895000128AF3122FE39003E6E4F0A3F00288D525
:10896000080808128A6D229003E6E0240D128A6C32
:10897000229003E61296AFFB901221128AF722741E
:10898000F4121540750A00750B00A2AFE433FEC265
:10899000AF1294526008EEA2E092AF028A449012A5
:1089A00029128AF3122FE3E94410F89003DD8009BD
:1089B00085080A85090B128A4C128A5D60D81283D9
:1089C000DE586870EB780A1219A2AC08AD09128360
:1089D000E91219CF9003E6E508F0A3E509F0128546
:1089E0009D40649003E4E014F0EEA2E092AF9003A7
:1089F000E6E0240E181812A765FEE9FF8E828F8329
:108A0000E0FA9003E6E0F8128A78F9121F79E9900B
:108A100003E1F0A3E4129E51E0A2E750189003E6B0
:108A2000E02412128A581229E19003E6E02413127E
:108A30008A581229D59003E6128A65A2E1B3E4337D
:108A4000F9122AD102835D9003E3809AE50824FBA2
:108A5000F582E50912A74922128A6CF92212A6387A
:108A6000E508450922E0240F128A6C22F812A72596
:108A7000E022851882851983128A7DE022128AFD00
:108A8000A3A3A3A32274F7121540EAFEEBFF122062
:108A9000B7128876EF12888B400A12841170059005
:108AA00082E880039082E9E0F9EEFCEFFD7ADD7B5D
:108AB000031222FDE9602FEEFAEFFB901227128AD3
:108AC000F3122FE3EE240EF582EF128B7C40081296
:108AD0008727121FC18019EEFAEFFB90121F128A2E
:108AE000F3122FE3800A8E828F83A374F1128B041A
:108AF000028FED128AF722128AFB22E0F8A3E0F53A
:108B000083888222128437121FB522C082C083124A
:108B10001FC1028B92C082C083790090040DE05483
:108B2000027007128B76500279E890040DE05460D1
:108B3000700FEA242FF582EB128428A2E15002790B
:108B4000E88A828B83A3A3A3A3E0C3947540027930
:108B5000E8EA242DF582EB1284287012EA242AF523
:108B600082EB128428700779F51220878024E9703F
:108B7000F8121FA380F6EA242FF582EB1283FDA2E0
:108B8000E222C082C0838A828B83740DF0122E731E
:108B90008000D083D082021967C082C0838A828B12
:108BA00083E4F0A3F0128B769082E8E0F8400F9017
:108BB00003E4E0C398400F79F112208780D490033A
:108BC000E3E0C39850F11294D580F174F612154089
:108BD000E9FE244AFAE43400FB1222CDEA4B601D80
:108BE000EE8A828B83A3A3A3A3F0EA244AF8EB3492
:108BF00000F98A828B83A3A312977480047A007B86
:108C000000029FEFC082C083900404E4F090040748
:108C1000F09003F0128C257402F09003F9128C2569
:108C200074010284497481F0A37420F0A32274F5C6
:108C300012154074F1121A4C85188285198374023A
:108C4000F07401121C12E9F060047AFF7BFF7402D9
:108C5000121C1212A7717508FC750903750A0078B9
:108C60000812199E7C0B7D007407121C1212A309B6
:108C70001219CF851882851983AA82AB83122E73AD
:108C8000740F800312A30D1219CF7F0302175974BA
:108C9000F712154074FE121A4C85188285198374D8
:108CA0000AF07401121C1212A6CF740202845574C9
:108CB000F012154012A48B121BB57808790C121310
:108CC00063780812199A7AF37B030283C274F41250
:108CD000154074CB121A4C900B40E0640F600D8568
:108CE0001882851983742E1296C480227AEA7B0337
:108CF00012838A12130A88088909E4F50AF50B78A9
:108D00000812199A7AEA7B031284031219CF743578
:108D100002835A74F112154074F7121A4CEAFEEBF2
:108D2000FF7800128E166007E06403600278E8EEB8
:108D300024171284401283775022E87021EE241702
:108D400012842CEE2422128E0B128E167022EE2428
:108D50001912A6E0900B4F129774802678E8E88EDF
:108D6000828F83A3129E517417F012209902A75B81
:108D7000900B4F74FEF0A304128E277A467B0B12E1
:108D80002B43EE2425F508EF340085080CF50D750E
:108D90000E00780C12199E7C0B7D007AFC7B03126E
:108DA000A30D1219CF1283B9128E317402128E27BD
:108DB000851882851983AA82AB83122B37EE242271
:108DC000F582EF3400128E1F12199E12957F121930
:108DD000CFEE2402F8EF12A767FAE9128398242451
:108DE000129B0178081219A27402121C12AC82ADF7
:108DF0008379831A1A129AF01219CFE96003028D4F
:108E00006DEEFAEFFB121FC7028D6DFAEF3400FB17
:108E100079501229A522EE24211283FA640222F548
:108E20008312A638780C22F0EE2419FCEF3400FDF2
:108E300022F0EE240D12A0A12274F612154074F750
:108E4000121A4C900407E070387401F0F9122A9B52
:108E5000851882851983AA82AB831220C37508FC0A
:108E600075090378081219A2900B551218657B0139
:108E70007404121C12AC82AD837A0312836F121930
:108E8000CF7409029FEC74F71215401290647004BD
:108E9000A374EBF0900407E0A2E25003C2E2F0E01A
:108EA000A2E1500512907580098E828F83742A1278
:108EB0009EC6028FED74F412154074FE121A4C1205
:108EC0008F74EE2402F8EF3400F91291A185188214
:108ED0008519831291BBE0F50B70128518828519F4
:108EE00083AA82AB8379531229A512A62612A31353
:108EF00012199E7C0B7D007AFC7B0312A30D1219C4
:108F0000CF8518828519831296AAA90B121FF1909A
:108F10000407E0A2E1500A8E828F83A3E0F9121FBA
:108F2000F7900407E4F0740202835A74F7121540B4
:108F3000EAFEEBFF8E828F83A374EBF0900407E0D0
:108F4000A2E1500579EB121FF7EEFAEFFB12202792
:108F5000028FED74F7121540128F74900404E4F040
:108F6000900407F07AFF7BFF8E828F83A3E0F912D3
:108F70001FF18079EAFEEBFF7901122AA17AEA7BE0
:108F8000031221B37AF37B031221B32274F7121573
:108F900040EAFEEBFF122021804C74F712154012BC
:108FA00090CDA3A3A3E06003E4800274EB128FD9F9
:108FB0005003C2E2F0E0A2E150051290758011A2C8
:108FC000E0500D8E828F83742AF0A374EB129EC63C
:108FD000EEFAEFFB121FD980148E828F83A3F090DC
:108FE0000407E0A2E222EEFAEFFB1221237F010246
:108FF000175974F6121540EAFEEBFF900407E0D211
:10900000E1F07901122A9BEE240D1290381219A278
:10901000EE240B128440121865EE2402EF3400FF98
:109020000E0E7401C0E01220C9E9FAD0E0FBEEFC9C
:10903000EFFD12836F029FECF508EF12A71378087B
:109040002274F71215401290647004A374EBF09030
:109050000407E0A2E25003C2E2F0E0A2E1500312F2
:1090600090758089EAFEEBFF7901122AA18E828F2A
:1090700083E0642022C2E1129D0BE0F9121FF72267
:1090800074F7121540EAFEEBFF7901122AA17AEA81
:109090007B0312A8F8E06003E4800274EB128FD91E
:1090A0005003C2E2F0E0A2E15003129075028FD0AB
:1090B00074F71215401290CD74EB128FDE5003C27C
:1090C000E2F0E0A2E15003129075028FEDEAFEEBB0
:1090D000FF7901122AA18E828F83A32274F71215C1
:1090E000401290F2028FE674F71215401290F202CD
:1090F0008FEDEAFEEBFF7AEA7B031221B3EEFAEF83
:10910000FB12204B2274F712154074EF121A4CEA2E
:10911000FEEBFF129CCB7A467B0B122B31E9605B96
:109120008518828519837409F07401121C1274EF7A
:1091300012A73C1291A1F87402121C12E81291BB02
:10914000A3A3E0C0E07404121C12D0E01291B7E0B7
:10915000640870168E828F83A3A3129195A3E0C03A
:10916000E07405121C12D0E080067405121C12E493
:10917000129D277406121C121291807411028455DC
:10918000AA82AB831220ED851882851983AA82AB4F
:1091900083122E73221291992212A87CA3A3A3A357
:1091A00022E8FAE9FB8A828B83129E4B88828983AC
:1091B000E0FCA3E0F9EC22129D1C22F0A3E9F08A66
:1091C000828B8312A87822C082C08312212F028B47
:1091D00092C082C0839004247459F0A37433F0A326
:1091E0007404F0A37434F090122F7497F0A37432C7
:1091F000F0A37471F0A37431F090041074EBF0A339
:10920000741FF090040DE04401028449C082C083C1
:10921000EAFCEBFDEA241612844D79021220A50225
:109220008B92C082C083790602A16E74F61215403B
:1092300074FE121A4C90040912945560077A097B47
:10924000041220BD90040FE4F09004CD12945560F8
:109250002C800D851882851983AA82AB831220BDCC
:10926000900408E0F91222DF8A088B09A808A909EE
:10927000851882851983129774E84970D6029FEA8F
:1092800074F6121540E9FA7B00900408E0F9122305
:1092900003029FEF74F712154074F0121A4CEAFEA5
:1092A000EBFF89088E828F83E0F874CD28F58274F5
:1092B00033129579C0E07401121C12D0E0F0640BF7
:1092C000700D8E828F83A3E9F012211102938CE03E
:1092D000700302938C640C60030293787404121C74
:1092E00012EEF0A3EF129CF3C0E07403121C12D034
:1092F000E01291B7A3121BEF7406121C12121BFB93
:109300008E828F83A3A3A3A3A3A3A3A3A312A6E7E1
:10931000740A121C1212839C240E128425A2E4509B
:1093200009851882851983E48012EE2411128409BC
:10933000900B62E0C398851882851983F0E0C0E045
:10934000740C121C12D0E0F0EE2414128425C0E03C
:10935000740D121C12D0E0F0EE2415128425C0E02A
:10936000740E121C12D0E0F0EE2416128425C0E018
:10937000740F121C12D0E0F07402121C12E508F0F7
:109380007401121C12AA82AB83122E737410028411
:1093900055C082C08390040FE07004790180027987
:1093A00000028B92C082C08390040FE064037004BB
:1093B000790180027900028B9274F61215409004B4
:1093C0000FE0C333F8E433F9742D28F582741239B1
:1093D000F5831297C8C2E7F0C333FCE82CF582E9A5
:1093E000128443A3E493FEC333FCE433FD742D2CB9
:1093F000F58274123D12AB44EC4D6005EE90040F03
:10940000F08A828B83E0C333FCE433FDE82CF582E1
:10941000E93DF583E493F508131313541F54FEF844
:10942000741E28F582740412844312945570051238
:1094300020FF801BE508540FC333FCE82CF582E9BC
:10944000129579C0E0740193F583D082122FE30264
:109450009FEF9003E6129E4BE8492274F0121540EC
:1094600074FE121A4C890FEAFEEBFF890874C212CF
:10947000957474331295791294C7603B8A828B83FA
:10948000E50FF0A3E4F08E0C8F0DF50E780C121999
:109490009E850F0A74D8250AF5827433129579FCDB
:1094A0007D00EA24020A0AEB1295881219CFAA0855
:1094B000AB091294D5800B851882851983E50F12AC
:1094C000959174020283C5FA7B001222CD8A088B23
:1094D00009EA450922900408E0F91222D92274EE23
:1094E00012154074FE121A4C890C8C088D09890ED5
:1094F00074C2250EF5827433129579F50EEA600672
:109500007405250EF50E850E10AA107B001222CDD3
:109510008A108B11AE10AF11EE4F60418E828F8397
:10952000E50CF0A3E4F0EE250EF8EF3400F98E829E
:109530008F83129D12E4F0F50A780812199E850CAB
:109540000874D81295747433129579FC12958112AF
:1095500019CFEEFAEFFB1294D57900800D851882B1
:10956000851983E50C129591791A74021219CF7F2F
:109570000A0217592508F5822212A0A4E493227C3E
:109580000B7D00EE2417FAEF3400FB1222AF7403B8
:1095900022F0791AAA82AB8312208722C082C0836C
:1095A000E990040802844974F612154074FE121AF8
:1095B0004CEAFEEBFFEE54207031803AE5A8F8C289
:1095C000AF9003E5E0141287318A828B8312A74E95
:1095D00090040B12A771122099851882851983E0D7
:1095E000641560077A0B7B041220BD7ADF7B0312BF
:1095F00022F1EA4B70C6EF54807008801290040B81
:109600001296B4900408E0F91222DFEA4B70EEEEF5
:109610005410600B851882851983742D1296C4EE40
:10962000A2E0500B85188285198374241296C4EE2B
:109630005402600B85188285198374251296C4EE36
:109640005404600B85188285198374261296C4EE23
:109650005408600B85188285198374281296C4EE0D
:109660005440600D7401121C1212A72F742C129614
:10967000C4EE5480600D7401121C1212A72F742FB7
:109680001296C49004091294556018E5A8F8C2AF68
:109690009004091296AA900409E4F0A3128731A35A
:1096A0001296B47A007B00029FEA1296AFFB22E08A
:1096B000FAA3E022EAF0A3EBF01220997A0B7B04E4
:1096C0001220BD22F0AA82AB8312209922C082C050
:1096D0008390040B12A6E7EA687002EB69700790AA
:1096E000040BE4F0A3F0028B9274F7121540EAFE2B
:1096F000EBFFEE4F70031227CBA2AFE433F508C2A5
:10970000AF8E828F831294556028E824FBFAE934E7
:10971000FFFB90040B12AB46E86C7002E96D70071A
:1097200090040BE4F0A3F08E828F83E4F0A3F01298
:109730002351E508A2E092AF028FEDC082C0839072
:109740000B4FE064FE7003A3E0F470097C467D0BD0
:10975000122B37801C8A828B83A3A3A3A3A3A3A36A
:10976000A37402F0900B4F12A6E78A828B831297A4
:1097700074028B92E8F0A3E9F022C082C083900BC0
:109780005912A6FB4004790380027902028B92C031
:1097900082C0838A828B83A3A3A3A3A3A3A3A3E0F2
:1097A00064027016900B4F1297C8687003A3E069AB
:1097B00070047901800F7900800BEAFCEBFD7A469A
:1097C0007B0B122B31028B92129E4B8A828B83E091
:1097D0002274EA1215408A088B098C128D137416B4
:1097E000121C1212A718750A008C828D83A3A3A3E2
:1097F000A3A3A3A3A3E0F510E9A2E75008750CFF0B
:10980000750DFF8006900B551299EFE9C2E7F5112F
:10981000EA240EF582EB1283CDEA500A1288711207
:10982000844374088007128871128443E41299F704
:10983000A2E2EA50071299E1748080051299E1745E
:10984000101299F7A2E4500CEA2411F582EB12846D
:1098500043E48011900B62E0C0E0EA2411F582EB52
:10986000128443D0E01299F7A2E05003750A20A2B7
:10987000E350067410450AF50A8A828B83A3A3E09D
:1098800024FFFEA3E034FFFF1299DA128428C39468
:1098900002E0400614129A047403450AF50A851181
:1098A00014751500740E7814121ADCE515F50B7496
:1098B0000265117012900B5A129A03900B5912A163
:1098C000FDF01299D1801A7403651170101299C8B5
:1098D0007C697D0BEEFAEFFB122B4380E5E511600E
:1098E00026E5106014E50E650C7004E50F650D703B
:1098F000087440450AF50A800E8E828F83E50D12AA
:109900009A16E50C129A0885100C750D00740A78E9
:109910000C121ADCE50D450BF50B7402651070187E
:10992000851282851383129A02851282851383120F
:10993000A1FDF01299D1801A74036510701012996C
:10994000C8AC12AD13EEFAEFFB122B4380E5E51025
:10995000600E8E828F83E50F129A16E50E129A081A
:10996000EEF8EFF9E824FF1EE934FFFFE508240DC7
:10997000F582E5091284287005900B458003900B51
:1099800051E0FA04F0EA88828983129E51E50B12B5
:109990009A16E50AF0E5082404F8E5093400F9E52B
:1099A000082402FAE5093400FBEEFC8A828B83E08E
:1099B000F50888828983E02508C39C129F3AEEF05F
:1099C000A3EFF0790002A6F6EE24F9FEEF34FFFFD4
:1099D00022EE24FF1EEF34FFFF22EA240DF582EB76
:1099E000221299EAEB12A0A422E82410F58222E0C8
:1099F000F50CA3E0F50D22F0EA240EF582EB1283BC
:109A0000FD22A3E08E828F83129A0C22F0EE24FFB7
:109A10001EEF34FFFF22129A0C8E828F832274EC89
:109A2000121540890A8A0F8C108D118B0B74141239
:109A30001C1212A6347416121C121299EFAA0B12E1
:109A40001F738A128B13A812A913E8FEE9FFE849D5
:109A5000604312843DE50B128E31E50AF0750E006D
:109A6000780C12199E12957F1219CF78081219A23C
:109A7000AC10AD11A90F129AEE1219CFE97016E5CC
:109A80000A24F960031470061283F3D2E5F0EEFAAB
:109A9000EFFB121FC780007F0C02175974F71215D5
:109AA00040EAFEEBFF7801EE242312842560027861
:109AB0000512843DE8128E317404F0EE2402EF3476
:109AC000000A0A1283982422129B01EE2420128499
:109AD00040121865129AF879031A1A129AF012199C
:109AE000CFE97007EEFAEFFB121FC7028FEDEEFA17
:109AF000EFFB1220D5740222EE2417FCEF3400FD98
:109B0000221283FA88828983129D1C7401F02274C8
:109B1000F31215408A088B09ECFEEDFF8A828B83D5
:109B20007405129CFB8A828B83A3A3F0EA2403F5BD
:109B30000AEB3400F50B850A8212A6E5EE24241206
:109B40008440121BEFE82411F582E9128443121BB2
:109B5000FB129CCBE8FAE9FB122B37850A82850BB6
:109B60008312A0971296AA88828983A3A3A3A3A392
:109B7000A3A3A3A3EAF0A3EB129CF3C0E01299E91C
:109B8000E9128443D0E0129CE22415129CDD129C61
:109B9000E2240E129CDD129D27850A82850B83E04C
:109BA0002416FAA3E03400FB1220ED8E828F83A3EB
:109BB000A3A3A3A3A3E0C0E0850A82850B83E024CE
:109BC0000D12A720D0E0129D03850A82850B831217
:109BD00096AAEA240BFCEB3400FD88828983E08C92
:109BE000828D83F0A3E4129CEBE08C828D83A31220
:109BF000A6F1FCA30808A983A2E7E433C0E0128819
:109C000070128443D0E0F074075C60047A01800233
:109C10007A0075F00374075CA42AFAE82AF8E9349C
:109C200000F9E5082405FAE5093400FB88828983F8
:109C3000E08A828B83129CEB850882850983A3A32B
:109C4000A3A3129F34E0FC5407C333FAEC13543837
:109C5000FCEA2CFAE82AF8E9129CC1A3A3A3A3A367
:109C6000A3A3129D12129CD4E02AFAA3E03400FBB5
:109C7000C3EA98EB99402B8E828F83A3A3E0F885EB
:109C80000882850983A3A3A3A3A3A3A3A3A3129CD0
:109C9000D4A3A3E0C39A28850882850983A3A3A33C
:109CA0008016850882850983A3A3A3A3A3A3A3A3E6
:109CB000E4F0850882850983A3A3A3A3A3F002830C
:109CC000D93400F985088285098322EE2412FCEF3D
:109CD0003400FD22E0FA8E828F83A3A32212A720F4
:109CE000E422F0850A82850B83E02212A708A8826D
:109CF000A98322F0EE242E1283FA22F0EE243112F0
:109D000083FA22129D0BA3129E4B22F08E828F8328
:109D1000A322A3A3E8F0A3E9129D1C22129D2022F6
:109D2000129D0BA3A3A322F0EE2407FCEF3400FD49
:109D30002274F51215408C088D09750A00780812F6
:109D4000199E7C0B7D00028C84021967C082C0833F
:109D50007918122087028B92C082C0838A828B83FB
:109D6000E0C3940B50031220F9028B92C082C0838F
:109D7000791980DE74F7121540EAFEEBFF900409B2
:109D800012945560109004091296AA1221057A09BE
:109D90007B041220BDEEFAEFFB1220B7900409EE0F
:109DA000F0A3EFF0028FED74F712154074DE121A73
:109DB0004CEAFEEBFF8E828F83E024FD601124FECF
:109DC000604E24ED600924FA6046146043804A74B2
:109DD00016121C12E4F0129AF8740B121C12AA82CA
:109DE000AB83122B437413121C127403F0900B59A3
:109DF00012A6E77402121C12129774740A121C1233
:109E00007402129E437414121C12E8F0A3E980102D
:109E10007416121C12740180BC7416121C12740287
:109E200012A730740B129E51A3E0C0E07401121C03
:109E300012D0E0129D277417121C12129180742206
:109E4000028455F0900B55129E4B22E0F8A3E0F9E6
:109E500022F08E828F832274F7121540EAFEEBFF08
:109E6000750800EE2420129EB47003A3E06960031D
:109E70007508E8EE24171283656016EE2423F58238
:109E8000EF1283D3E508701AEEFAEFFB1220E1809F
:109E900020EE242312842560EB900430E070E575F9
:109EA00008E88E828F83A3E508129E517419129ED2
:109EB000C6028FED12A0A1129E4B900B55E06822B6
:109EC0008E828F83742912843712209922C082C017
:109ED0008374F1121A4C7402121C127404129F3A09
:109EE000A3E0C0E07403121C12D0E0F0EA2420F5D5
:109EF00082EB12A6E3740D121C12129774EA241757
:109F0000FCEB3400FD7404121C12AA82AB83122BEA
:109F1000377404121C12AA82AB831220CFE96003AB
:109F2000129FCF7402121C12AA82AB83122E73747A
:109F30000F0284AFA3A3E8F0A3E9F08A828B832207
:109F400074F612154074E8121A4C8A088B097402D0
:109F5000121C127403F0EA2412FEEB3400FFEEFC34
:109F6000EFFD7404121C12AA82AB83122B438508E6
:109F700082850983129FC8C0E0740C121C12D0E0C5
:109F8000F0129FB8121C12AA82AB831220EDEEFAD7
:109F9000EFFB1220CFE96003129FCF129FB8121C73
:109FA00012AA82AB831220ED7402121C12AA82AB99
:109FB00083122E7374188034E5082407FCE50934F5
:109FC00000FD740D2212870CA3A3128AF7E02285EC
:109FD000188285198374FFF0A312A64479531229BD
:109FE000A5900B4F74FFF0A3F02274021219CF7FDB
:109FF0000202175974F612154074D4121A4CEAFE74
:10A00000EBFF12A08CE0A2E65018900B5512A0971F
:10A01000E0687003A3E0697009900431E0604112C8
:10A02000212F740B121C12A882A9837403121C1214
:10A0300012A599851882851983742B1296C4900BEA
:10A040003AE060087408121C12E0601085188285DE
:10A0500019837405F0AA82AB83122E73742C808C42
:10A06000900B5EE060BC12836270B7EE2407129022
:10A07000381219A2900B551218657B017C467D0B96
:10A080007A0379061283711219CF80D08E828F8362
:10A09000A3A3128AF7A322129E4BEE242A12A0A198
:10A0A00022F582EF3400F58322C082C08374EF1260
:10A0B0001A4C8518828519837409F07401121C12D8
:10A0C00074EE12A6D00284AD74F7121540E9FFA217
:10A0D000AFE433F508C2AFEF600312299312292DC4
:10A0E00012A157900431E0F91229BD900B55129638
:10A0F000AA1229C3900B591296AA1229C97A697B10
:10A100000B1229CF7E0012A145129455600912A1AD
:10A1100045128AF3122FE30EEEC3940740E8122192
:10A120008312207B900432E4F0121F6D900431E41E
:10A13000F07A587B0B79521229A5E508A2E092AF7C
:10A140007900028FEDEEC333F8E433F9741028F58B
:10A1500082740439F58322900B68E0F91229E190AA
:10A160000B67E0F91229D522C082C0837909122039
:10A170009F028B92C082C08390041E749BF0A374D4
:10A1800033F0A3740EF0A37434F0A374B6F0A37488
:10A1900033F090040DE4F0A3F0122927028B920211
:10A1A000196774F7121540EAFEEBFFECF8EDF98E33
:10A1B000828F83740712A20312A1FDA3A312A2032C
:10A1C000A3A312A1FDA3A3A312A704A3121BEF8EA6
:10A1D000828F83A3A3A3A3121BFB8E828F83A3A3CF
:10A1E000A3A3A3A3A3A3E4F0E82415F582E91284B2
:10A1F0000C12A904A3A3A3129774028FEDE08E8220
:10A200008F832212A708A3A3A3A3A32274F4121579
:10A2100040EAFEEBFF900434E412A322E0C394046E
:10A22000400690043474E8F08E828F83A3A3A3A326
:10A23000A3A3A3E0C3940F40158E828F83A3A3A38F
:10A24000A3A3A3E06403601590043474E8F08E8245
:10A250008F83A3A3A3A3A3A3E06403700E90040DB4
:10A26000E0A2E0400690043474E8F0EEFCEFFD7AE2
:10A27000337B0412214D8E828F83A3A37808121B97
:10A28000B5740A78081219E99004477808121BD3AC
:10A290008E828F83A3A3A3A3A3A3A3E090044B1256
:10A2A000A32C90044CF0A3740AF0900B68E0900487
:10A2B0004EF0900444128C257404F0EE240A12A38C
:10A2C0001612199E7C0B7D007A4F7B0412A30D128F
:10A2D00019CF900434E07020A3E060069004347439
:10A2E000EAF0900435E0F91229ED8E828F8374260E
:10A2F000F07904122A9580078E828F837429F0EEFC
:10A30000FAEFFB12209902835DAA82AB831222AF7F
:10A31000740322EE2407F508EF12A713750A0078DC
:10A32000082212A32622129D20A3A32212A326A351
:10A33000A3A3E02274F412154074F7121A4CEAFE3B
:10A34000EBFF900435E0702A90044DE0640A60222F
:10A350001229FFE9C0E090044DE0F890043CE028A9
:10A36000F812A76524F512A746D0E0F090043BE070
:10A3700004F09004477808121BB57401780812198C
:10A38000E99004477808121BD390044DE004F0E5EF
:10A3900008A2E04006E0C3941D40D7E0641D60665B
:10A3A0007A4D7B0479E11229A5900435E0600464BC
:10A3B000027009EEFAEFFB12215F804D7408121C47
:10A3C00012740212A73074FFF0A3F0900435E06419
:10A3D00001700679087A80800479077A8375084FBE
:10A3E00075090478081219A27508FF7509FF780825
:10A3F0001219A27B007404121C12AC82AD8312836A
:10A40000711219CF8003129EC002835874F0121586
:10A4100040750801750900750A00750B0090044D20
:10A42000E078081219427808121B859004377808E2
:10A43000121B3B900435E06403700F12A48B121BB7
:10A44000B57808790C121363803575080175090019
:10A45000750A00750B0090044BE0780812194290C1
:10A4600083097808121B2890832D780C121BB5786D
:10A4700008790C121363900435E070031229F978FF
:10A480000812199A7A3E7B040283C2900B631283EE
:10A490004D90832D780C2274F512154074D4121A45
:10A4A0004CEAFEEBFF900435E064026008E06401D2
:10A4B000600302A594900434E4F0740B121C12A8FB
:10A4C00082A9837403121C1212A59990044CE0F81F
:10A4D00090043BE0C398400302A55EA312A634900B
:10A4E000043BE0F50A803C850882850983A3A3A389
:10A4F000A3A3A3A3A3A312A6E77414121C12E068DB
:10A500007003A3E0697013740B121C12AC82AD834C
:10A51000AA08AB09122B31E97044150AE508242179
:10A5200012A70FE50A70C0740B121C12A982AA832D
:10A5300089088A09750A00780812199E7C217D0015
:10A5400090043BE08CF0A4F8A9F0A3E028FAA3E083
:10A5500039FB12A30D1219CF90043BE004F0900BCD
:10A560003AE0600E7408121C12E0700690044CE091
:10A57000700D851882851983AA82AB83122E739081
:10A58000044CE0600F90043BE0F890044CE06870ED
:10A5900003129EC0742C028C87E8F0A3E9F0EEFC55
:10A5A000EFFD851882851983AA82AB831220E722EA
:10A5B00074F612154074FE121A4CEAFEEBFFEE24FC
:10A5C0001A12842564037051EE2423128425640337
:10A5D000704712A6268E828F83A3A312A634850805
:10A5E00082F58312A64C795012A61C12A64C794B08
:10A5F0001229A5AA08AB0979E112A61CA312834768
:10A60000851882851983F0A3E912A640795312298F
:10A61000A5900434E4F0129EC0029FEA1229A58599
:10A62000088285098322EE2412FAEF3400FB794A6E
:10A630001229A52212A63822E0F508A3E0F5092286
:10A6400012A6442212A734AA82AB83221296AFF933
:10A65000EA851882851983F0A3E9F0E5082402123F
:10A66000A70F851882851983AA82AB8322C082C076
:10A6700083900434E064E860267A3E7B041221B3C0
:10A680001229F37904122AA1900435E064037006BC
:10A69000900434E060097A4E7B0479E11229A57AAE
:10A6A000337B04028B8DC082C08374F5121A4CEA8E
:10A6B000FCEBFD851882851983AA82AB8312214D9C
:10A6C0007401121C1274FC12A6D0740B0284AFE940
:10A6D00012A644122E7322C082C083790702A16E93
:10A6E000F582EF3400F583129E4B22E0FEA3E0FFDB
:10A6F0002212A708E0227F0E021759C3E094FEA39E
:10A70000E094FF2212A70822F088828983A322F511
:10A7100008E5093400F50922E0F50EA3E0F50F2263
:10A72000F812A72522A3E03400F98882898322E465
:10A7300012A73422F085188285198322F0EE2402B4
:10A74000F8EF3400F922F582E934FFF5832212A7ED
:10A750005222E0851882851983F02274091219CFDC
:10A760007F07021759A3E03400F9E822FB888289A9
:10A7700083EAF0A3EBF022C082C08390045AE4F095
:10A78000A3F090045CF0A3F0908301121BEF9012F1
:10A7900037121BFB908301121BEF90123B121BFB25
:10A7A00090045EE402844774F412154090045EE461
:10A7B000F0A3F090045A129455603412A86BC08232
:10A7C000C0839012377808121BB5D083D0827808E6
:10A7D000121A77501A12A85812A912121A77500694
:10A7E00012A912121BD390045A12A86412977490E3
:10A7F000045C12945590045E602E129455601E9075
:10A80000045C12A874C082C08390045E12A9151261
:10A810001BB5D083D0827808121A77501090045C50
:10A8200012A8641297748005129455602512A871BD
:10A83000C082C0839012377808121BB5D083D082B3
:10A840007808121A77500B12A871121BEF1228C742
:10A8500080031228CD02835D1228BB8A088B098CE5
:10A860000A8D0B22129E4B90045E2212870DA3A329
:10A870002290045E12A8782212A87C22128AFBA3DE
:10A88000A32274F412154090045E1294556066126F
:10A89000A86B7808121BB575831275823778081279
:10A8A0001A77500B1227CB90045E12945560461213
:10A8B000A85890045E12A915121923503812A871D5
:10A8C000C082C08390830D7808121BB5D083D082DC
:10A8D0007808121A7750031227CB90045E12A6EB69
:10A8E000EEFAEFFB12A8F8A3A3A312A904128AF3AD
:10A8F000122FE380B202835D1221B38E828F83A375
:10A90000A3A3A322A3E0F98E828F83A3A3A3A3A36F
:10A91000A32290045A12A87878082274F0121540E5
:10A920008A088B098C0A8D0B7410121C1280248EDD
:10A93000828F83A3A3C082C08390830D780C121BE7
:10A94000B5D083D082780C121A7750031227CB8EA1
:10A95000828F8312841D60428E828F83A3A3780826
:10A96000121AEF12A99D7002EF6970C38E828F8355
:10A97000A3A3C082C08390830D780C121BB5D08333
:10A98000D082780C121A7750A690830D121BEF8E8E
:10A99000828F83A3A3121BFB80B50283C890045E41
:10A9A000129E4BEE682274F0121540A2AFE433F50C
:10A9B00008C2AF90045C12A6EB90045A121865907E
:10A9C0001237780C121BB5780C121B74AA0CAB0D45
:10A9D000AC0EAD0F12219574021219CF803B8E82FE
:10A9E0008F83A3A3C082C083901237780C121BB54B
:10A9F000D083D082780C121A774013901237780CDB
:10AA0000121BB58E828F83A3A3780C121AA18E829B
:10AA10008F8312A6E7E8FEE9FFEE4F70C190123770
:10AA2000C08290123B780C121BB5758312D08278CD
:10AA30000C121A62601590123B121BEF9012371223
:10AA40001BFB901237121BEF1228B5122189E50863
:10AA5000A2E092AF0283C874F0121540EAFEEBFF49
:10AA6000A2AFE433F50CC2AFECFAEDFB8C828D8320
:10AA70008008AA0EAB0F8A828B8312A718E50E45B9
:10AA80000F60228E828F83A3A3C082C083850E8233
:10AA9000850F83A3A37808121BB5D083D0827808D2
:10AAA000121A7750CD8A828B83EEF0A3EF129E515B
:10AAB000E50EF0A3E50F12AAC912A9A07002EF6972
:10AAC0007003122189E50C8087F08C828D8322EE41
:10AAD000FAEFFB1221A10283C874F0121540EAFEBE
:10AAE000EBFF7410121C127808121BB512AB031284
:10AAF0001B618E828F83A3A37808121BD37C5A7D9F
:10AB00000480CC12837E7808790C2274F7121540E9
:10AB1000ECF8EDF98C828D838004A882A98312ABB6
:10AB2000468C828D83E58245836014EA65827003DA
:10AB3000EB658370E51296AF12A76C7901800279FC
:10AB400000028FEDF583E0FCA3E0FD2274F71215FF
:10AB500040EAFEEBFFA2AFE433F508C2AF7C5A7DBA
:10AB6000041221ADE9700B7C5C7D04EEFAEFFB1260
:10AB700021AD12A99D7002EF69700312218902971D
:10AB80003274F7121540E9FE900302E4F0EE9003F0
:10AB900001F07CBD7D0A7A037B03122B4390126E79
:10ABA000E090030BF0122FB102B50C74F4121540B3
:10ABB0008A088B09EB5480605B90030112CB96608E
:10ABC0004A8E828F83E06401703212BD8D1218614B
:10ABD000EE241212D217F50A780A1219A612AC47FF
:10ABE0001219A2EE240B12AD25121865EE241712CD
:10ABF000CBA61221CB74091219CF8008E064027031
:10AC000003122F33EEFAEFFB1222D3AA08E50964F0
:10AC100080FB8030EA5402600C90121C7401F0EA50
:10AC20006402FA801FEA54046005EA640480F3EACF
:10AC30005408600C122FABE5086408FAAB098004D5
:10AC40007A007B0002AD1DEE240FF50AEF3400F50B
:10AC50000B780A2274F41215408A088B098A828BB9
:10AC600083A3A3A3E0241012B833FA12BE04700326
:10AC700002AD038E828F837402F0A3E412BDF2A3AF
:10AC8000A3A3A3E8F0A3E912BB88A3A3A3A3A3A350
:10AC9000A3F0E5082403F8E50912B439241012B62C
:10ACA000A18E828F83A3A3A3A3F0EE2409FA12AD91
:10ACB0000512B868F5838882E0A2E58E828F83A3AF
:10ACC000A3A3A3A3500474018001E4F0E5082403C6
:10ACD000F88882898312CAE1EA12D175EB12AD2895
:10ACE00012AD1012199E12D18EEB12B8988E828F6F
:10ACF00083A3A312BD9A1219CFEEFAEFFB900301C2
:10AD000012BE148018EF3400FB8E828F83A3A3221F
:10AD1000E0F508A3E0F509750A007808227F04022F
:10AD20001759EE240CF582EF12BDDE22A3A3A3A3D4
:10AD300012C7DEEA2212AD392212BB6FE8F0A3E996
:10AD400022F582EF12C56AF822C082C083EA4B6006
:10AD50001890039BE06402701090121CE4F0EAFC6F
:10AD6000EBFD7A0212B3BA801290121C7401F07AD1
:10AD7000027B00900301E0F912240502B3ADC0820A
:10AD8000C08390127BE075F005A4FCADF079007AE9
:10AD90007D7B0D1222BB7B008012EB75F005A4F8C1
:10ADA000A9F012AF2974FEF0A304F00B90127BE01F
:10ADB000F8EBC39840E402B3ADC082C0837C007B53
:10ADC0000080037C010B90127BE0F8EBC398504F9E
:10ADD000EB75F005A4F8AAF0EAF912AF227003A30C
:10ADE000E0F460E112AF19E82403080808E912B49E
:10ADF0003924FFF0A3E034FF12C55AF8A3E0F9E8C4
:10AE00004970C0EB75F005A4F8EAF912AF19888211
:10AE1000898374FEF0A30412CE94A3E4F080A6EC20
:10AE2000A2E0500312B3B402B3AD74F6121540EAB7
:10AE3000FEEBFF90127BE0700302AF14EE241112C0
:10AE4000D217700302AF148E828F83A3A3A3A3A390
:10AE5000A3A3A3A312BB7B6402600F8E828F83A384
:10AE6000A3A3A3A3E0700302AF147C0080010C90A5
:10AE7000127BE0F8ECC3985045EE240B12AD25127E
:10AE8000C7DAEC75F005A4FAABF0747D2AF582748C
:10AE90000D3BF583E0687003A3E06970D1EE2412E6
:10AEA00012D217FBEC75F005A4F8A9F0747F28F511
:10AEB00082740D39F583E06B70B4790080587C00A2
:10AEC00080010C90127BE0F8ECC39850EDEC75F02B
:10AED00005A4F8A9F012AF227003A3E0F470E31206
:10AEE000AF19EE240B12AD2512BAA2EAF0A3EB12B1
:10AEF000AF3488828983A312B820740C12C39B7A62
:10AF000008FB900301E0F912240B8B09EA45097054
:10AF10000312B3B4790102B3DC747D28F8740D39DF
:10AF2000F92212AF29E064FE22747D28F582740DA7
:10AF300039F5832212B402E02274F212154074F340
:10AF4000121A4CEAFEEBFF8E828F83A3A3A3A3A366
:10AF5000A3A3A3A3A3E0F50A90121CE0700579BA9D
:10AF600002B24E750801750900750C00750D007C64
:10AF7000087D007900851882851983AA82AB831227
:10AF800022BB7405121C12740112B27654046012B2
:10AF90007402121C12E0D2E612B2765408700375E5
:10AFA0000803E05410600674404508F508E05408B2
:10AFB00060227402121C12E044C012B27654206067
:10AFC0000A7403121C12E0D2E080087403121C12EF
:10AFD000E0D2E1F08E828F83A3A3A3A3A3A3A3A3B4
:10AFE000E07018121E6585188285198312BBBE7425
:10AFF00002121C12E0D2E2F002B0A0640F701574CD
:10B0000002121C12E0D2E312BE2B12BBB14508F5AE
:10B010000802B0A08E828F83A3A3A3A3A3A3A3A39C
:10B02000E064028E828F83700512AD3580C9A3A3C0
:10B03000A3A3A3A3A3A3E0640370138518828519B7
:10B0400083AC82AD83EEFAEFFB122F9380528E8297
:10B050008F83A3A3A3A3A3A3A3A3E0640170419040
:10B06000039FE0601C7402121C12E0D2E312BE1AAD
:10B0700085188285198312BFA8750910750AFF808B
:10B08000187402121C12E0440C12CFF974FDF0A3E4
:10B0900074FFF074044508F5088E828F8312D1CCBA
:10B0A00012C1C4503A7402121C12E0540C701B8E70
:10B0B000828F8312CAE1122651E9700579BB02B270
:10B0C0004E7402121C12E0D2E5F012C1C45010748A
:10B0D00002121C12E0540C64047004E0D2E5F0EE9D
:10B0E000241112D217C0E07404121C12D0E012B85E
:10B0F00047121C12E0600302B2477408121C1212BD
:10B10000B25A12B26CEE241812D217C0E0E812D173
:10B110005FE912AD28D0E0F0EE241912D217C0E09A
:10B120007408121C12E0241312B416D0E012B854A2
:10B130006401701190039FE0C0E07408121C1212A9
:10B14000B253D0E0F07408121C1212B6792417FA28
:10B15000EF12B6A8FCE8241CF582E912AD28EC1227
:10B16000C39B8E828F83A3A3A3A3A3A3A3A3A3E0C4
:10B17000C0E0E82422F582E912AD28D0E0F074089E
:10B18000121C1212B265E50AF07408121C1212B6F3
:10B190007E2424F582E912CAA9A3E50D12CB12FC84
:10B1A000A3E0FDE82426F582E912AD28ECF0A3ED3A
:10B1B00012B3E112BB9EE82428F582E912AD2812F1
:10B1C000CC53C0E0E8242FF582E912AD28D0E0F09E
:10B1D000EE241B12D217C0E07408121C1212CFCD3D
:10B1E000D0E0F0EE241A12D217C0E07408121C123C
:10B1F000E0242E12B416D0E012CFF112AD111219C4
:10B200009EEE241112AD2512BB9E740B121C12125D
:10B21000BD941219CFEE241512D2175440601B9022
:10B22000032012BBF26013851882851983AA82ABB2
:10B230008390032112B451122FE38518828519835C
:10B24000AA82AB83122F09740C121C12E0F9740D40
:10B2500002B2AFE0241512B41A2212B682240FF5FE
:10B2600082E9340022E0242312B41A22F583E5088F
:10B27000F0A3E509F022F0EE241512C5672274F759
:10B280001215407E638A828B83E0600C7905122F51
:10B2900063E9F87456C398FE900347E0600CF91216
:10B2A0002F63E9F8EEC39824F2FEEEF902B50C1212
:10B2B00019CF7F0602175974F512154074F8121A47
:10B2C0004CEAFEEBFF8C088D09750A0112D1AB1216
:10B2D000B85D700D90034F12B47CE8F0A3E9F080E4
:10B2E00039851882851983AA82AB83121E7185184D
:10B2F00082851983AC82AD8312B859700F121E6B10
:10B30000850882850983EAF0A3EB80D2AC08AD09F9
:10B31000EEFAEFFB121C31E9F50AA90A740802BB28
:10B32000D374F6121540EAFEEBFF7A0C7B00122371
:10B330004BEA4B606BEE242012D2178A828B83F08B
:10B34000EE242112B3A3F0EE242212B3A3A3F0EE55
:10B35000242312B3A3A3A312BDD312C7E2E8F0A320
:10B36000E912C55F12C7E3A3A3E8F0A3E912C38DF6
:10B370008A828B83A3A3A3A3A3A3A3A3F0EE242F6A
:10B3800012D217C0E012B82C12AD28D0E012BBC404
:10B390008A828B83A3A3A3A3A3A3A3A3A312BFA85F
:10B3A00002B3DC12C5678A828B83A322F0D083D0DC
:10B3B000820219677CF47D017A087B00900301E02A
:10B3C000F91223F92212B3C92212B3CD2212BDEA17
:10B3D000A3A32212BB96A3E0221219CF7F02021769
:10B3E00059F012B3E912BDDE22EE240FF582EF22EE
:10B3F000F582EF12BDDEE422E0F91223032212B43B
:10B400000222F0EE2412F582EF3400F583221219A5
:10B41000CF7F0802175912B41A2212B4632212BD48
:10B42000EAE022C082C08312BC2412B3F302B3ACA0
:10B4300012BB8F22790102196712B87E22F8EF340D
:10B4400000F98808890922EEFAEFFB900318E0F86A
:10B45000A312B45D22E0F812B45CA322A3E0F5834A
:10B4600088822212B46722F8A3E012B46E2234005C
:10B47000F9888289832212B91E64052212C7DE85EB
:10B48000088285098322C082C08312BC2412B4932F
:10B4900002B3AC12BDDE74012202B434C082C08398
:10B4A0009003167487F0A3742FF0900318747BF048
:10B4B000A3742FF090031A7475F0A3742FF0900307
:10B4C0001C7481F0A3742F02B3AC74F7121540EA18
:10B4D000FEEBFF12B502A2E550268E828F8312CAC0
:10B4E000E190031612B44E122FE38E828F83E0F8A0
:10B4F000A312BF89A312BBF2700612B502C2E5F017
:10B50000800A8E828F8312B455A3E0227F01021736
:10B510005974F512154012B66712B67E2420F582D2
:10B52000E912D21AFE74035EF50A12BA8C12AD2823
:10B5300012B67988828983F0A3A882A983E50A607C
:10B54000097402650A600302B5D8740C5EFF6015C9
:10B5500074086F601074046F701D7402650A7005C2
:10B56000EEA2E4402D8A828B83A3A3A3A3A3A3A36B
:10B57000A3E0242312B6C9740C6F701012B66224B3
:10B580002412B6B1242412B67412B6CC7402650A21
:10B590007005EEA2E4404112B662242612B6B12430
:10B5A0002612B687A312B6DB12B68712B6DB12B626
:10B5B0007412B6CCEF600F74086F600A740C6F6081
:10B5C0000574046F70128A828B83A3A3A3A3A3A321
:10B5D000A3A3E0242212B6C98A828B83A3A3A3A3C8
:10B5E000A3A3A3A312B6977005EEA2E150178A8217
:10B5F0008B83A3A3A3A3A3A3A3A3E0242E12BA9394
:10B6000012B6C2800E90030212B6C2900302E0048A
:10B6100012B878A3A882A983EEA2E7504212B662BC
:10B62000242112B68712B6CC8C828D8312B6976015
:10B630002E8A828B83A3A3A3A3A3A3A3A3E0243076
:10B6400012B6C9EEA2E150178A828B83A3A3A3A3EB
:10B65000A3A3A3A3E0243112B6A188828983F002B8
:10B66000BBD612B667E022EA2408FCEB3400FD8C5E
:10B67000828D832212BA97A32212C7DEEE2212B65F
:10B68000822212BE25E82212B68B22F508A3E034EE
:10B6900000850882F58322E0242112BA97E0540342
:10B6A00022FAA3E012B6A8223400FB8A828B83E040
:10B6B0002212B68B12B6C2A3A882A9838C828D8374
:10B6C000E022E088828983F02212BA9712B6D02253
:10B6D000E088828983F0A308A9832212B6D08C82E5
:10B6E0008D83E0242822C082C0838A828B8312B596
:10B6F00006F8740358F98A828B83A3A37401F0E9D6
:10B7000060057402697061740C58FC601474086CF4
:10B71000600F74046C70137402697005E8A2E44051
:10B720001D8A828B83A3A37402F0740C6C700A8A46
:10B73000828B83A3A3E02402F07402697005E8A25F
:10B74000E440258A828B83A3A3E02404F0EC600FFD
:10B7500074086C600A740C6C600574046C70098A5F
:10B76000828B83A3A3E004F0E8A2E750318A828BA6
:10B7700083A3A3E00412CC57F9A3E0F5838982A345
:10B78000A3A3E0540360178A828B83A3A3E004F091
:10B79000E8A2E150098A828B83A3A3E004F08A82A5
:10B7A0008B83A3A3E00402B3ACC082C0838A828BE4
:10B7B00083A3A3A3A3A3A3A3A3A3A312BBF2600980
:10B7C0008A828B83A3A312B7CC02B3ADA3A3A3A396
:10B7D000A3A3A3A312BDA31223512274F7121540F1
:10B7E000EAFEEBFF12C7D688828983A3A3A3A3A393
:10B7F000A3A3A3E4F012B820A3A3A3A3A3A3A3F03D
:10B80000A3F0E812CA93E912B81A122F51EEFAEF18
:10B81000FB122F5D02B50CF582ED12BDDEE4F022C5
:10B82000A312B8252212B878A3A3A322EA240BF509
:10B8300082EB2212D13D24092212BDDE12D1D07535
:10B840000E00780C22740112B88312B84E22122F07
:10B850000F740C2212BAC9E022EEFAEFFB12B861A3
:10B8600022122B3DE964012212B86FF8A3E022EA0C
:10B87000F0A3EB12B878E022F0888289832212B418
:10B880006EE022F0851882851983AA82AB8322128A
:10B8900022AF74032212C81712BDDEE0FC7D002225
:10B8A000021967C082C0838A828B83A3A3A3A3A348
:10B8B000A3A3A3E070528A828B83A3A3E0F812B9FA
:10B8C0001A6401604312B9146402603C12B9146432
:10B8D00003603512B9146404602E8A828B83A3A39B
:10B8E00012B476602312B914640A601C12B914648D
:10B8F0000B601512B914640C600E12B914640D605B
:10B90000077904122B2B800990031E12B44E122FBC
:10B91000E302B3AD8A828B83A3A312B91E2212B4B1
:10B920005CE02274F612154074FA121A4CEAFEEB2F
:10B93000FF7403121C12EEF0A3EFF07403121C123A
:10B94000AA82AB83122F3F12D214600302BA8785FA
:10B9500018828519837432F07405121C12C082C0DB
:10B96000838E828F83A3A3A3A3E0D083D082F8E049
:10B9700028C0E07401121C12D0E012BAE3C0E074D7
:10B9800002121C12D0E012BAC2F8A3E0F9E8496032
:10B9900026E82417F582E912AD28C082C083E82486
:10B9A00016F582E912D21AD083D082F8E028F87412
:10B9B00001121C12E028F0851882851983AA82AB37
:10B9C00083121C798A088B09A808A909E849700321
:10B9D00002BA7A8E828F8312BAA2A3A3EAF0A3EBF3
:10B9E00012BACFA3A3E0C0E0E82420F582E912ADAB
:10B9F00028D0E012D00CC0E0E82421F582E912AD95
:10BA000028D0E012BADEC0E0E8242AF582E912ADBF
:10BA100028D0E0F07405121C12E0FA12BA8C12D28F
:10BA20001A2A12C1D0E8242BF582E912AD2812BBE4
:10BA3000BE7405121C12E0C0E0E8242DF582E91264
:10BA4000AD28D0E012BAC2FAA3E0FBEA4B6019E8D5
:10BA5000242BFAE912AD06A3A3A3A3A3A3A3A3E0F7
:10BA6000241612BA9312BAAA8E828F83A3A3A3A319
:10BA7000A3A3A3A3E8F0A3E9800CEEFAEFFB122F37
:10BA80004B12AD227410F0740602B3D9E8240BF502
:10BA900082E92212BA9722FCA3E03400FD8C828D49
:10BAA000832212BDA38882898322E0FC8A828B8351
:10BAB000E02CFCA3E03400FD8A828B83ECF0A3ED44
:10BAC000F02212BAC9A3A3E02212BEC3A3A322F09C
:10BAD000E812D15FE912BDDE740112BE2B2212BA48
:10BAE000E9E02212BAE9A3E02212CC62A32274F7A1
:10BAF000121540EAFEEBFF12D214701E12BB241284
:10BB0000BBF2600612B447122FE312D214700B126C
:10BB1000CAD5121C7312AD22E9F0EEFAEFFB122F18
:10BB20004B02B50C122F578E828F83A3A3A3A3A31E
:10BB3000A3A3A3A3A32274F6121540EAFEEBFF8C85
:10BB4000088D09122651E9700479018011AC08AD05
:10BB500009EEFAEFFB90031C12B44E122FE302B36E
:10BB6000DC12CFFDE02212BB6FE8F0A3E9F022E087
:10BB7000F8A3E0F98518828519832212BDA3121E4D
:10BB8000C5E92212B467E02212B3C512BB8F22E0CE
:10BB90008E828F83A32212BDE3A3A3A3A32212BB91
:10BBA000A222E0FCA3E0FD22740112BE2BA3A3E0BD
:10BBB0002212BB6674042212241D8E828F83EAF047
:10BBC000A3EBF02212BBC82212BE2FA3A312BE25E4
:10BBD00022740D1219CF7F03021759C082C083123D
:10BBE000BBEB7439F0A3742F02B3AC122F6F900328
:10BBF0001E2212B682492274F7121540E9FE12BCC9
:10BC00002412AD2812BBF2601888828983A3E05405
:10BC100003700EEEFB12BA8C12AD2812BC3012BCAF
:10BC20002A02B50CEA12CA93EB22E0F91221C522CE
:10BC3000E0FA88828983A3A32274E81215408A0857
:10BC40008B098C168D178914741A121C12E0F50AD0
:10BC5000A3E0F50B741C121C12E0F513741D121CEA
:10BC600012780C121BB512D18EEB12D21A242DFAB7
:10BC70007B001222CD8A108B11AE10AF11EE4F70E7
:10BC80000302BD7B8E828F837401F08508108509C5
:10BC900011751200781012199E7C157D00EE241883
:10BCA00012BD7E1219CF8516108517117810121942
:10BCB0009E7C097D00EE240212BD7E1219CF7418FD
:10BCC000121C1212BF9C850A82850B83E0C0E0EE35
:10BCD000240F12AD25D0E012BDAEC0E0EE2411124B
:10BCE000AD25D0E012BDA9C0E0EE241012AD25D0E4
:10BCF000E012B3FEE51312BDD3E4F0A3F012BD8D44
:10BD0000780C121BD3EE241712AD25E51412B3D311
:10BD1000F8A3E0F9EE240D12AD2512BDCD12D188A5
:10BD200012D21A6025EE242612C1BC242DF812BDB1
:10BD3000C512D17A12B83912199E12D18612B8984A
:10BD40008A828B8312BD9A1219CFEE241912D21750
:10BD50005403601D90031412BBF2600CEEFAEFFB6B
:10BD600012B451122FE38013EEFAEFFB1222D380AC
:10BD70000AEEFAEFFB90030112BE1402D19DFAEF16
:10BD800012BD84223400FB1222AF740322EE24136E
:10BD900012BDDB22E0242B12B41A12BDA31222AF73
:10BDA000740322E0FAA3E0FB2212BDBCE02212BD24
:10BDB000B3E02212BDB72212BDBCA322F0850A82D5
:10BDC000850B83A322EF3400F98A828B8312BB692F
:10BDD000E50822F0EE242612BDDB22F582EF3400C6
:10BDE000F5832212B3CDA3A3A322F085088285098F
:10BDF000832212BDF62212B41EF8A3E0F98E828FC0
:10BE000083A3A3227B001222CD8A0A8B0BAE0AAF3A
:10BE10000BEE4F22E0F91222D92212BE1E2212BED0
:10BE20002F12BE2522E0F8A3E0F92212BE2F22F045
:10BE30008E828F8322C082C083E990121DF090030E
:10BE40001074D3F0A3742EF090031274C1F0A37495
:10BE50002EF090031474AFF0A3742E02B3AC74F7F9
:10BE6000121540EAFEEBFF8908EE4F70031227CB54
:10BE700090032212BBF27008900322802212C7DACC
:10BE800088828983A3A3A3A3A3A3A3A3A312BEB55C
:10BE900088828983A3A3A3A3A3A3A3A3A370DEEE95
:10BEA000F0A3EF12BEBBA3A3A3E4F0A312BEBBE5B5
:10BEB00008F002B50C12BDA3EA4B2212BEBF22123B
:10BEC000BEC32212CC66A3A3A32274F7121540901E
:10BED0000322800D8E828F83A3A3A3A3A3A3A3A376
:10BEE000A312D157EE4F60348E828F83A3A3A3A3F6
:10BEF000A3A3A3E06970DD8E828F83A3A3A3A3E035
:10BF00006A7003A3E06B70CC8E828F83A3A3A3A37C
:10BF1000A3A3E06C70BEEEFAEFFB80047A007B0016
:10BF200002B50C74F712154090032212D1579003FA
:10BF30002212AD30687002EB69701712BF8912C708
:10BF4000DA90032212BFA890032212D15780301238
:10BF5000D14AEE4F60298E828F83A3A3A3A3A3129D
:10BF6000AD2C687002EB6970E68A828B83A3A3A371
:10BF7000A3A3A3A3A3A312BF96A3A3A312BFA81214
:10BF80002351EEFAEFFB02B50C12B45DA3A3A3A3F9
:10BF9000A3A3A3A3A32212C1E5A3A32212C7DEEE8B
:10BFA000240BF582EF12BDDE12BB692274F012156C
:10BFB0004074FA121A4C8A088B098A828B83A3A3D5
:10BFC000A3A3A3A3A3A3E0600D640160098A828BED
:10BFD0008312BB7B6005790202C1B785088285099F
:10BFE00083A3A3A3A3A3A3A3A3E064037015740472
:10BFF000121C12AC82AD83AA08AB09122F93E97010
:10C000001380D385088285098312C7DA7404121C51
:10C010001212BFA812D16412D21A243212C1D01245
:10C02000234B8A0A8B0BAE0AAF0BEE4F700302C193
:10C03000B57C327D0079001222BB7402121C12AA58
:10C0400082AB83850882850983A3A3A3A3A3A3A3AB
:10C05000A3A3E0F91222077402121C12E0C0E0EE62
:10C06000242D12AD25D0E0F0EE242CF50AEF34009B
:10C07000F50B7403121C12E0850A82850B83F0799C
:10C0800001EEFAEFFB122EE585080C85090D750E01
:10C0900000780C12199E7C1C7D00EE240B12BD7ED4
:10C0A0001219CFEE243012C1BC2432080812BDC5CB
:10C0B0002411F8E50912D1C7FCE9FD8C828D8312A9
:10C0C000B679242E12AD2512BDCD12C53C12D194E5
:10C0D00012199E8C828D8312BB9E8A828B8312BD25
:10C0E0009A1219CF7404121C1212C1E112BFA89047
:10C0F000030212C1D7F0900302E00412C56E242A95
:10C1000012CA98750D00850A82850B83E0780C129F
:10C110001ADC8A828B83E50CF0EE242912AD25E52A
:10C120000C12CFF9E4F0E5082415F582E50912C1F7
:10C13000CA74015007121C1274018004121C12E40C
:10C14000F0EE242712B43D851882851983AA82ABAC
:10C15000831221EFE924FE850882850983F0F50822
:10C16000750900EE242E12AD2512BB9EECF8EDF9F8
:10C17000AA08AB0912130AE88E828F83A3A3A3A394
:10C18000A3A3A3A3F0ECF8EDF9AA08AB0912130AD4
:10C190008B09EA4509600F8E828F83A3A3A3A3A313
:10C1A000A3A3A3E004F0EE242012D217440812CB7C
:10C1B0001A790080027910740602B40E12D1C5FA01
:10C1C000E9FBEE22EE2415F582EF12C56AA2E02209
:10C1D000FAA3E03400FB2212BB8FA3A3A3A3A3A363
:10C1E0002212C1E52212BE258E828F83A3A3A3A3B0
:10C1F0002274F4121540EAFEEBFF12BBB7901268EE
:10C20000E0F8EE242B12D217C398400302C3641245
:10C21000CAB07015EE242B12D2170412C38DC0E0E1
:10C22000EE242912AD25D0E0F0EE242812D217FC1E
:10C230007900800109EE242C12AD41E9C398502603
:10C24000750801750900E97808121ADC12CAB055A0
:10C250000860E1E92CFC750801750900E97808120D
:10C260001ADCE04508F0EE242712C37BEE242E12E0
:10C27000AD25EC8A088AF0A4F8ABF0E42BF9E0983D
:10C28000F8A3E099F9C3E89508E99400EE40392451
:10C290002712AD4112CAB06037EE242D12AD25121F
:10C2A000C387A3E4F0EC7054EE242012D21744208C
:10C2B00012B854C0E0EE242612AD25D0E0F0EE24F2
:10C2C0003012C37BA3E08059242912AD2574FFF0FE
:10C2D00090033FE0FA90126BE0F508EA8508F0A4BD
:10C2E000ABF075F064A4FAADF075F064EBA42DFB2F
:10C2F0008E828F83A3A3EAF0A3EB80A8EE24201202
:10C30000D21754DF12BDD3ECF08C08EE242712D2E2
:10C31000178508F0A4FAABF0EE2430F582EF12C3D3
:10C3200072FBEE241E12AD25EAF0A3EB12C395C0FA
:10C33000E0EE242512AD25D0E0F0EE241C12AD2550
:10C34000E812C39B90032412BBF2600BECF912B409
:10C3500051122FE3E97018EE240BFAEF3400FB12B0
:10C360002F9F800B7BE9EE2422F582EF12C5460257
:10C37000AD1D12C56A2AFAA3E03B22F582EF12C373
:10C38000822212CB0CFA2212BB8FA3F022F0EE24F1
:10C390002A12C5672212BEBFA3E022F0A3E4F02256
:10C3A00074F412154090032212D15712241D8A0AE8
:10C3B0008B0B7CFF7DFF8020E0C398FAA3E099FB04
:10C3C000C3EA9CEB9D500E8E828F83A3A3E0C3989B
:10C3D000FCA3E099FD12D14AEE4F605912C7D6E591
:10C3E0000AC398F8E50B99F98E828F8312CADFC3CE
:10C3F000E89AE99B8E828F83A3A340BCA3A3A3A347
:10C40000E06402701DEE240B12CAB3600CEE24101F
:10C4100012AD2512CAE11222D3EEFAEFFB122ED989
:10C420008007EEFAEFFB122ECD7A017B0090121DF1
:10C4300012B3F8801474FF6C700374FF6D600A7A95
:10C44000017B0090121D12B3BF02AD1D74F01215D6
:10C45000408A088B09ECFAEDFB890A7C0112D16451
:10C4600012CAA28A0C8B0DAE0CAF0DEE4F700302F8
:10C47000C539E50A600302C539E50812C53CE0F894
:10C48000EE242812D21768600302C539EE242C125C
:10C49000C37BE82AF8E43400F98E828F83A3A3A338
:10C4A000A3A3A3A3A3E0FAE89AE99400C365D03359
:10C4B000401412C7C112CAB6700C7B0012D15DE5E0
:10C4C0000912C546807312C7C112CAB67031EE2474
:10C4D0002C12D217F9EE242912AD257508FF750923
:10C4E00000E97808121ADCE508F0EE242A12AD25DE
:10C4F000E50812C55F29F0EE242B12B3F08022E587
:10C50000082414F8E5093400F9E0C0E0EE242A120A
:10C51000AD25D0E012C55AC0E0EE242912AD25D0D9
:10C52000E012C56E242D12AD2512B430A312C39BA8
:10C530007A01FB90121D12B3F802B4112413F58294
:10C54000E50912BDDE2212C382EE241412BDDB12F5
:10C55000BC2AEEFAEFFB122ED92212B878E022F0B4
:10C56000EE242812C56722F582EF12CB0C22F012BE
:10C57000D1A2F0A3EBF0EE2274E812154074FD1284
:10C580001A4CE9851882851983F08A0A8B0B8C1660
:10C590008D17741B121C1212C7B9741D121C12784D
:10C5A0000C121BB58A828B83A3A3E0F91221E38AC4
:10C5B000128B13EA451370077A007B0002C7B47A26
:10C5C000127B0012234B8A088B09AE08AF09EE4F8D
:10C5D000700302C7B07C127D0079001222BB740187
:10C5E000121C12AA82AB83850A82850B83A3A3E067
:10C5F000F9122207EE240FF508EF12D1817402120E
:10C600001C12E0850882850983F07902EEFAEFFBBF
:10C61000122EE585168285178312C1E1E8F0A3E9A1
:10C6200012C8058E828F83A3A3A3A3A3A3A3F0752F
:10C6300014FF751500850882850983E07814121AA5
:10C64000DC12AD22E514F0851282851383A3E0F895
:10C6500012B91AC0E0EE240B12AD25D0E012C80FBB
:10C66000F508EE240D12AD25E508F012CABBE085F1
:10C6700008F0A42424FAE5F03400FB1222CD8A0845
:10C680008B09EE241012AD2512BBBEEA45097003DA
:10C6900002C7A58A828B83741A12C39B8A828B83FA
:10C6A000A3A3F0A312C7F912C7E212BFA8AC16AD3C
:10C6B00017EA2406FAEB3400FB122201850A828570
:10C6C0000B83A3A3A3E0C0E0E508240FF582E509EE
:10C6D00012AD28D0E0F090035C12C7DAE508241010
:10C6E00012C7CA12C81FA312C7DAE508241212C75C
:10C6F000CA12BDAEC0E012C7C112AD28D0E0F0E54D
:10C700000A12CA93E50B12D21AC0E0E5082415F507
:10C7100082E50912AD28D0E012C7F0C0E0E5082498
:10C7200016F582E50912AD28D0E012D21EE0C0E075
:10C73000E5082417F582E50912AD28D0E012D21ED3
:10C74000A3E0C0E0E5082418F582E50912AD28D081
:10C75000E012BB61C0E0E5082419F582E50912ADDD
:10C7600028D0E0F0E508241AF582E50912AD287812
:10C770000C121BD3E5082424F8E5093400F9E50878
:10C780002422F582E50912BFA5E50A12D15FE50B67
:10C7900012D21AC0E0E508241FF582E50912AD287F
:10C7A000D0E0F0800BEEFAEFFB122ED97E007F0076
:10C7B000EEFAEFFB740302D19AE0F510A3E0F51155
:10C7C00022E5082414F582E50922F582E50912BD67
:10C7D000DEE8F0A3E9228E828F8312C7DE2212BE2A
:10C7E0002522E0F8A3E0F98A828B83A3A3A3A322E6
:10C7F000F0851082851183E02212C7FD2212BDB799
:10C80000A3A3A3A322F012D16CE50B12C56A22F0F8
:10C8100012C81712C56A22E50A12D18FE50B22123F
:10C82000C7FDA3A3A32274E81215408A0A8B0B8CC0
:10C83000108D1189147418121C12E0F516A3E0F57E
:10C8400017741A121C12780C121BB5750900EA2411
:10C8500013F582EB12D21AF50890032412BBF26092
:10C8600011A90890032412B44E122FE3E9600302C9
:10C87000CA907C0285108285118312CAE112D16CA4
:10C88000E50B12CAA28A128B13AE12AF13EE4F70D1
:10C890004B850A82850B83A3E0A2E0400302CA9085
:10C8A000780C12199A78161219A2A914AC10AD11AD
:10C8B000AA0AAB0B122EBB74061219CF8A0C8B0D71
:10C8C000AE0CAF0DEE4F700302CA908E828F83A321
:10C8D000A3A3A3A3A3A3A3E50812CB1A85080C8ED8
:10C8E000828F83A3A3A3A3A3A3A3A3E024FFF8E4BD
:10C8F00034FFF9E8650C7001E97003750901EE2455
:10C900000B12CAB3700302CA43850A82850B83A344
:10C91000E0A2E0500375080012CAECE50C98E49917
:10C92000C365D033401EE0F8EE240E12D21728F073
:10C93000750CFF750D00E8780C121ADCEE12CA9324
:10C94000EF12CAA912D173E50B12B83912199E124F
:10C95000B89585080CEE240D12D217850CF0A4F8BA
:10C96000A9F0EE241012D217242212B6A128FAA39D
:10C97000E039FB12B88F1219CF750C0112CAC778B3
:10C980000C121ADC12D214450CF0E509A2E0506535
:10C99000EE240C12CA9812CAC704780C121ADC8A48
:10C9A000828B83E0450C12CB1285080C850CF0A419
:10C9B000F812C81712D21AFCE82CFCE5F03400FD7E
:10C9C000EE241012AD2512CAE512CC53F47026EEF7
:10C9D000240BF50CEF3400F50DEE241012AD2512EA
:10C9E000CAE1850C82850D8312BE14850C82850DEB
:10C9F0008374FF804D12BBB790033FE0FA90126B37
:10CA0000E0F50CEA850CF0A4FAABF0F8EBF9901223
:10CA100068E0F50CE8850CF0A4F8ACF0850CF0E9C2
:10CA2000A42CF9EA28F8EB39F9E875F064A4F8AA1F
:10CA3000F075F064E9A42AF98E828F83A3A3E8F04D
:10CA4000A3E9F012CAEC12D141E8650C7001E9606B
:10CA50000EEE240C12CAB36006E509A2E05031EED6
:10CA6000240E12D217C0E012CABBD0E0F012D214CA
:10CA7000C0E0E50A2414F582E50B12AD28D0E0F001
:10CA8000AC0AAD0B85108285118312CAE1122E917A
:10CA900002D19D240CF5822212D1C5FAE9FB750C56
:10CAA000FF2212CBBD122EDF2212BDDEE50CF022DA
:10CAB000EE2429F582EF12C56AF422E50A2413F563
:10CAC00082E50B12BDDE22750D0012CB02F5F0E5FA
:10CAD0000884E5F0228E828F83A3A3A3A3A3A3A33C
:10CAE000A312BDA322E0242012B41A2285080CEE62
:10CAF000240E12C567F812CB02FAE82AF8E43400D3
:10CB0000F922EE240FF582EF12CB0C223400F583CC
:10CB1000E022F0EE240D12C56722F07A017B00902E
:10CB2000121DE0F912230322C082C08390121D124D
:10CB3000BE1402B3AD74F41215408A088B09EB548D
:10CB400080703BEAA2E05047122EC7E5086401FA64
:10CB5000AB09803F8E828F83E06401701A12BD8D15
:10CB600012186112AC471219A2EE241212CBA612AF
:10CB70002EB574061219CFEEFAEFFB1222D39012E3
:10CB80001D12CB9670CEAA08E5096480FB80047A5A
:10CB9000007B0002AD1DE0F91222DF8A0A8B0BAE8A
:10CBA0000AAF0BEE4F22F582EF12CBBDEE2402FC52
:10CBB000EF3400FDEE2418FAEF3400FB2212CB0C08
:10CBC000F922C082C08390032680048C828D831258
:10CBD000CC0460298C828D83A3A3E069600574FF77
:10CBE0006970E88C828D83A3A3A3E06A7003A3E03D
:10CBF0006B70D8EC2403FAED3400FB80047A007BE0
:10CC00000002B3AD12BBA2EC4D2274F7121540E93D
:10CC1000FC74FE6C70047D0180027D009003268010
:10CC2000096C70027D018882898312BBF2601F88C3
:10CC3000828983A3A3A3E06A7003A3E06B70E7ED8E
:10CC4000A2E088828983A3A3E050D6F9800279FE0E
:10CC500002B50CECF0A3EDF08A828B83E02212CCBB
:10CC6000622212CC6622F08E828F83A3A3A3227449
:10CC7000F61215408C828D83A3A312CE6DF0EA24A8
:10CC800017F582EB12D21AC0E0EC12D18FED12AD83
:10CC900028D0E0F0EA241DF582EB12AD2812C7DAA5
:10CCA000EC12D1C0ED12AD2812CE6DA3F0A3F0129C
:10CCB000D1BFEB12AD2812CE5FA3A3A3A3A3A3EE13
:10CCC000F0A3EF12C55AFE8C828D8312CE8C7403B2
:10CCD0005EFEC39403400FEC240D12B817EC241031
:10CCE00012B81702CE47EE600574026E70748C8223
:10CCF0008D83E0540CFE740C6E700302CDE4E0A250
:10CD0000E4400D88828983E08C828D83A312CEB6A5
:10CD100074086E600302CDE4EC12CA93ED12B49372
:10CD2000F08A828B83A3A3A312CFB770148C828D59
:10CD300083E0440C12CE7BA3A312CE5FEEF0A3EFF0
:10CD4000F08C828D83E0A2E4401812CE4A12CE9974
:10CD500012CE53A3A312CE998C828D83A3A3A312C8
:10CD6000CE8C88828983E0C0E0EC12D16EED12ADEA
:10CD700028D0E012CE8C8C828D83E0A2E7507C8894
:10CD8000828983E0FE8C828D8312CEB674FC5E6055
:10CD90000302CCD78C828D83A3E054036403700319
:10CDA00002CCD78C828D83A3E054036051888289A2
:10CDB00083E0C0E0EC2413F582ED12AD28D0E01240
:10CDC000CEB78C828D83E0540364027031888289EF
:10CDD00083E0C0E0EC2414F582ED12AD28D0E0121F
:10CDE000CEB7801AEC240C12B817740C6E600302D4
:10CDF000CD2112CE4A12CEA402CD41A3E4F0EC1212
:10CE0000D175ED12BFA5EC2410FEED3400FFEA242D
:10CE10001DF582EB12D21AF5088E828F83E0C3983B
:10CE20002508F508F0EA2417F8EB12B439C3950881
:10CE3000C0E0EC12D1C0ED12AD28D0E012C55AC34B
:10CE40009508500302CCD702B3DC88828983E012B4
:10CE5000CE5322F508A3E0FFE5088C828D8322E003
:10CE6000FEA3E0FF8C828D83A3A3A3A322E412CEB2
:10CE70007222F08C828D83A3A3A32212CE83A3A35C
:10CE8000A3A322F08A828B83A3A3A32212CE94A809
:10CE900082A9832212B878A322A3A312CEA48882E7
:10CEA0008983E022A3A3A3A3F0A3EFF0E824020860
:10CEB00008E93400F922A312CE9408A9832274F55C
:10CEC00012154074F3121A4C8A088B09ECFEEDFF20
:10CED0008E828F83E0540CF50AE0A2E75006E50A43
:10CEE000D2E7F50AE50AD2E1F50A12CFB97006E5F4
:10CEF0000AD2E4F50AE0A2E55006E50AD2E5F50A11
:10CF00007C087D007900851882851983AA82AB830D
:10CF10001222BB7402121C12E50A12CFECE0C0E030
:10CF20007403121C12D0E012CFF912B26E74051203
:10CF30001C1212B845121C12E070797408121C12EF
:10CF4000E0241212B41612BBA8C0E07408121C121E
:10CF500012CFD4D0E012D00CC0E07408121C121210
:10CF6000B265D0E0F07408121C1212BF9612CFDB2B
:10CF700012B85412CFBF12BBBEEE241112D217C08A
:10CF8000E0E8242EF582E912AD28D0E0F0EE24147A
:10CF900012D217C0E07408121C12E0243112B41629
:10CFA000D0E012CFF1C0E07408121C1212CFCDD025
:10CFB000E012D00502BBD1A3A3E05403640122FA1E
:10CFC000A3E0FBE82428F582E912BDDE22E024304C
:10CFD00012B41A22E0242212B41A2212BDA3E824A9
:10CFE00026F582E912BDDEEAF0A3EB2212BE2BA3E6
:10CFF00022F0EE241312C5672212CFFD22F085180D
:10D00000828519832212B883122F092212CC5EE086
:10D010002274F71215407E008A828B83A3A3A3A3F8
:10D02000A3A3A3A3A3E06402607B12B82C12D21ABC
:10D03000707312BC2412AD2812BBF260688882891A
:10D0400083E05403705FA3A3A3A3A312D0A8E06A54
:10D050007003A3E06B704E8882898312D0A8A3A3CB
:10D06000E0FFA3E0F5838F82A3A3A3A3A3A3E06AB9
:10D070007003A3E06B702E88828983A3A3E0F88CF1
:10D08000828D83A3A3E0F9A3E0F5838982A3A3E0C3
:10D090006860118C828D83A3A3E0F812B91A540C36
:10D0A000640470010E02B2AAA3A3A3A312BDA38CB1
:10D0B000828D832274F612154074FC121A4CEAFE1B
:10D0C000EBFFECFAEDFB8A828B83A3E0540360163E
:10D0D00090031212BBF2605C7900EEFCEFFD12B41B
:10D0E00051122FE3804E851882851983EEF0A3EF4D
:10D0F000F07402121C12EAF0A3EB12CFF9AC82AD6D
:10D10000837A8B7B2E121E0B8A088B09A808A9092B
:10D11000E849602088828983A3A3A3A3A3A3A3A330
:10D12000A37406F07A0088828983E0240C12D13936
:10D13000F9121D5D740402B3D912D13D2212BB83D2
:10D1400022E824FF18E934FFF9228E828F83A3A3FB
:10D15000A3A3A3A3A3A3A3E0FEA3E0FF22E50824C7
:10D1600012F58222E50812D16EE50922E50A2411A2
:10D17000F58222E50A240EF58222240EF582E509C5
:10D18000223400F50922E50812D18FE50922EA24AC
:10D1900010F5822212D1D0780C221219CF7F100202
:10D1A000175912241D8E828F83EA2212D1AF2212C8
:10D1B000D1B7EEFAEFFB22121E5FEAFCEBFD22EA8A
:10D1C000240DF58222F8EF3400F9E82212D1D022A2
:10D1D000E0F50CA3E0F50D2274F7121540890890D4
:10D1E000032812BBF2600AA90812B451122FE3807F
:10D1F00002790102B50C74F7121540E9FE90032A7A
:10D2000012BBF2600AEEF912B451122FE3800279D8
:10D210000002B50CEE240CF582EF12C56A22F085EF
:10D220001082851183A322C082C0838A828B83E00F
:10D23000D2E7F012253702DCB1C082C08379001238
:10D24000D6D112EA38C082C08390032C12E668D08F
:10D2500083D082C3E09CA3E09D500C12EBF0FAA3B4
:10D26000E012D26A60010902DCB1FBEA75F00BA49E
:10D27000FAA8F075F00BEBA428FB90032EE02AF837
:10D28000A3E03B8882F583E0540F2274F712154027
:10D29000890812D6D112D777ACF075F00BE9A42C1F
:10D2A000F990032EE028FEA3E039FF7401650860C1
:10D2B000067402650870208A828B8312D76312E39A
:10D2C0006A74026508701B12D62212D7AA70138ED8
:10D2D000828F83E4F0800BEA2403FCEB12D7451223
:10D2E000D751EEFAEFFB122F4502DFD774F4121577
:10D2F0004012EFDC79008E828F83E06076890A89A4
:10D300000B8065E50A75F00BA4FAA8F075F00BE543
:10D310000B12D2777046E50A75F00BA4F8AAF075E7
:10D32000F00BE50B12D7898E828F83E0850882850A
:10D33000098312D86B850882850983A312E36AEEFC
:10D340002403FCEF12D74E12DAC712E9C7AA08ABC2
:10D3500009122F45790190032C12E683E50A240176
:10D36000F50AE50B3400F50B12D62AE50A9AE50B0F
:10D370009B409002E74774F5121540EAFEEBFF74FC
:10D380000B121C1212DE89750A01EC4D602BEC1297
:10D39000EFF8ED12EA3812E3617901122F27E50860
:10D3A0004509606F850882850983A312EFE679023B
:10D3B000AA08AB09122F27805AE5084509602B12ED
:10D3C000EA4812E41912DAC812D794700CEEFAEF98
:10D3D000FB122F21E9F50A80CBEE2403FA12D6CCFA
:10D3E00070317903EEFAEFFB80CA8E828F83A3E05F
:10D3F00064FE7003A3E0F4700BEE24030A0A0A1221
:10D40000D6CC700CEEFAEFFB122F21E9F50A80035F
:10D41000750A00A90A7F0302175974F71215409084
:10D42000032C12DFDCEA4B602FEA75F00BA4FAA89C
:10D43000F075F00BEBA428FBEAFEEBFF12234B90F8
:10D44000032E12DFDC90032E12E66F6012EEFCEF6B
:10D45000FD79001222BB800790032EE4F0A3F002B6
:10D46000DFD790032C12E5F3C3EE98EF9922C08228
:10D47000C083EC4D6005122B4380097C087D007948
:10D48000001222BB02DCB174F61215407900EA4B9F
:10D4900060187800880812EBBBEB12EBEC600479A3
:10D4A00001780808E8C3940840EA02D9F774F71233
:10D4B000154074F3121A4CECFEEDFF8518828519A5
:10D4C00083E4F004121C12EAF0A3EB12E75A74038F
:10D4D000121C12AC82AD83EEFAEFFB1225AFEEFA0E
:10D4E000EFFB121C2502DFD274F712154074F31201
:10D4F0001A4CECFEEDFF851882851983E4F0EAFCF6
:10D50000EBFD7403121C1212D8647401121C121267
:10D51000DFF08E828F8312E36A74FE68700374FFFB
:10D5200069600479018002790002DFD2A90802DF74
:10D53000D774F7121540EAFEEBFF7508008E828F54
:10D5400083E0602212D568701D12D5738A828B83A6
:10D55000E08F838E82F8E058700CE0F88A828B832B
:10D56000E048F0122F4580C4122F2DE9F508740110
:10D5700065082212EFF112D77B12D6BDFAA3E0396B
:10D58000FB2274F41215408A088B097C007D00127E
:10D59000D62212D75112D6E212EFE3790085088223
:10D5A000850983A3E064FE7003A3E0F460717E004C
:10D5B0007F008062EEFAEF12D26A6057EEFAEFFB5C
:10D5C000EA75F00BA4FAA8F075F00BEBA428FB9019
:10D5D000032EE02AF50AA3E03BF50B8508828509B6
:10D5E00083A312E750850A82850B83A3E06A700348
:10D5F000A3E06B701EE50A2403FAE50B12D6CD708A
:10D600000AE50A2403FCE50B12D74E12D6D679019F
:10D6100012EA4F12DA0D12D62AEE9AEF9B409502CB
:10D62000E747EA24030A0A0AEB2290032C12EA04D1
:10D63000C32274F31215408A088B098A828B83A354
:10D6400012EFE612D6D112EFE3750C0012D62212B9
:10D65000D6CD70547E007F00804912D6AFFAA3E089
:10D66000398A82F583E0540F603612D6AFF50AA3EB
:10D67000E039F50BE50A2403FCE50B12D75834001A
:10D68000FB122B3DE964017017850A82850B83A389
:10D6900012EA17A312E36A12D6D6750C0112EA4FEA
:10D6A00012DA0D12D46240B2A90C7F05021759EEAE
:10D6B000F8EFF9E875F00BA4F812D6BD22AAF075C0
:10D6C000F00BE9A42AF990032EE02822EF12D7A448
:10D6D0002212EFF7EB2212D6E212DAD1EEF0A3EF2C
:10D6E000F022E50812EFF8E5092274F5121540EA78
:10D6F000FEEBFF8E828F83A312EFE67C007D00EEAF
:10D7000024030A0A0AEF12D751EEFAEFFB122F2D6B
:10D71000E9F50A7401650A702912EFF112D777AAA8
:10D72000F075F00BE912D789850882F58312D7636B
:10D7300012D794700DE5082403FCE50912D74512B1
:10D74000D75102D4133400FDEE2403FAEF2212D78E
:10D75000583400FB1225AF223400FDE5082403FAFB
:10D76000E50922A312D7682212D76C22E0F8A3E0C1
:10D77000F98E828F83A32212D77B223400F5831285
:10D78000E5F7E875F00BA4F82212D6C3F508A3E07C
:10D7900039F50922E8F0A3E9F0E5082403FAE509E0
:10D7A00012D7A42212D7AA6401223400FB121C252E
:10D7B000E92274F312154074E6121A4C12EFDC756C
:10D7C0000C01750800750900750A00750B008518B5
:10D7D00082851983E4F0EE2403FCEF3400FD74032A
:10D7E000121C1212D864E964017023740B121C120B
:10D7F00012E3617401121C1212E7547003A3E06972
:10D800006051851882851983858208858309740D86
:10D81000121C12E412D86B740E121C1212E36A74FA
:10D820000D121C12AA82AB83121C3DE96401700B1D
:10D83000740D121C1285820A85830B780A1219A2B4
:10D84000AC08AD09EEFAEFFB122F1B74021219CFD0
:10D85000E9F50CEEFAEFFB121C37A90C741A121939
:10D86000CF02D6AA12D903121C4322F08E828F83D4
:10D87000A312E5F32212D9FCC3E89AE99B22E8241B
:10D880000108E93400F922E493F8740193F9227451
:10D89000F212154074F3121A4C8A088B09ECFEED53
:10D8A000FF750A00EEFAEFFB121C618A0C8B0DA8C3
:10D8B0000CA90DE849603E88828983E06508700400
:10D8C000A3E06509602F88828983A3A3A3A3E0C393
:10D8D0009405502112EA3C8518828519837401F061
:10D8E000121C1212EA40EEFCEFFD7403121C12121D
:10D8F000D8FC750A01A90A740D02E40512D90312B5
:10D900001C4F22AA82AB831225AF8518828519830A
:10D91000AA82AB8322C082C083EAFCEBFD7A007B43
:10D920000002DCAEC082C0837C007D0002DCAE74ED
:10D93000F412154074F3121A4CEAFEEBFF8C0A8DB8
:10D940000BC3EC94F8ED94FF4007EE4F700302D93F
:10D95000E4750800750900802A851882851983748A
:10D9600001F012DA26121C1212DA34601374031258
:10D970001C12AC82AD83EEFAEFFB122B3DE9704531
:10D9800012DE73903425E412EC0BE50898E5099952
:10D990005052E50875F012A4F8AAF075F012E509E6
:10D9A000A42AF912EBFE60D8EE4F70AD74FF650A41
:10D9B000700474FF650B60C812DA16650A7004A360
:10D9C000E0650B70BBE50875F012A4F508A8F075CA
:10D9D000F012E509A428F50974962508FA740B35A8
:10D9E00009FB80047A007B0002E74212E64BC3EA9F
:10D9F0009CEB9D221219CF7F02021759E493FA740F
:10DA00000193FB22EA24010AEB3400FB22EE2401FD
:10DA10000EEF3400FF2212DA1A22749628F582746F
:10DA20000B39F583E022749828F582740B3912E5DE
:10DA3000F1740B22E8F0A3E912E382121C49E922F7
:10DA4000C082C0839003387499F0A3741DF002DC87
:10DA5000B174F7121540EAFEEBFF90035EE0640834
:10DA6000601BE0640460168E828F83E054036401BF
:10DA7000704812DAC712E3FCE06406703D8E828FB4
:10DA800083A3A3E064FE7003A3E0F4602D8E828F75
:10DA900083A3A312DFF090034FE0687003A3E06953
:10DAA000700BEE2415F582EF12EBEC6008121E29C4
:10DAB000E9F5088008121E2F80F67508C2EEFAEF0D
:10DAC000FB12235102D52CEE12DACC22240BF58264
:10DAD000EF3400F5832274F41215408A088B098A0A
:10DAE000828B83E0F8A3E0FAE82AFAE43400FB1220
:10DAF000234B8A0A8B0BAE0AAF0BEE4F6060850892
:10DB000082850983E0FC7D0079001222BB8E828F22
:10DB100083A3A312EFE6121E658E828F83A3A3A3B5
:10DB2000A312DFDC850882850983E0F8EE28F8EF90
:10DB3000340012E365850882850983A3E0C0E01202
:10DB4000EA32D0E0F0121E77EE240E12EA35E91226
:10DB5000E738E0C0E0EE241112EA35D0E0F0EEFA4A
:10DB6000EFFB02E74774F412154074EB121A4C8A6B
:10DB7000088B098C0A8D0BE9FE90035EE06404605B
:10DB800005E06408700479C2802EA37808121BD3C4
:10DB9000EE90036512DCEF121BD37405121C12E920
:10DBA000F07404121C127401F07407121C12E4F0D9
:10DBB00090035E740212DCA7741502E74474F61237
:10DBC000154074EB121A4CEAFEEBFF12E66C600390
:10DBD00002DC617A077B0012234B90033012DFDCFA
:10DBE00012E66C60788E828F83121BEF90033112E5
:10DBF000E3FF121BFB12EEB8C0E012DC6DD0E0F0C8
:10DC0000EE2405FAEF3400FB8A088B098A82F5833B
:10DC1000E0C0E012DC68D0E012DC83E0C0E012DC9F
:10DC200068A3D0E012DC7D121BEF85188285198372
:10DC3000121BFB88828983E0C0E07405121C12D09D
:10DC4000E0F0850882850983E0C0E07404121C12AC
:10DC5000D0E0F07407121C1212DCA6800679108046
:10DC6000027901741502D9F412DC6DA322900330FD
:10DC7000E0FAA3E0F5838A82A3A3A3A322F08E8215
:10DC80008F832212E37822C082C08312E66C600D7B
:10DC900090033012E9F9900330E4F0A3F0121DB1C3
:10DCA000121F0102DCB1E412E382122E4922121C7F
:10DCB00067D083D08202196774F412154074EB1296
:10DCC0001A4C8A088B098C0A8D0B90035E74011222
:10DCD000DCEF121BD37405121C12E9F07404121C41
:10DCE000127403F07407121C1212DCA602DBB812C5
:10DCF000DFE278082274F71215407C01121C9D02A5
:10DD0000DFD774F212154074FC121A4CE9851882A0
:10DD1000851983F0EAFEEBFF8C0A90035C12E6683B
:10DD2000121DA58A088B09EA4509700579CA02DE29
:10DD30006E8A828B83A3A3A3A3A3A3A3E064FE7034
:10DD400003A3E0F4700579C302DE6E90035C12E772
:10DD500050121F25850882850983A3A3A3A3A3A32B
:10DD6000A3A3A3A3E00490036F12DFC57402121CE7
:10DD7000127402F014121C12AA82AB83121EB98A0A
:10DD80000C8B0DAE0CAF0DEE4F700302DE6512DA98
:10DD9000C712E40D7406F0A3A882A9839003491268
:10DDA000EA0A12E5D0F0EE241312EA35740112E902
:10DDB000A77440F0A3E412E731A3A312DE8012E3BC
:10DDC0006AEE241112EA35E50AF0EEFAEFFB121CB6
:10DDD00073E9FE600302DE6790035E7409F0E508F4
:10DDE000240712DE77AA08FB794B122E3D850882A4
:10DDF00085098312DFB712E36A900351E0F88518B2
:10DE000082851983E068600CE090035112E37E790B
:10DE1000E1122E3D90125212DFF0901254E0687021
:10DE200003A3E069601A90033212E36A901254125D
:10DE3000E750121E8F90125412E6687A0112E653D0
:10DE40007A007B049003A9E0F91224059012541281
:10DE5000DE8974027808121ADCAC08AD09FA7B047A
:10DE600012E65580027E1090053AE4F0EEF9740453
:10DE700002E405E5082401F508E5093400F5092266
:10DE800012DE842212D76CA322E0F508A3E0F50984
:10DE90002274F612154074E2121A4C851882851904
:10DEA00083ECF0A3EDF0EAFEEBFF89087428121C66
:10DEB00012E0F50990035EE064046005E064087018
:10DEC0000579C202DFB27429121C12E064FE7003ED
:10DED000A3E0F4700579C302DFB290035E7403120D
:10DEE000E37E7950122E3D7429121C12AA82AB8354
:10DEF000794B122E3D85188285198312DFBE12E3FD
:10DF00006AE508900351F07429121C1212DFB7124F
:10DF1000E36AE50990034912DFC574CE55094480D0
:10DF2000C0E07412121C12D0E0F0740F121C1274B4
:10DF300002F07429121C1212DFF07407121C121264
:10DF4000E36A12DFEA7410121C1212E36A740512FB
:10DF50001C12E508F0741B121C12E4F090036474A8
:10DF60000FF07A647B037954122E3D900363740F93
:10DF7000F07A637B037947122E3D900363E0C394EC
:10DF80000F50237405121C12E0C0E07402121C1220
:10DF9000D0E0F07404121C127401F004121C12AAD6
:10DFA00082AB83122E4F7405121C12AA82AB83120D
:10DFB0002E43741E02D9F412E5F39003522212E5A7
:10DFC000F390035C22F0EEFCEFFD7A707B03122BE2
:10DFD0004322740D1219CF7F01021759EAF0A3EB07
:10DFE000F022F0851882851983228518828519838D
:10DFF00012E5F32274F412154074F9121A4C8A08CF
:10E000008B098C0A8D0B8518828519837808121B61
:10E01000D37404121C12E9F07405121C12E4F0749B
:10E0200006121C12E412E37E121C85740702E744F8
:10E0300074F41215408A088B098A828B8312EA5283
:10E04000EE4F700302E13990030C12E66F60158AFF
:10E05000828B83A3A3E0F9EEFAEFFB90030D12E3AA
:10E06000FF122FE38E828F83A3A3A3A3A3A3A3A353
:10E07000A3E0640270718E828F83A3A3A3A3A3A3E2
:10E08000E05402700302E10B850882850983A3A393
:10E09000E064E960768E828F83A3A3A3A3A3A3A3E6
:10E0A000A3A3A3E07014901268E0048E828F83A370
:10E0B000A3A3A3A3A3A3A3A3A3F08E828F83A3A34D
:10E0C000A3A3A3A3A3A3A3A3E01412E13C7404F0AD
:10E0D00090126912E9A1E8F0A3E912EC4A8B0BEA6D
:10E0E000450B700312EBC68E828F83A3A3A3A3A359
:10E0F000A3A3A3A3E0640260128E828F83A3A3A3D1
:10E10000A3A3A3A3A3A3E06406702E8E828F83A390
:10E11000A3A3A3A3A3E0A2E0501F850882850983DF
:10E12000A3A3E0F9EEFAEFFB122EF78E828F83A302
:10E13000A3A3A3A3A3E054FEF002E74712E378A34E
:10E14000A3A32274EC12154074DD121A4CEAFEEB04
:10E15000FF8C088D097437121C12780C121BB575D0
:10E160000A007405121C12AC82AD83122E97741231
:10E17000121C12E070087415121C12E06020740565
:10E18000121C12E0A2E6501E8E828F83A3A3A3A3CB
:10E19000A3A3A3A3A312E750121EC5E96008790345
:10E1A000122B2B02E34F7405121C12E0540C640472
:10E1B0007005750B018003750B00E0A2E550197521
:10E1C0000A01E50BA2E0401012EFED12E74C122F0E
:10E1D00003E96004790480C87405121C12E0A2E609
:10E1E00050227406121C12E0540370187405121C9D
:10E1F00012E0540C640C600CE0540C64086005756B
:10E20000100180037510007405121C12E05403F80D
:10E21000740268700C12EFED12E74C12255502E300
:10E220004F740168703AE510A2E0500312E357748E
:10E2300005121C12A882A9837403121C12E8F0A311
:10E24000E912E5E785188285198312E370E0C0E0E2
:10E250007402121C12D0E012E37E122FBD02E34FB3
:10E26000E8600302E34F900346E0640170108E8281
:10E270008F83A3A3A3A3A3A3E0700302E1D474221A
:10E28000121C12740212E5E7741A121C1212E36ACD
:10E29000E510A2E050087405121C1212E357E50BBA
:10E2A000A2E0EE5069240FF582EF12EBECC0E074AF
:10E2B00017121C12D0E0F090030E12E66F700302EA
:10E2C000E34F121E658A128B13A812A913741A1237
:10E2D0001C12E0687003A3E0697074780C12199A3C
:10E2E000780A1219A678081219A2A910740C121C27
:10E2F00012AC82AD837421121C12AA82AB839003EC
:10E300000E12E3FC122FE374071219CF8041FAEFCB
:10E31000FB122FA5E96038780C12199A780A1219A5
:10E32000A678081219A290035C121865EE2412F563
:10E3300082EF12EBC17423121C12AC82AD83740EF7
:10E34000121C12AA82AB83122EF174091219CF7417
:10E35000231219CF02EC4512EFED12EA00122E91B2
:10E3600022E0F8A3E0F9EE12DACCE8F0A3E9F0221B
:10E37000E8F0A3E912E3782212EBDCA3A32212E374
:10E38000822212DFE2AA82AB832274F712154012B6
:10E3900024FB02DFD7C082C08312250702DCB174E0
:10E3A000F712154012250D02DFD7C082C083122557
:10E3B0001302DCB1C082C08312251902DCB174F7EC
:10E3C00012154012251F02DFD774F71215401225CF
:10E3D0003102DFD774F7121540EAFEEBFF890874AB
:10E3E00001650870147900121D09903438E493FC1B
:10E3F0007900EEFAEFFB121CEB02DFD7E0F8A3E0A6
:10E40000F5838882221219CF7F0602175912E41170
:10E410002212E5F7888289832212E5F3EE2212EBBD
:10E42000F8692274F012154074F5121A4C8A088BA0
:10E4300009890A8C0BE9A2E050147508FC7509FFE4
:10E44000A2E15005D2E402E4E5D2E302E4E512E7FA
:10E45000207003A3E0697005790002E5B2AC0A7987
:10E4600002AA08AB09121D27E960EDE50AF50C7850
:10E470000C1219A679027CFE7DFFAA08AB0912E6F0
:10E48000731219CFE9600302E5B0E50AC2E5F50AA7
:10E4900090039CE07051E50AA2E6404B7403121C05
:10E4A00012AC82AD83AA08AB09121C2BE9703212A0
:10E4B000E65E8A0C8B0DA80CA90DE8FEE9FFE84981
:10E4C0006025EE24020A0AEF12D7AA601AEE24028F
:10E4D000FCEF3400FD7403121C12AA82AB83122BD2
:10E4E00043E50AD2E5F50A90033AE0F50C90034FB4
:10E4F000E0F50EA3E0F50F780E1219A27D017C0065
:10E5000090033AE0F9AA0EAB0F121D0F7402121914
:10E51000CFE9F890033AE004F0E8600302E5B0E5E3
:10E520000AA2E55004740E80027406C0E074011261
:10E530001C12D0E012EA588A0E8B0FAE0EAF0FEE0F
:10E540004F606912E5D012E5E7888289837401F093
:10E550007478550AA312EFFDE50C12EFFDA3E50850
:10E56000F0E50912E5BFE4F0E50AA2E5500F7403F7
:10E57000121C12AC82AD83E8240612E5B68E828F9F
:10E5800083A3A374FDF0A374FFF0E50B6015903432
:10E5900039E493F8E50BC3985009EE241312EA35D9
:10E5A000E50BF0EEFAEFFB121C7380067910800287
:10E5B00079C7740B8047FAE93400FB122B43228899
:10E5C000828983A3A3A3A312E5CB2212EA28A32264
:10E5D000EE241712DACE7401F0121E5FEE241A1226
:10E5E000DACEEAF0A3EB22F012EFF1340012E5F1FB
:10E5F00022F58312E5F722E0F8A3E0F9221219CF01
:10E600007F0802175974F61215407A007B1012EB3E
:10E61000D360089003BB7401F08029900ABCE064C9
:10E62000019012667006E0FC79018004E0FC790339
:10E630007A007B00121CEB90342D12E6477A007BA7
:10E640001012E65502D9F712E64B22E493FC74014E
:10E6500093FD227B009003A9E0F91223F922900395
:10E660005C12E679121F132212E9BB2290033012CA
:10E67000EA1122121CFD740122E0FCA3E0FDAA08AD
:10E68000AB0922E0F50AA3E0F50B2274F212154063
:10E690008A088B09ECFEEDFF890A790012E72070E9
:10E6A00003A3E069700479018073750B0190034F37
:10E6B000E065087004A3E06509601F750B00780B26
:10E6C0001219A6A90AEEFCEFFDAA08AB09121EDD7D
:10E6D00074011219CFE9F50B80417900EEFAEFFBD6
:10E6E000121D21EA4B602B8A828B83A3A3A3A3A3D1
:10E6F000A3E05418601C7508FE7509FF780812190C
:10E70000A28A828B83A3A312186512EEA31219CFDB
:10E7100080097901EEFAEFFB121CE5A90B02E4086F
:10E72000121D2D8A0C8B0DA80CA90D90034FE068CB
:10E730002212E738A3A3A322F0850882850983A3C8
:10E74000A322740D1219CF7F040217593400F583E8
:10E7500012EA042212D768E0682212E382121C3DFA
:10E76000227F0A02175974F2121540EAFEEBFF8C61
:10E770000A8D0B8908740E121C12E0F50974FC6EE8
:10E78000700374FF6F7005790002E4087900121DB0
:10E790002D8A0C8B0DAE0CAF0D90034FE06E700305
:10E7A000A3E06F7006E509A2E650DCA90912EE3479
:10E7B000706179007AFE7BFF12EE34705674185542
:10E7C00009700302E89D78007900800312D87E90DA
:10E7D000342B12D875400302E89DE8FAE9FBEA758C
:10E7E000F007A4FAACF075F007EBA42CFB740A2A2E
:10E7F000F582740C3BF583E0541870D0E875F0078F
:10E80000A4F8AAF075F007E9A42AF9740428F874AA
:10E810000C39F988828983A3A3A3A3A3A3E0541886
:10E82000600974185509700302E78788828983EEAE
:10E83000F0A3EFF074FE650A700474FF650B6003CB
:10E8400012E9C188828983A3A3A3A3A3A3E509F046
:10E85000A2E0500D88828983A3A3A3A3A3A3D2E23D
:10E86000F07401650888828983A3A3A3A3A37038E9
:10E87000740112E9E1E054186028903437E4938879
:10E88000828983A3A3A3A312E9AF121F2B8B0DEAE6
:10E89000450D600302E7877800790080397902022C
:10E8A000E78990034EE080D7E06401700302E787B8
:10E8B00088828983A3A3A3A3A3A3E054186007902D
:10E8C0003437E493800490034DE012E5BFE508F08F
:10E8D00002E78712D87E903431E493FAC3E89AE9CC
:10E8E0009400400302E7877A007B00804BEAFCEB50
:10E8F000FDEC75F007A4FCAEF075F007EDA42EFD5D
:10E9000074062CF582740C3DF58312EA52E8FCE99A
:10E91000FDEC75F017A4FC85F00975F017EDA42542
:10E9200009FD74A82CF582740B3DF583E06E70032D
:10E93000A3E06F609E12DA0490342B12D9EB40AD45
:10E9400012E647EC6A7002ED6B7088E875F017A468
:10E95000F8AAF075F017E9A42AF974A828FE740B38
:10E9600039FF7C177D007900EEFAEFFB1222BB8E97
:10E97000828F8312E9C790035C12E9A1A3A3A3A32A
:10E98000A3A3E8F0A3E912E9A77401F0EE240E12A4
:10E99000EA35740112E9CF12130212EA32E802E8F2
:10E9A000CF12DE84A3A322F0EE240F12DACE22F0DF
:10E9B00012E9B8AA0AAB0B2290035CE0FCA3E0FDCD
:10E9C0002288828983A3A3E50AF0A3E50BF022F055
:10E9D000903434E4932401F8E43400F97A027B00A3
:10E9E0002212E5CBA32212D887E822ECFEEDFF909D
:10E9F0003432E493F8E9C3982212EA041223512234
:10EA00003400F583E0FAA3E0FB22E088828983F0FA
:10EA10002212E5F7E8492212E5F385088285098389
:10EA200022F0A30412EA2822F088828983A3A3A3F8
:10EA3000A322EE240DF582EF12DAD1228882898397
:10EA4000E508F0A3E509F02212D6E212DAD122900D
:10EA5000032CE0FEA3E0FF2212E382121EB922740F
:10EA6000F212154089098A0A12E9EB400479008004
:10EA70004075080080020508E508C39509502AE59D
:10EA800008C333F8E433F9EE28F582EF39F583C093
:10EA900082C083121E658A0C8B0DD083D082E06504
:10EAA0000C7004A3E0650D70CDE50A650870BE79B1
:10EAB0000102E40874F6121540E9FE7900121D2DDA
:10EAC000EEF9121D218A088B09A808A909E84960F6
:10EAD0000612F009F98002790402D9F774EE1215D2
:10EAE00040EAFEEBFF890A8C0C8D0B7412121C128B
:10EAF00012DE8912EBA612E9F25051890E750F0051
:10EB00007403780E121ADC743A250EF582740D35F2
:10EB10000FF583E0F8E50CC398502DE50B602475E4
:10EB2000110074037810121ADC74342510F8740D77
:10EB30003511F988828983A3A3A3A3A3A3E50C12AB
:10EB4000EBB0F0790002E761790380F979007AFE91
:10EB50007BFF12EBA6E49365107004790280E6E572
:10EB60000B60E0890E750F007403780E121ADC74C6
:10EB700034250EF8740D350FF988828983A3EEF0E1
:10EB8000A3EF12EBB012E9E1E50C12E5C774FF1236
:10EB9000EEC6E50AF090034DE088828983A3A3A323
:10EBA000A3A3A3A3809C121D1BE9F510903430226F
:10EBB00012F001A3E508F0A3E50922EA2508F58291
:10EBC0002212EBF8F9227A207B009003A9E0F912D7
:10EBD00023032212EC538B09EA450922F08E828F1F
:10EBE00083A3A3A3A322E412D888C32212EBF822A2
:10EBF00012EFF7EB12EBF8223400F583E022749A5F
:10EC000028F582740B39F583E0F42212EBE7223900
:10EC1000F583E02274F4121540750A008002050A9B
:10EC2000903435E493F8E50AC398500D850A08122C
:10EC3000EC3C12E41E70E7E4F002E7477474250828
:10EC4000F582740D227F0C021759F07A2012EC51D4
:10EC5000227B009003A9E0F912240B2274F612150E
:10EC600040E9FC790080010990343012E9F2503912
:10EC7000890875090074037808121ADC743512EBE0
:10EC8000BC740D12ECACE06A7003A3E06B70D88921
:10EC90000875090074037808121ADC743412EBBC8E
:10ECA000740D12ECACE06C70BE02D9F73509F58337
:10ECB0002274F712154089085308407E007F0080B7
:10ECC00056EEF8EFF9E875F007A4F8ACF075F00728
:10ECD000E9A42CF9740428F582740C12EC0F6A7004
:10ECE00003A3E06B702E74FE6A700374FF6B7003F5
:10ECF00002ED85EEF8EFF9E875F007A4F875F00776
:10ED0000E9A42CF9740A28F582740C12EC0F544013
:10ED10006508607112DA0D90342B12EDAA40A21230
:10ED2000EDA57002E96F707674FE6A700374FF6B74
:10ED3000706C7E007F00800312DA0D90342B12ED90
:10ED4000AA505BEEF8EFF9E875F007A4F8AAF075A1
:10ED5000F007E9A42AF9740828F582740C12EC0F64
:10ED600070D6A908EEFAEFFBEA75F007A4FAA8F04E
:10ED700075F007EBA428FB74042AF582740C3B128F
:10ED8000E74E121D09EE75F007A4FEA8F075F00716
:10ED9000EFA428FF74042EFA740C3FFB80047A0061
:10EDA0007B0002DFD712E9E66E2212EBE6EE98EF67
:10EDB000992274F21215408A088B09890B8C0A7902
:10EDC00000121D2DA90A12EE34601988828983A3CE
:10EDD000A3A3A3A3E0650B700B88828983A3A3126E
:10EDE000EA52800A7401650B7045AE08AF0974FEE3
:10EDF0006E700374FF6F603712EE42121F2BEA4BE6
:10EE000060239003D812E66F600C8A828B83A3E0A4
:10EE100060137900801B903434E493F88A828B83EA
:10EE2000E0C39840EDE5086E7003E5096F70BB79AB
:10EE30000102E408121D218A0C8B0DA80CA90DE813
:10EE4000492212E9B8EEFAEFFB2274F4121540EAF7
:10EE5000FEEBFFE9A2E6501B79FF122EA38B0BEA13
:10EE6000450B600990034FE0FAA3E080327AFE7B05
:10EE7000FF802D121C5B8A0A8B0BA80AA90BE8499C
:10EE8000601A88828983A3A3A3A3E0640160D58864
:10EE9000828983A3A3A3A3E0640260C8EEFAEFFB18
:10EEA00002E747790090034F12E9BB8A828B8312F5
:10EEB000EA04121D33740422EE2404F8EF3400F93E
:10EEC00088828983E022F0888289832274EC12157B
:10EED000408A108B11ECFEEDFF7414121C12E0F549
:10EEE0000CA3E0F50D7416121C1212E683E9600CF7
:10EEF00075080078081219A6790B80657900EEFA7A
:10EF0000EFFB121D218A088B09EA4509605B8A82A2
:10EF10008B83A3A3A3A3A3A3E0A2E0504C78101279
:10EF200019A2AC0CAD0DAA0AAB0B121F377402125A
:10EF300019CF8A0A8B0BA80AA90B74FE6870037498
:10EF4000FF696025850882850983A3A312E36A759A
:10EF5000080078081219A6790CAC10AD11EEFAEF82
:10EF6000FB121EDD74011219CF02EC4574F7121565
:10EF7000407804790C7C007D00804D88828983A3D1
:10EF8000A3A3A3A3A3E0A2E0402E88828983A3A326
:10EF9000E06A7003A3E06B701F88828983A3A3A338
:10EFA000A3A3E06401701188828983A3A3A3A3A310
:10EFB000740312EFFD12EFE6EC24010CED3400FDBA
:10EFC000E82407F8E93400F990342BE493FE740147
:10EFD00093FFC3EC9EED9F40A202DFD7EAFEEBFF5A
:10EFE00012EFF112DAD174FEF0A304F022AC82AD7C
:10EFF00083EE12EFF8EF22EA240BF5822212F001E1
:10F0000022F088828983A3A3228882898374FEF0F8
:10F01000A30412F0011412EA21E412E5CBF022C09D
:10F0200082C0837C037D037A3B7B05122B43121C39
:10F030006D02FB1774F412154074F5121A4CE9FEB8
:10F04000EAFF74016E600874026E600302F16FEFF4
:10F05000600874036F600302F1209012447402F0A0
:10F0600090124BE06032E4F0750801F509F50AF5FD
:10F070000B1222C7EA540F240B780812194290058C
:10F08000BE7808121BD39005C27808121BD39012C9
:10F09000587808121BD3806F9005C6E0600D90056C
:10F0A000C7E070079005C6E01480619005C7E4F0E2
:10F0B0009005BE7808121BB59083317808121B1595
:10F0C000E5084509450A450B600E908325121BEFA4
:10F0D0009005BE121BFB80179005BE7808121BB569
:10F0E000740178081219429005BE7808121BD3905B
:10F0F00005BE121BEF9005C2121BFB9005C2121B2E
:10F10000EF901258121BFB9005C67405F090124246
:10F110007403F079009005C2121BEF121C7F804C23
:10F1200074016F704A74016E901244702E740AF06C
:10F130007401121C12E4F07402121C127403F09099
:10F14000830D121BEF7404121C12121BFB740812A5
:10F150001C12E412F8F9121D998024740AF090121E
:10F160005CE0F9901258121BEF121C91E960107CC0
:10F17000E87D037A017B0090054FE0F91223F974D2
:10F180000B02F94274F41215408909900460E0FE04
:10F19000A3E0800F8A828B83A3E509F08E828F83A0
:10F1A00012FC6EFFEE4F60528E828F83A3A312F982
:10F1B0003460E98E828F83A3A3A3E0F5838882A3C2
:10F1C00012F934F5087AD1F91222E5EA4B70C57AC2
:10F1D000027B001222CDEA4B700E7A107B00900564
:10F1E0004FE0F912230380B48A828B8374D1F0A399
:10F1F000E509F0A9081222D980A2121E65900531F6
:10F2000012F8DA121E5F02F94574F4121540890BE8
:10F21000740C121C1212F8EF750A008002050AE540
:10F220000AC3950B502F7D0080010DEDC39C50ED5E
:10F23000E50AC333FEE433FFEA2EF582EB3F12F218
:10F240006AF509ED12F25A65087004A3E0650970C9
:10F25000D979018002790002F945C333FEE433FF16
:10F26000E82EF582E93FF583E022F583E0F508A377
:10F27000E02274F612154012F2F77003A3E06D70ED
:10F280001775085475090578081219A2EEFA1226A6
:10F290001574021219CF801A750802750980780852
:10F2A0001219A28C088D0978081219A212F32012E3
:10F2B00019CF02F33774F612154012F2F77003A358
:10F2C000E06D701775086175090578081219A2EECE
:10F2D000FA12261B74021219CF801A7508037509D9
:10F2E0008078081219A28C088D0978081219A212C8
:10F2F000F3201219CF8040EAFEEBFF12F30FFAA3BE
:10F30000E0F9EA2400FCE439FD900531E06C2212BA
:10F31000F92D12FC2EE0F8A3E0F988828983E0221F
:10F32000EE12FB78EF12FC16FD7C8012F9541226C7
:10F330002D7404221219CF7F0202175974F6121588
:10F340004074FE121A4CEAFEEBFF85188285198381
:10F35000E4F0A3F012F970FA88828983A3A3E0F99C
:10F360007509007508006005C394F14005750882B1
:10F37000802F900531E06A7003A3E06B7020851840
:10F3800082851983AA82AB831221E9E9F5098518E0
:10F390008285198312FB1370087508838003750832
:10F3A0008085188285198312F893A908EEFAEFFB7D
:10F3B000122621E509601485188285198312FB1332
:10F3C000600985188285198312FB1E740202F334CA
:10F3D00074F2121540EAFEEBFF750A00750B00127D
:10F3E000F446121E65EA65087003EB650970121297
:10F3F00021F5E914F50A79017A8A7B051221FB804F
:10F4000003750B8012F94A12F950F50C780C121999
:10F41000A6750C8A750D05780C1219A2780A1219B6
:10F42000A678081219A2E50BF50878081219A61299
:10F43000F90DF582EF12F9097A057B8012262774FF
:10F44000071219CF801412F8E012F8F3888289832A
:10F4500012FCA8F508E439F509227F060217597451
:10F46000F6121540E9FE7F00802F8A828B8312F20C
:10F470006CF9E5082400E439F509EF33F8E433F9D1
:10F48000EC28F582ED39F583E508F0A3E509F0EA0B
:10F4900024020A0AEB3400FB0FEFC39E40CC02F3B8
:10F4A0003774E812154074FB121A4C8A168B1785B4
:10F4B0001882851983E4F07403121C12E4F0A3F09F
:10F4C00004121C12E4F012FB50F50AA3E0F50B85C0
:10F4D0000A82F58312FCA4FEE439FF850A82850BBB
:10F4E00083A3A3E0FA850A82850B83A3A3A3E0F993
:10F4F000EAF508E439F509E50A2404F50AE50B34D0
:10F5000000F50BEEFAEFFB121EC5E96401702C1238
:10F51000FB3C1219A6E4F508F50978081219A2783F
:10F52000081219A69005311218657508807808121E
:10F5300019A612F8AE1219CF02F881EEFAEFFB12FB
:10F540001EC5E9700C900531E06E7003A3E06F708A
:10F55000BE12F8998814602EC333FAE433FB1223E9
:10F560004B7403121C1212F8DA7403121C1212FBF1
:10F570001360137403121C1212F88BA9141225DFE6
:10F580008A0A8B0B800375140012F899880F602A81
:10F59000C333FAE433FB12234B7401121C1212F82A
:10F5A000DA7401121C1212FB13600F7401121C1288
:10F5B00012F88BA90F1225DF8003750F00900460ED
:10F5C000805D850A82850B83A3A3A3A3A3A3A3A322
:10F5D000E4F0A3F0AA0AAB0B851282851383A3A3E0
:10F5E00012F8A912F934F91222D9851082851183F3
:10F5F000E0C0E0851882851983E0F8748A28F582D6
:10F60000740512FB4CD0E012FB0E04F0E515A2E0ED
:10F610005007AA10AB11122351851282851383E083
:10F62000F512A3E0F513E5124513700302F7F9850F
:10F630001282851383A3A312F93460DD85128285BB
:10F640001383A3A3A3A3A3A3A3A3E0A2E050CA850B
:10F650001282851383A3A3A3A312FB1385128285B1
:10F660001383A3A3601F12F934FA790185128285EE
:10F670001383A3A3A3A312F939122FE38A108B11CA
:10F68000751501800F12F8A9A3A3E0F510A3E0F50A
:10F6900011751500E5104511700302F60C851082F6
:10F6A000851183A3E065087004A3E0650960030287
:10F6B000F60C851082851183A3A3A3A3A3A3A31291
:10F6C0001865851082851183A3A3A3A3A3A3E0FCDF
:10F6D0007405121C1212F923A9141225C174021206
:10F6E00019CFE9703C851082851183A3A3A3A3A33E
:10F6F000A3A3A3A3A3121865851082851183A3A3D6
:10F70000A3A3A3A3A3A3A3E0FC7403121C1212F9E6
:10F7100023A90F1225C174021219CFE9700302F652
:10F720000CE50F2514C333240AFA7B001222CD8A7C
:10F730000A8B0BEA450B700302F5EA8A828B83740D
:10F74000D2F0851682851783A3A312F8EF8A828BE5
:10F750008312F9018A828B83A3A3A3A3E51412FC6D
:10F76000AEE50FF0E5146038EA2405FAEB3400FB4F
:10F77000E50A240AF8E50B3400F98A828B8312F932
:10F78000037403121C1212F8CD12199EE514C33330
:10F79000FCE433FD8A828B8312FB251219CF800D86
:10F7A0008A828B83A3A3A3A3A3E4F0A3F0E50F7045
:10F7B0000302F5C2E514C333F8E433F9E50A28F887
:10F7C000E50B39F9E8240AFAE93400FB850A828559
:10F7D0000B83A3A3A3A3A3A3A3A312F8DA74011218
:10F7E0001C1212F8CD12199EE50FC333FCE433FD51
:10F7F00012FB941219CF02F5D4851882851983E083
:10F80000602712FB3C1219A675088A75090578084D
:10F810001219A27403121C1212FB461219A69005AB
:10F82000311218657508008029EEFAEFFB121EC52B
:10F83000E9702A12FB3C1219A675088A7509057829
:10F84000081219A275080078081219A6900531123D
:10F85000186578081219A612F8AE1219CF7403129F
:10F860001C1212FB1360087403121C1212FB1E748C
:10F8700001121C1212FB1360087401121C1212FBFD
:10F880001E74051219CF7F1002175912F893AA0A95
:10F89000AB0B22E0FCA3E0FD22850A82850B83E00E
:10F8A000F8A385820A85830B2212F939A322E51673
:10F8B0002402FCE5173400FDE516240FF582E51758
:10F8C00012F9627A067B80122627740722E0F50C73
:10F8D000A3E0F50D750E00780C22EAF0A3EBF02200
:10F8E00012F92D12FC2E22EE2404FE12FB662212C7
:10F8F000F8F322E0F8A3E0F92212F968AA82AB83B8
:10F9000022A3A3E8F0A3E9F02212F96222EE240276
:10F91000FCEF3400FDEE240F22AC82AD838518820B
:10F9200085198312F92722E0FAA3E0FB22EE2413C3
:10F93000F582EF2212F939E022E0F8A3E0F583889E
:10F9400082221219CF7F04021759EE12FB78EF22A0
:10F9500012FC1622EE2402FAEF3400FBEE240FF51F
:10F9600082EF12FC2EE0F922F0851882851983229D
:10F9700012F30FFCA3E0FBEC2274F612154074E0C6
:10F98000121A4C851882851983AC82AD831225F733
:10F990007402121C12AE82AF83121E5FEEFCEFFDEA
:10F9A000122B3DE9601D121E658A088B09A808A963
:10F9B00009851882851983E0687003A3E0697003E4
:10F9C00002FB09121F557402121C1212F919121EA1
:10F9D000D1E96401700302FB097418121C12AA8297
:10F9E000AB83121E717402121C12AC82AD837418A8
:10F9F000121C12AA82AB83122B3DE96032121E6BDD
:10FA00008A088B09A808A909851882851983E068E6
:10FA10007003A3E069601885188285198312F8EFD6
:10FA200090035212F9037A527B03794B122E3D74E4
:10FA300002121C1212F919121F3D790012F91D123F
:10FA40001D09740B121C12E412FB0EF8A3E0F974EA
:10FA50000C121C1212F903740B121C12AA82AB8333
:10FA6000121C3DE9604B7C087D0079007418121C63
:10FA700012AA82AB831222BB740E121C12AC82AD8E
:10FA8000837418121C12AA82AB83122B3DE96021E9
:10FA90007402121C12AC82AD83740E121C12AA8264
:10FAA000AB831225AF740B121C12AA82AB83121CFB
:10FAB0004F7402121C12AC82AD83740E121C12AA77
:10FAC00082AB831225AF740B121C12AA82AB831275
:10FAD0001C43E96034740C121C1212F8EF85188272
:10FAE000851983E0687003A3E069601D851882852D
:10FAF000198312F8EF740C121C1212F903740B1212
:10FB00001C12AA82AB83121C4F742002F33412F928
:10FB100068E02212FB2C22D083D08202196712F9EE
:10FB2000271223512212F92712FB9422E0F8A3E0B6
:10FB3000F9E849223400F98882898322E51612FB0C
:10FB400078E51712FC2AE0F50878082212FC2A2230
:10FB5000A3F012FB562212FB5A22EA2413F582EB81
:10FB60003400F583E022EF3400FF8E828F83E022A1
:10FB7000F0A3E9F012FC0C22240EF582227F010290
:10FB8000175912FB8622F088828983E022EA241327
:10FB9000F582EB221222AF74032212FB9E22F08E1A
:10FBA000828F83A32274F7121540EA2413F8EB1214
:10FBB000FB34E0FAA3E0F5838A8212FC3312FB8265
:10FBC000F8A3E0F988828983A3E0FA88828983A375
:10FBD00012FC80A312F90402FB7DFAE5093400FB54
:10FBE000122B4322FAA3E0F9EA85088285098322D1
:10FBF0008E828F83E0850882850983A3A3A3A3A3B4
:10FC00002212FC052212FB9E0EAF8322EE24020E6E
:10FC10000EEF3400FF2212FC2EE022F08A828B834A
:10FC2000A3A322E0FAA3E0F9EA2212FC2E22340078
:10FC3000F58322E08C828D832274F61215408C08A5
:10FC40008D0912FC6712FC6E12FC7512FC892402ED
:10FC500012FC93850882850983A3A3A3A3A3A3A36E
:10FC6000A3A3A3F002F33712FB8D12FC2A2212F891
:10FC7000F3E8FEE922FF8E828F83E012FC7F22FAF6
:10FC8000A3E0F9EA8C828D832212FB70EEFCEFFD7B
:10FC9000E5082212FBDA8E828F83A3A3A3A3A3A37A
:10FCA000A3A3E02212FCA82212FC2324002212FCAF
:10FCB000B6A3A3A3A32212FC1BA32274F612154021
:10FCC0008C088D0912FD26850882850983121BFB8D
:10FCD00012F8E7850882850983A3A3A3A312FD4B2D
:10FCE000C39406500512FBF4803885088285098389
:10FCF000A3A3A3A3E064FE600E850882850983A305
:10FD0000A3A3A3E0F4701C12FBF0A312FC0185086E
:10FD100082850983A3A3A3A3E0F4700712FD3BF03F
:10FD2000A3E9F002F33712FD337904EEFAEFFB1288
:10FD300022C12212FB5AFEA3E0FF228E828F83E0B3
:10FD400012FBE4A3A3A3A3A3A3A32212FB9AAE8254
:10FD5000AF8322F075E1E275E1FF02FE3CC008E5E9
:10FD6000A8F8C2AF75C300E5A2F508E5A3F9E8A2BB
:10FD7000E792AFA8087A007B02121302E8F9D008D4
:10FD8000021967C082C083759C019061E47401F020
:10FD900075E1E275E1FFE5A8C2AF759B007591EFD3
:10FDA000A2E792AFE5A8C2AF759B007591F7A2E7F5
:10FDB00092AF02FE3CC082C08312FDDC75E1B875D3
:10FDC000E10F805DC082C08312FDDC75E11775E133
:10FDD0008175E11075E1D275E18180451228E575E4
:10FDE000E1BC22C082C083900B91E012FF65F8C293
:10FDF000AF75C300E5A2F9E5A3FA900B30E09412C9
:10FE00005008E97005EA7002790175C30389A28A76
:10FE1000A3E8A2E092AF12FE9F122AB975E1E18039
:10FE20001B75E11075E1D275E1D975E10175E10944
:10FE300075E1BA75E10175E1C575E1D2D083D08273
:10FE4000021967C082C08312FDDC80DB74F71215D3
:10FE50004012FE9FA2AFE433FEC2AF75C300E5A21D
:10FE6000E5A4FF740F5FF8740F98F5089061E2F055
:10FE7000122AA7900B8C7401F075E1E175C300E5BF
:10FE8000A2E5A46F600FE508C39402400874FF2543
:10FE9000089061E2F0EEA2E092AF7F010217599064
:10FEA00061A4E0D2E4F0E0D2E3F022C082C083900B
:10FEB00061E4E070179061A4E0A2E4500FE0C2E4B6
:10FEC000F0E0A2E3500312291B122AFB02FE3C744D
:10FED000F61215401228DFE9FF900B38E02F24ECD2
:10FEE000F875F01484FE75F014A4C898F80E9061AB
:10FEF000E47402F0EE12FF65FAC2AF75C30388081E
:10FF000075090074097808121ADCF8A909900B30F9
:10FF1000E0C394125006E97003087900E8F5A2E9FD
:10FF2000F5A3EAA2E092AF75E1E275E1FFE5A8C2B0
:10FF3000AF759B007591EFA2E792AF75E1BC75E1DB
:10FF4000B875E1D29061A4E0D2E4F075E1E1122845
:10FF5000DFE9C39F500A9061E2E06E7003E014F0A5
:10FF60007F020217599061E2F075A1FDA2AFE43360
:10FF700022C082C0839061A4E0C2E402FD53C0822B
:10FF8000C0839061A4E0C2E3F0122B1302FE3CC0D8
:10FF900082C0839061A4E0C2E4F09061E4E0700567
:10FFA000122AFB800DE064017005122AF58003120D
:10FFB0002B0702FE3CC082C0837A107B0012234BC9
:10FFC0009004CDEAF0A3EBF07C107D0079001222C2
:10FFD000BB79001220AB7901121D3F79021227DD97
:10FFE0007903122FC37904122EEB79051224AD790F
:10FFF00006122573790712246BD083D08202196709
:020000040001F9
:1000000074F412154074F8121A4C7E008E08900495
:10001000AFE4F07F79750A08750B00780A1219A20F
:100020007402121C12AC82AD837A007B00EFF912CD
:10003000895E1219CF851882851983E0F47003A3B5
:10004000E0F470139004AFE07004EFF080197A01CF
:10005000EFF912235D80107404121C12E0F4700397
:10006000A3E0F46002EFFE0FEFC3947F40A7EE9091
:1000700004AF601EE0600FF91223697A007B00EE86
:10008000F912236F8013EEF9122369EE9004AFF09A
:100090008007E06004F91223697F79AC087A007B5D
:1000A00000EFF91223638B0BEA450B60057508011D
:1000B0007F780FEFC3947F40E2E508A2E050147F01
:1000C000797C007A007B00EFF91223630FEFC39471
:1000D0007F40EE9004AFE0704A7F007A00128128E2
:1000E00064F87004A3E064077004EAFF802AEFC399
:1000F00033F8E433F9128134C082C083128128F8C6
:10010000A3E0F9D083D082C3E098A3E0995002EA3B
:10011000FF0AEAC3940640C574792F9004AFF0F942
:10012000122369790102899CEAC333F8E433F91296
:100130008134E02274A328F582740439F583227493
:10014000F712154074F8121A4CEAFF8518828519C7
:1001500083E4F0A3F0EF60087402121C12E480073D
:100160007402121C1274FF1287BD7A007B001223E6
:100170009374081219CF7F0102175974EE121540BB
:1001800074F8121A4C890C8A0E8B0F8C0D750A08A4
:10019000750B007E007F007508087509007808124D
:1001A00019A27402121C12AC82AD83AA0AAB0BA96D
:1001B0000C12895E1219CF851882851983E0F470BC
:1001C00003A3E0F470030283097402121C12128567
:1001D000CF40087508FC7509FF800D7402121C12CF
:1001E0001285D8F508E9F50974F8C3950AF874077B
:1001F000950BF9C3E89508E99509501AEE2400F823
:10020000EF3408F9E8C3950AFEE9950BFF750A007B
:10021000750B08028309128EC2128324E849700309
:100220000282DFE50E450F604AA80EE50F547FF904
:10023000851882851983E0687003A3E06960030272
:1002400082EFE50F548070137406121C12E0F470F4
:1002500003A3E0F460030282EF80117406121C1203
:10026000E0F47003A3E0F470030282EFAA0AAB0B80
:100270000283207402121C1212932BA90C1285A562
:100280007404121C12E0687003A3E0697046E50D67
:10029000602E7406121C12E0F47003A3E0F4704F99
:1002A000851882851983E0FAA3E04480FB12237548
:1002B000EA4B603B7C019004B0E0F9122381802F6F
:1002C0007406121C12E0F47003A3E0F460217AFFBC
:1002D0007BFF804C7C01AA0AAB0BA90C122381E5A1
:1002E000082408F8E5093400F9EE28FEEF39FFE5A7
:1002F0000A2508F50AE50B3509F50BC3E50A94F85C
:10030000E50B94075003028197E50C1285B1E50ACD
:10031000F0A3E50B128357EEF0A3EFF07A007B0019
:100320007408800E851882851983E0F8A3E0F9220D
:1003300074041219CF7F0A02175974F7121540E995
:10034000FE122801EE1285B17408F0A3E41283575F
:10035000E4F0A3F0028176F074B128F582740339D9
:10036000F5832274EE12154074F7121A4C89088A2C
:100370000A8B0B7E007F00750C01750D00780C1246
:1003800019A27402121C12AC82AD83EEFAEFFB903C
:1003900004AFE0F912895E1219CF8518828519839E
:1003A000E0F460081285C6790002859AEE24010EF9
:1003B000EF3400FFC3940840BE7E087F007401F054
:1003C0009004AFE01285B1E0F50CA3E0F50D750ED9
:1003D00008750F00780E1219A27403121C12AC8259
:1003E000AD83EEFAEFFBA90812895E1219CF7401F2
:1003F000121C12E0F47003A3E0F470030285707421
:1004000003121C121285CF4008750EFC750FFF8079
:100410000D7403121C121285D8F50EE9F50F74F84D
:10042000C39EF874079FF9C3E8950EE9950F500332
:1004300002857074F8C3950CF87407950DF9C3E83C
:10044000950EE9950F500B851882851983E4F0020B
:100450008579EE2408FEEF3400FF7401121C12129D
:10046000832AE849700302855C7401121C12E0655E
:100470000A7004A3E0650B700302855C7403121C10
:1004800012129308EEFAEFFBA90812859F121C12B4
:10049000E0687003A3E069600302855C7407121CC6
:1004A00012E0F47003A3E0F4700B7C00EEFAEFFBB3
:1004B000A90812238175090078091219A6E4F5101C
:1004C000F51178101219A27406121C1212930874F6
:1004D00004121C121288BD9004AFE0F91223AB7411
:1004E000031219CFE97003028447E50C2408F50CC8
:1004F000E50D3400F50D780E1219A2780C1219A230
:100500009004AFE0FCEEFAEFFBA9081223A57404F7
:100510001219CF7403121C121285E912859F121C46
:1005200012E0687003A3E069600302844774051257
:100530001C121285E91223878A108B11A810A911A9
:100540007405121C12E0687003A3E0696003028462
:10055000477401121C121285E91223B7EE250EFE14
:10056000EF350FFFC3EE94F8EF940750030283C0FA
:10057000851882851983E070051285C68014E50A06
:10058000450B700E1287A1A908122369E508900493
:10059000AFF0851882851983E0F97409028332125D
:1005A00085A574052212238D8A108B11A810A9111C
:1005B000221285B522C333F8E433F974A528F582F5
:1005C000740339F583229004AFE0F912236922C342
:1005D000E094FCA3E094FF221285DC22E02403F8DF
:1005E000A3E03400F9E854FC22129308AA0CAB0DE6
:1005F0009004AFE0F92274F4121540EAFEEB800398
:1006000074804FFF7508797C00EEFAEFFBA90812A1
:1006100023638B0BA90BEA496008E5089004B0F04E
:1006200080150508E508C3947F40DCEF548060D056
:100630009004B0E4F0FAFB0289A174EE1215407444
:10064000F6121A4C890A8A0C8B0D8C088D09741CC1
:10065000121C12128ED7C3EC94F4ED94FF400E8559
:10066000188285198374FCF0A374FF801CEC2403AA
:10067000F8ED3400F9E854FC2408F8E93400F98571
:100680001882851983E8F0A3E9F07F007C069004C6
:10069000AFE004FEEEC3947F40027E799004AFE0A9
:1006A0006E602B74872EC333F8E433F9749728F502
:1006B00082740439F5831288BDE4C39AFA74089BE6
:1006C000FB12812F2AFAA3E03B1287AC50080E1CC4
:1006D000EC70C102879AEC700302879AEE128EE1E9
:1006E000FA7408991287AC40030287777510088F57
:1006F0001178101219A27404121C12AC82AD837A04
:10070000007B00EEF912895E1219CF7406121C12DA
:10071000E0F47003A3E0F4700B1287B67A04FBEEEA
:10072000F9122399AA0CAB0DEEF912236FE9606A56
:10073000E50AF50B780B1219A6780E1219A2AC086F
:10074000AD09AA0CAB0D9004AFE0F91223AB740312
:100750001219CFE960059004AFE0FFE50A700AEED8
:10076000850E82850F83F080311287A1EEF9122366
:1007700069EE9004AF80EFE50AF50B780B1219A62D
:10078000780E1219A2AC08AA0CAB0DEEF91223AB2D
:1007900074031219CFE96002EEFFEFF9740A0283C5
:1007A000327A019004AFE0F912235D22FB12832418
:1007B000C3EA98EB9922851882851983E4F0A31285
:1007C0008EFA2274F212154074F8121A4C89098CB0
:1007D00008EA24F8F50AEB34FFF50B750C08750DE3
:1007E00000780C1219A27402121C12AC82AD83AAFA
:1007F0000AAB0B12895E1219CFE50870237406123A
:100800001C12E4F0A3F07404121C12AC82AD83E558
:100810000A2404FAE50B3400FBA90912239380197A
:100820007402121C12128EEB1287B6AA0AAB0BA925
:1008300009122393E50912884374081219CF7F0621
:10084000021759C333F8E433F974B128F5827403FD
:1008500039F583E02EF0A3E03FF02274F412154046
:1008600074FE121A4C851882851983ECF0A3EDF002
:100870008908EAFEEBFFEE24FCFEEF34FFFF85184B
:1008800082851983AC82AD83EEFAEFFB1223997552
:100890000A02750B00780A1219A27402121C12AC1B
:1008A00082AD83EEFAEFFBA90812895E1219CF859B
:1008B00018828519831288BD740202899EE0FAA30A
:1008C000E0FB2274F012154074FC121A4C890C8A59
:1008D0000A8B0BECFEEDFF750800750900EE240392
:1008E000F50EEF3400F50F7402780E121BC4AE0E35
:1008F000AF0F128CA56049750E04750F00780E12AB
:1009000019A27402121C12AC82AD83AA0AAB0BA905
:100910000C12895E1219CFE50A2404F50AE50B349E
:1009200000F50B7800880E128B4FE0FAE5082AF5E7
:1009300008E5093400F50908E8C3940450B480E5DB
:10094000AA08AB0974041219CF7F08021759E5826F
:100950002510FCE5833400FDAA0CAB0DA90E12276F
:10096000F574022274F4121540E9FE750801750948
:100970000078081219A28A088B0974027808121BE1
:10098000C48E0AF50B7409780A121ADCE5082400F3
:10099000FAE509350BFB1227FB0288B87408121917
:1009A000CF7F0402175974F712154074FC121A4CC9
:1009B0008C828D83E0851882851983F08C828D83EB
:1009C000A3E0C0E07401121C12D0E0F07402121C0B
:1009D0001274FFF07403121C1274FF128EF61223AD
:1009E00093740402817374EE12154074FC121A4C55
:1009F0008909EAFEEBFF8C0C8D0D7416121C121285
:100A00008ECFEE5403F508606A74FC5EFE750E042A
:100A1000750F00780E1219A27402121C12AC82AD6E
:100A200083EEFA12895E1219CFE50C450D60298517
:100A30000A82850B83E0C0E085080E128B4FD0E060
:100A4000128B620508E50C24FFF50CE50D34FFF56B
:100A50000DE508C3940440D1851882851983AC82C2
:100A6000AD83EEFAEFFBA909122393EE2404FEEF07
:100A70003400FFE50C5403F508850C0E850D0F744A
:100A800002780E121BC4850E0C850F0DE50C450D6A
:100A9000604D780C1219A2AC0AAD0B8E0E8F0F743C
:100AA00002780E121BC4850910F511740978101212
:100AB0001ADCE50E2400FAE50F3511FB1227FB7452
:100AC000021219CF7402780C121ADCA80CA90DEED0
:100AD00028FEEF39FFE50A28F50AE50B39F50BE5A5
:100AE000086069750E00750C04750D00780C1219FC
:100AF000A27402121C12AC82AD83EEFAEFFBA909BC
:100B000012895E1219CF8025850A82850B83E0C089
:100B1000E0850E0C851882851983E582250CF58207
:100B2000E5833400F583D0E0128B62050E85080C56
:100B300074FF250CF5080470CF851882851983ACE5
:100B400082AD83EEFAEFFBA909122393028330856D
:100B50001882851983E582250EF582E5833400F538
:100B60008322F0850A82850B83A385820A85830B05
:100B70002274EE12154074FC121A4C890E8A0C8BEA
:100B80000D8C0B7416121C12E0F508A3E0F5097425
:100B900018121C12E0FEA3E0FFE5085403F50A60FA
:100BA00060F510C3E5089510F508E5099400F5090E
:100BB00075100475110078101219A27402121C121B
:100BC000AC82AD83AA08AB09A90B12895E1219CFBA
:100BD000EE4F602A75100178101219A2850A107460
:100BE00002121C1212894E1219CF128CB4050AEE91
:100BF00024FF1EEF34FFFFE50AC3940440D2128C99
:100C0000C1EE5403F50A8E108F1174027810121B76
:100C1000C4AE10AF11802975100475110078101240
:100C200019A27402121C12AC82AD831289581219D7
:100C3000CFE50C2404F50CE50D3400F50D128CC144
:100C4000128CA570D2E50A60597E007510048E11D1
:100C500078101219A27402121C12AC82AD83AA0879
:100C6000AB09A90B12895E1219CF80197510017892
:100C7000101219A28E107402121C1212894E12192F
:100C8000CF128CB40EAF0A74FF2FF50A0470DD8505
:100C90001882851983AC82AD83AA08AB09A90B120F
:100CA0002393028330EEF8EFF9E824FF1EE934FFC6
:100CB000FFE84922E50C2401F50CE50D3400F50DA3
:100CC00022851882851983AC82AD83AA08AB09A955
:100CD0000B122393E5082404F508E5093400F5090F
:100CE0002274EC12154074F8121A4C89088A108B81
:100CF00011ECFEEDFF741C121C12128ED7741E1222
:100D00001C12E0F50CE91285B1128ECF7509008531
:100D10001882851983EAF0A3EBF07402121C12EE1C
:100D2000F0A3EF128EF6AA0AAB0BA9081223937553
:100D3000120875130078121219A27402121C12AC58
:100D400082AD83AA0AAB0BA90812895E1219CF855E
:100D50001882851983E065107004A3E065116003B3
:100D6000028E6B7402121C12E06E7003A3E06F60BF
:100D700003028E6BE50C7003028E49850E82850F8F
:100D800083EEF8EFF9E85403F50CE582458370151E
:100D9000E875F0FFA4F8AAF075F0FFE9A42AF9E8D5
:100DA000FAE9FB80207A007B00800AE0FCEA2CFA5A
:100DB000EB3400FBA3E8FCE9FDEC24FF18ED34FF65
:100DC000F9EC4D70E6E50C601E7404C3950CF895C3
:100DD000E0F9E875F0FFA4F8ACF075F0FFE9A42C99
:100DE000F9EA28FAEB39FB7404121C12EAF0A3EBBF
:100DF000F0128EC2E50E450F6017780E1219A2EEA2
:100E0000FCEFFDAA0AAB0BA90812239F740212196A
:100E1000CFEEFCEFFDAA0AAB0B12931D7404121C5B
:100E200012E0687003A3E06970227404121C1212AD
:100E300093557404121C12E0687003A3E069700CEF
:100E400085188285198312934E7509017402121C4C
:100E500012C3E094F4A3E094FF40067EFC7FFF8081
:100E6000437402121C12128EEB80397402121C128F
:100E7000C3E094F4A3E094FF40067EFC7FFF80086B
:100E80007402121C12128EEB128EDFF8740899F99C
:100E9000C3E89EE99F5008128EDFFE740899FFE5B3
:100EA00008128843E508C333F8E433F974A528F53C
:100EB000827403128850A90974081219CF7F0C029A
:100EC0001759E50A2408F50AE50B3400F50B22E072
:100ED000F50AA3E0F50B22E0F50EA3E0F50F22E5FD
:100EE000081285B512832AE4C398221285DC2408EF
:100EF000FEE93400FF22128EFA22F085188285194D
:100F000083AC82AD8322C082C0837900E9C333FC05
:100F1000E433FD74E22CF58274823DF583E06A705F
:100F200003A3E06B600709E9C3940340DFD083D0DB
:100F30008202196774F6121540E9FE8A088B09ECE3
:100F4000FAEDFB129026500E12902FEE12903BE518
:100F500008F0A3E509F07F02021759C082C083128E
:100F6000235780C974F2121540EAFEEBFF8C088DFE
:100F700009740E121C12128ECF794E1227C5E97019
:100F800004790A8037EEFAEFFB122375EA4B601002
:100F9000EEFCEFFD9004B0E0F91223B77900801C5D
:100FA000780A1219A2AC08AD09EEFAEFFB7901122A
:100FB000237B74021219CFE960C7790902883E7455
:100FC000F412154074F8121A4CEAFEEBFF12902648
:100FD000503F12902FE09004B012903B1288BD75E4
:100FE0000A08750B00780A1219A27402121C12ACBE
:100FF00082AD83EA24F8FAEB34FFFB9004B0E0F909
:1010000012895E1219CF7402121C121288BD028955
:101010009CEEFAEFFB1223758B0BA90BEA4970BF0C
:101020007A007B0080E81223B1E9F8C394032274AC
:10103000B128F58274043400F58322F0E81290415F
:1010400022C333F8E433F974B428F582740439F513
:10105000832274E812154074F5121A4C8A168B1705
:101060008C0C8D0D7423121C12E0F512A3E0F51305
:10107000751100794E1227C5E97005790A0292FEB2
:10108000E512451370030292FCAA16AB17122375E2
:101090008A088B09A808A909880A890B7401121CFF
:1010A00012E8F0A3E9F09004B0E0F510E8450B7009
:1010B0000579090292FE7508087509007808121969
:1010C000A27405121C12AC82AD83EA24F8FAE9344A
:1010D000FFFBA91012895E1219CF7405121C12E5CC
:1010E0000C2512F8E50D3513F9C3E098A3E09940FB
:1010F0008A12930E121C12128ED7AE12AF137508FD
:1011000000807175140175150078141219A274020B
:10111000121C12AC82AD83AA0AAB0BA91012895E15
:101120001219CF851882851983E0F8850E82850F04
:1011300083E06860267508017407121C12C3E098EA
:10114000F0A3E09400F0850E82850F83E0F8740729
:10115000121C12E028F0A3E03400F0E50A2401F5A7
:101160000AE50B3400F50B850E82850F83A385827B
:101170000E85830F128CA5708AE508A2E040030259
:1011800092FC851882851983E4F08582088583099D
:1011900078081219A27407121C12129308AA16AB2F
:1011A00017790012237B74021219CFE9F508700336
:1011B0000292A67405121C121285CF40067EFC7F97
:1011C000FF800B7405121C121285D8FEE9FF1293E2
:1011D000337409121C12E0F47003A3E0F4700A7C6B
:1011E000007401121C12129343780C1219A2780A8F
:1011F0001219A2AC087405121C121288BDA9101293
:1012000023A574041219CF12930E121C1212186522
:10121000AC12AD13AA0AAB0BA90812239F740212D9
:1012200019CF7405121C12E0C3950CF8A3E0950DBC
:10123000F9E8C39512F50EE99513F50F780E12191A
:10124000A2E50A2512F50AE50B3513F50B780A120B
:1012500019A2AC087405121C12E0250CF8A3E035A5
:101260000DF9E82512FAE93513FBA9101223A5742C
:10127000041219CF1293337405121C1212932B12FD
:10128000931D7407121C12E0687003A3E0697016C6
:101290007407121C121293557407121C12E0687026
:1012A00003A3E069600575110A80087403121C121B
:1012B00012934E851882851983E060266510700BA5
:1012C000740A651170051285C680171287A18518EA
:1012D000828519831285C9851882851983E0900457
:1012E000AFF0851882851983E06510600F740A6578
:1012F0001160097C01EC121C12129343A911740BAA
:101300001219CF7F10021759E0FCA3E0FD22E50A75
:10131000250CF50AE50B350DF50B742522A90812ED
:10132000238D8A0C8B0DA80CA90D22129308AA0AF2
:10133000AB0B22E5081285B5E0C39EF50AA3E09F3A
:10134000F50B22E0FAA3E0FBA910122381221293ED
:10135000641223B7221293641223878A0C8B0DA880
:101360000CA90D22E0FCA3E0FDAA0AAB0BA9082200
:1013700074F0121540EAFEEBFF8C0A8D0B7410120C
:101380001C12E0F50CA3E0F50D7412121C12E0F52E
:1013900008A3E0F50912902650278882AE82780CC7
:1013A0001219A2AC08AD09EE129041E0250AFAA389
:1013B000E0350BFB74B12EF58274043400F58380A4
:1013C00023EEFAEFFB122375EA4B7004790A801EB4
:1013D000780C1219A2AC08AD09EA250AFAEB350B14
:1013E000FB9004B0E0F912895E1219CF79000289EE
:1013F00049C082C083791C7AE07B81122BBB029B9F
:101400008E74F7121540E9FE74016E7005122525E1
:10141000800312252B02999F74ED1215408A088BC8
:10142000098C0A8D0B7413121C1212970F603F1255
:1014300096FEE41296E9121C12A982AA8389108AE8
:1014400011751200781012199E129C6F1219CF8E0E
:10145000828F83A3A3A3A3A37415129624A3129926
:10146000A78E828F83E8F0A3E912973A8002790170
:101470007F0B02175974F1121540EAFEEBFFEE24C0
:1014800060F582EF12A3EA2403F50A7ACD7B0612F7
:101490009E2E6058129685E8FAE9FB900AAB1296E8
:1014A0008E1294F37402F0EE245EF582EF12A3EA3A
:1014B000F50CA3E0F50D750E00780C12199EEE24C4
:1014C00060F582EF12A3EAFC7D00EA24030A0A0A0F
:1014D000EB129C7A1219CF850882850983A3A3A3F6
:1014E000A3A3E50A129E3F12973F800279047F076B
:1014F000021759E8F0A3E9F08A828B832274F21272
:1015000015407AAE7B091227BF8A088B09EA450984
:1015100070030295DF129685880A890B8A828B8375
:10152000A3A312A52D8A0C8B0DAE0CAF0DEE4F7040
:10153000030296161226DBE97023850A82850B8347
:10154000A3A3A3A3A3E06003029616850A82850BDA
:1015500083A3A3A3A3A3A3E06003029616EE24141F
:10156000F582EF12A3EA6003029612900AAB129979
:10157000A7850A82850B83A3E8F0A3E9F0850A8298
:10158000850B837403F0A3A3A3A3A3E07018850ABB
:1015900082850B83A3A3A3A3A3A3E070098E828FEC
:1015A00083A3E4F080068E828F83A3E0850A828580
:1015B0000B83A3A3A3129624E0F9E5082406FCE517
:1015C000093400FDAA08AB091224958A0A8B0B780E
:1015D0000A12179F010002DF95E39503960796799B
:1015E00000803C750A00780812199E7C4F7D00EE41
:1015F000240FFAEF129C7A1219CF7AAE7B091227C8
:10160000AD80DC790B80187AAE7B091227AD792486
:10161000800D790A80097AAE7B091227AD79207F87
:1016200006021759129E68A3A3A32274F61215404E
:10163000EAFEEBFF7ACD7B061227B9EA4B60411236
:101640009685129A6B88828983A3ECF0A3EDF088CB
:10165000828983740412974BE088828983A3A3A3B1
:10166000129735740412A3CF129B588E828F83A3D6
:10167000A3A3A312968EA3A31294F312973D800204
:101680007905029B53EA2406F8EB3400F922129BF9
:1016900061A32274ED1215408A088B098C0A8D0B08
:1016A0007413121C1212970F603A1296FE740112F4
:1016B00096E9121C12A982AA8389108A1175120058
:1016C000781012199E129C6F1219CF8E828F83A3ED
:1016D000A3A3A3A3741512974BE508F0A3E5091281
:1016E000973A80027902029470F0A3E50AF0A3E52C
:1016F0000B12972CE50CF0A3E50DF0741522EE24E7
:1017000006F8EF3400F9880E890F8882F5832212DB
:10171000971D8A0E8B0FAE0EAF0FEE4F22E0F50C29
:10172000A3E0F50D7ACD7B061227B922F0888289D5
:1017300083A3A3A322129AD4A32212974BA3A3E4B8
:10174000F07ACD7B061227B3790022F08E828F8348
:101750002274F5121540EAFEEBFF7ACD7B061227C4
:10176000B9EA4B6027EE240FF508EF3400F5097550
:101770000A00780812199E7C4F7D00129C81121974
:10178000CF7ACD7B061227B37900800279037F03DD
:1017900002175974F61215407ACD7B061227BFEA5C
:1017A0004B602A8A828B83A3A3A3A3A3E0F9EA2434
:1017B00006FCEB3400FD1224958A088B0978081288
:1017C000179F010002CD97D297CD97D2977900024B
:1017D0009B537ACD7B061227AD80F2C082C083EA8C
:1017E0004B700479FF800E900680E06A7003A3E0DE
:1017F0006B70F07900029B8E74F7121540EAFEEBD5
:10180000FF8908EE4F700479FF802312987D701EC7
:101810007900900680129BD9EA4B7011900680EEF9
:10182000F0A3EFF0E508A3F0A3E4F080010902992A
:101830009F74F612154012987D603F890875090063
:1018400074027808121ADC74802508FA74063509C7
:10185000FB8A828B83A3A3E0F88A828B83A3A3A352
:10186000E0C3985013890875090074027808121AA9
:10187000DC1298A804F0800279FF029B5312268D97
:1018800074FF692274F612154012987D601789085A
:1018900075090074027808121ADC1298A860041402
:1018A000F0800279FF029B5374832508F582740649
:1018B0003509F583E022C082C0838A828B83A3A38B
:1018C000E4F0A3129AD012991F12991FA3A3041235
:1018D00094F7A3E41294F774FFF0A3A3A3A3A3A324
:1018E000A3A3A3E4F0EA240B129927E4129AE2A33B
:1018F000A3A3A3F0EA240C129FEA240D129FEA127C
:1019000099257401F0EA2414129FEA245E12992E9C
:101910002460129FEA246112992E2463029B89F0AD
:10192000A3129AE622240EF582EB12A41922129F2A
:10193000EFA3F0EA22C082C083900624E0601290F8
:101940000620E06A7003A3E06B70067A1C7B0680B9
:10195000047A007B00029B8E74F7121540EAFEEBBE
:10196000FF1299A4EE687002EF697007900AADE467
:10197000F0A3F08E828F83129BD712269FEE240E47
:10198000F582EF12A3EAF912265DEEFAEFFB1226BA
:10199000A58E828F83A3A3A3A3A3A3A3A3E4F07F15
:1019A00001021759900AAD1299AB22E0F8A3E0F9B1
:1019B0002274F6121540EAFEEBFF900624E0701F39
:1019C0001226AB8B09EA450970157A1C7B06122694
:1019D000A5900620EEF0A3EFF07A1C7B0680047A37
:1019E000007B00029B5374F21215408A0A8B0BECA9
:1019F000FEEDFFEE4F70067A007B00806BEEFAEF93
:101A0000FB122699E9F460EFAA0AAB0B1226B78AFB
:101A1000088B09EA45097009EEFAEFFB12269F8050
:101A2000D68A828B83A3A3EEF0A3EFF07401650A3C
:101A30007002E50B8A828B83A3A3A3A3A3A37003E5
:101A4000E4800274FFF0A3F090829374101218697E
:101A5000900AA9121865129A6B1226637412121951
:101A6000CFE97093AA08AB0902961F900AAB129CAB
:101A7000952274F21215408A0A8B0B8C088D09741A
:101A80000E121C12129E39EE4F70067A007B0080F7
:101A90003CEEFAEFFB122699E9F460EFAA08AB09D5
:101AA0001226B7EA4B7009EEFAEFFB12269F80DB95
:101AB0008A828B83A3A3EEF0A3EF129AD0E508F0FD
:101AC000A3E509129AE2E50AF0A3E50BF002961FDE
:101AD000129AD422129AD822F08A828B83A3A3A3CB
:101AE000A322129AE622129AD8A3A32274F71215FF
:101AF000401299A4E8496042129B4B129E39900A09
:101B0000ADE0240EF8A3E03400F988828983E0F97F
:101B100012265D900AAD129BD91226A5129B3F7426
:101B200001F0A3E4F0129B3FA3A3E4F0A3F0129B07
:101B300045EEF0A3EFF079008002790102999F123F
:101B40009B45A3A322900AADE0F8A3E0F583888229
:101B5000A3A3227F02021759129B61E8F0A3E9F0C8
:101B600022E0F8A3E0F98A828B8322C082C083EA54
:101B70004B60128A828B83A3A3A3A3A3A3A3A3E096
:101B8000543FF9800279008005129927E4F0D08350
:101B9000D082021967C082C083900AAD129BD9120D
:101BA0009BC7600574046870047901800279008025
:101BB000DDC082C083129BC760057404687004791D
:101BC000018002790080C71226CFE9F874036822E9
:101BD0007A847B06021967A3A3E0FAA3E0FB2274D0
:101BE000F1121540ECFEEDFF129C878E828F83125E
:101BF000A3DF24FDF5088E828F83A3A3129C5E12BF
:101C0000199EAC087D00EE2403FAEF129C7A12199B
:101C1000CF0294EE74F11215408C088D09129C8746
:101C200085088285098312A3DF24FDF50AE50824CF
:101C300002FEE5093400FF8E828F83E50A129C5E66
:101C400012199EAC0A7D00E5082404FAE509129CED
:101C50007A1219CF8E828F83E004F00294EE1297ED
:101C60002CA982AA83890C8A0D750E00780C227C1F
:101C7000107D00E50E2405FAE50F3400FB129C816F
:101C8000221222AF74032212A413129B61A3A3A3F6
:101C9000A3129C9522E0FCA3E0FD2274E9121540FA
:101CA0008C0A8D0B890D7417121C12E0F87418122F
:101CB0001C12E0F514A3E0F515741A121C12E0F5DD
:101CC0000CC3944340057921029DAE74FF6A7003F2
:101CD00074FF6B7005790E029DAEE8602A1226D55E
:101CE000E9701C850A82850B83A3A3E0700C850A2A
:101CF00082850B83A3A3A3E060057920029DAE90AB
:101D00000AAD129E39802C1226AB8A088B09AE08C8
:101D1000AF09EE4F60E41226DBE97017850A828571
:101D20000B83A3A3E070D3850A82850B83A3A3A3AF
:101D3000E070C7E50D607C7AAE7B09129E2E60864E
:101D4000EA2406F50EEB3400F50F850A10850B1119
:101D5000751200781012199E7C047D00E50E240394
:101D6000129C771219CF850E82850F83A3A3A3A39C
:101D7000E0C2E6F0851410851511781012199E85C1
:101D80000C0AAC0A7D00E50E2407129C771219CFCD
:101D90007407250C850882850983A3A3A3A3A31236
:101DA0009E3F7401F07AAE7B091227B379007F0F52
:101DB0000217597403250C900686F0850A82850B5C
:101DC00083A3A982AA8389088A09750A0078081260
:101DD000199E7C037D007A877B06129C811219CFA5
:101DE000900687E0D2E6F0751600781412199E85E9
:101DF0000C08AC087D007A8A7B06129C811219CFF0
:101E0000900686E0F8EE245EF582EF12992A748738
:101E1000F0A37406F0EE2460F582EF12992AE8F040
:101E2000EEFAEFFB122669E96082790380801227BF
:101E3000B98A088B09EA450922E0FEA3E0FF2212D5
:101E4000A3D3129E5EE8F0A3E912974BA3A3A3A32A
:101E5000129E5EA3A3A3E8F0A3E9129E6822129942
:101E6000AB85088285098322F0850882850983A3D2
:101E7000A32274F6121540E9FE8A828B83A3E090B8
:101E80000687F0EEA3F0A3E4F0A3F0A37407F0A399
:101E9000E4F075080278081219A675088B75090612
:101EA00078081219A275080078081219A679017C21
:101EB000877D068A828B83A3A3129BD71226F37495
:101EC000041219CF029B53C082C0838A828B83A3E2
:101ED000E064FE8A828B83A3700474018002E004B4
:101EE000029B8D74F7121540EAFEEBFF908293740B
:101EF00010121869900AA912186512A4481219CF75
:101F0000E96004790280127901EEFAEFFB1226F9FA
:101F1000E9600479038002790002999F74F6121532
:101F20004012A3FE8E828F83A3740112974BE4F0BC
:101F300012271D850882850983A3A3A3A3E0A2E03D
:101F400050168E828F83A3E4F0F9EEFAEFFB12268F
:101F5000F9E9601279038010EEFAEFFB122675E9B9
:101F600070F212A3EFF07900029B53C082C083EAA3
:101F70001299257402F01299A4EA687002EB696064
:101F8000051226B180031226C97900029B8EC082F9
:101F9000C083EA241412A3E7603BEA240B12A3E7F0
:101FA00004F0C3940F402EEA240C12A3E7C3940557
:101FB00040151299A4EA687002EB6960051226B117
:101FC00080131226C9800EEA240B129FF912A3E790
:101FD00004F0122681029B8EC082C083EA240B1279
:101FE0009FEA2414129FF9029B89129FEFEA22F5BF
:101FF00082EB3400F583E4F022129FEFEA240C22F6
:10200000E9601114600E1460221460131460261429
:10201000602B8013EAC39405400D790002196774A0
:10202000F92AC3944340F3790180F174FA2AC394E6
:102030004440E780F2EAC3940440EC80DDEAC394B4
:102040000780F674F6121540740A121C12129E399B
:10205000EB900AA970087402F0A374208004EAF0DF
:10206000A3EBF074FF6C700374FF6D900AAB700704
:102070007401F0A3E48004ECF0A3EDF0900AADE469
:10208000F0A3F07A1C7B061226A5900624E4F090BB
:102090000680F0A3F0A3F0A3F075084FF5097808C7
:1020A0001219A275089C75090978081219A27909F4
:1020B0007CD57D067ACD7B061227A174041219CF38
:1020C00075084F75090078081219A27508A37509DB
:1020D0000A78081219A279037CB67D097AAE7B09C9
:1020E0001227A174041219CFEF601C7901EEFAEFE8
:1020F000FB122693EEFCEFFD7A017B001226BD90C9
:102100000AADEAF0A3EBF07CC87D007A017B0012F7
:102110002471029B5374F612154012A3FEEE246341
:10212000F582EF12A3EAFA8E828F83A3A3A3A3A35F
:10213000A3A3A3E0543F14601414700302A2041478
:10214000700302A2A014700302A2A08040888289BA
:1021500083E0600C14604C24FC700302A1F4802D19
:1021600012A50870288E828F83A3A3A3A3E0F47026
:1021700003A3E0F4700D12A42F7003A3E0697012A2
:1021800012A41EEEFAEFFB122705E96047790D0253
:102190009B538E828F83A3A3A3A3A3A374FFF0A357
:1021A000F080EA790112A50A70E38E828F83A3A3DF
:1021B000A3A3E0F47003A3E0F4700D12A42F700346
:1021C000A3E06970CD12A41E7901EEFAEFFB12268E
:1021D000F9E970B98E828F83A3A3A3A3A3A3A3A3BA
:1021E000A3A3E4F0EE2408F582EF12A3EA54C0445E
:1021F00002F08050790512A50A7092EEFAEFFB12F8
:102200002711808988828983E0600A24FD603A145E
:10221000606F02A18D12A508600302A18D12A42F88
:102220007003A3E069600302A18D90829374101281
:102230001869900AA912186512A4481219CFE9600A
:102240000302A18D790002A18F790312A50A600310
:1022500002A18D850882850983A3A3A3E060030200
:10226000A18DEEFAEFFB12270BE9600302A18D8E20
:10227000828F83A3A3A3A3A3A3A3A3A3A3E402A1E5
:10228000F1790412A50A600302A18D8508828509EF
:1022900083A3A3A3E070ADEEFAEFFB12271D80A489
:1022A00088828983E0601514605914606314700398
:1022B00002A33C14700302A39D02A18D12A5086025
:1022C0000302A18D12A42F7003A3E069600302A191
